S01800004762544D6F64756C65535733305765622E737265637E
S3150800800000000120D9E70008DDDF0008E5DF0008E9
S31508008010EDDF0008F5DF0008FDDF000800000000BE
S3150800802000000000000000000000000005E0000855
S3150800803011E00008000000001DE0000829E0000823
S3150800804029E8000829E8000829E8000829E80008BE
S3150800805029E8000829E8000829E8000829E80008AE
S3150800806029E8000829E8000829E8000829E800089E
S3150800807029E8000829E8000829E8000829E800088E
S3150800808029E8000829E8000829E8000829E800087E
S3150800809035E0000829E8000829E8000829E800086A
S315080080A029E8000829E8000829E8000829E800085E
S315080080B029E8000829E8000829E8000829E800084E
S315080080C029E8000829E8000829E8000829E800083E
S315080080D029E8000849E000085DE0000871E00008AA
S315080080E029E8000829E8000829E800080000000037
S315080080F00000000000000000000000000000000072
S31508008100000000000000000029E8000829E800082F
S3150800811029E8000885E0000829E8000829E8000899
S3150800812029E8000829E8000829E8000829E80008DD
S3150800813029E8000829E8000829E8000899E0000865
S3150800814029E80008ADE0000829E8000829E8000841
S315080081500000000000000000000000000000000011
S315080081600000000000000000000000000000000001
S3150800817000000000000000000000000000000000F1
S3150800818000000000000000000000000000000000E1
S3150800819000000000000000000000000000000000D1
S315080081A000000000000000000000000000000000C1
S315080081B000000000000000000000000000000000B1
S315080081C000000000000000000000000000000000A1
S315080081D00000000000000000000000000000000091
S30D080081E05FF8E0F166666666C9
S315080081E810B5054C237833B9044B13B10448AFF3DB
S315080081F800800123237010BD5002002000000000F3
S315080082086065010808B5034B1BB103490348AFF37A
S31508008218008008BD000000005402002060650108BF
S31508008228034613F8012B002AFBD1181A01387047A0
S3150800823881F0004102E000BF83F0004330B54FEA01
S3150800824841044FEA430594EA050F08BF90EA020F6E
S315080082581FBF54EA000C55EA020C7FEA645C7FEA01
S31508008268655C00F0E2804FEA5454D4EB5555B8BF24
S315080082786D420CDD2C4480EA020281EA030382EA95
S31508008288000083EA010180EA020281EA0303362D27
S3150800829888BF30BD11F0004F4FEA01314FF4801CFA
S315080082A84CEA113102D0404261EB410113F0004F0C
S315080082B84FEA03334CEA133302D0524263EB4303C3
S315080082C894EA050F00F0A780A4F10104D5F1200E61
S315080082D80DDB02FA0EFC22FA05F2801841F10001BC
S315080082E803FA0EF2801843FA05F359410EE0A5F190
S315080082F820050EF1200E012A03FA0EFC28BF4CF0C1
S31508008308020C43FA05F3C01851EBE37101F0004576
S3150800831807D54FF0000EDCF1000C7EEB00006EEB83
S315080083280101B1F5801F1BD3B1F5001F0CD349080D
S315080083385FEA30004FEA3C0C04F101044FEA445264
S3150800834812F5800F80F09A80BCF1004F08BF5FEAEB
S31508008358500C50F1000041EB045141EA050130BDCB
S315080083685FEA4C0C404141EB0101013C28BFB1F5DD
S31508008378801FE9D291F0000F04BF01460020B1FA28
S3150800838881F308BF2033A3F10B03B3F120020CDAFB
S315080083980C3208DD02F1140CC2F10C0201FA0CF0D9
S315080083A821FA02F10CE002F11402D8BFC2F1200C3E
S315080083B801FA02F120FA0CFCDCBF41EA0C019040F4
S315080083C8E41AA2BF01EB0451294330BD6FEA04043D
S315080083D81F3C1CDA0C340EDC04F11404C4F1200228
S315080083E820FA04F001FA02F340EA030021FA04F33A
S315080083F845EA030130BDC4F10C04C4F1200220FA91
S3150800840802F001FA04F340EA0300294630BD21FACE
S3150800841804F0294630BD94F0000F83F4801306BF94
S3150800842881F480110134013D4EE77FEA645C18BF88
S315080084387FEA655C29D094EA050F08BF90EA020F1F
S3150800844805D054EA000C04BF1946104630BD91EA17
S31508008458030F1EBF0021002030BD5FEA545C05D11A
S315080084684000494128BF41F0004130BD14F5800459
S315080084783CBF01F5801130BD01F0004545F0FE41CD
S3150800848841F470014FF0000030BD7FEA645C1ABF02
S31508008498194610467FEA655C1CBF0B46024650EA39
S315080084A8013406BF52EA033591EA030F41F4002165
S315080084B830BD00BF90F0000F04BF0021704730B5EB
S315080084C84FF4806404F132044FF000054FF00001C0
S315080084D850E700BF90F0000F04BF0021704730B581
S315080084E84FF4806404F1320410F0004548BF404256
S315080084F84FF000013EE700BF42004FEAE2014FEAAB
S3150800850831014FEA02701FBF12F07F4393F07F4F85
S3150800851881F06051704732F07F4208BF704793F088
S315080085287F4F04BF41F40021704730B54FF460749B
S3150800853801F0004521F000411CE700BF50EA01029E
S3150800854808BF704730B54FF000050AE050EA010247
S3150800855808BF704730B511F0004502D5404261EBB7
S3150800856841014FF4806404F132045FEA915C3FF4F8
S31508008578D8AE4FF003025FEADC0C18BF03325FEA95
S31508008588DC0C18BF033202EBDC02C2F1200300FA46
S3150800859803FC20FA02F001FA03FE40EA0E0021FA6B
S315080085A802F11444BDE600BF70B54FF0FF0C4CF459
S315080085B8E06C1CEA11541DBF1CEA135594EA0C0F0B
S315080085C895EA0C0F00F0DEF82C4481EA030621EA46
S315080085D84C5123EA4C5350EA013518BF52EA033581
S315080085E841F4801143F4801338D0A0FB02CE4FF033
S315080085F80005E1FB02E506F00042E0FB03E54FF063
S315080086080006E1FB03569CF0000F18BF4EF0010E5A
S31508008618A4F1FF04B6F5007F64F5407404D25FEA56
S315080086284E0E6D4146EB060642EAC62141EA555109
S315080086384FEAC52040EA5E504FEACE2EB4F1FD0C4B
S3150800864888BFBCF5E06F1ED8BEF1004F08BF5FEAC9
S31508008658500E50F1000041EB045170BD06F000467B
S3150800866846EA010140EA020081EA0301B4EB5C0428
S31508008678C2BFD4EB0C0541EA045170BD41F4801120
S315080086884FF0000E013C00F3AB8014F1360FDEBF45
S31508008698002001F0004170BDC4F10004203C35DA21
S315080086A80C341BDC04F11404C4F1200500FA05F3A4
S315080086B820FA04F001FA05F240EA020001F0004245
S315080086C821F0004110EBD37021FA04F642EB0601BB
S315080086D85EEA430E08BF20EAD37070BDC4F10C04E5
S315080086E8C4F1200500FA04F320FA05F001FA04F2A9
S315080086F840EA020001F0004110EBD37041F1000195
S315080087085EEA430E08BF20EAD37070BDC4F120059F
S3150800871800FA05F24EEA020E20FA04F301FA05F207
S3150800872843EA020321FA04F001F0004121FA04F2AF
S3150800873820EA020000EBD3705EEA430E08BF20EA7F
S31508008748D37070BD94F0000F0FD101F000464000B9
S3150800875841EB010111F4801F08BF013CF7D041EA3B
S31508008768060195F0000F18BF704703F0004652003F
S3150800877843EB030313F4801F08BF013DF7D043EA10
S315080087880603704794EA0C0F0CEA135518BF95EAC6
S315080087980C0F0CD050EA410618BF52EA4306D1D14D
S315080087A881EA030101F000414FF0000070BD50EA6C
S315080087B8410606BF1046194652EA430619D094EAF6
S315080087C80C0F02D150EA013613D195EA0C0F05D1E0
S315080087D852EA03361CBF104619460AD181EA030134
S315080087E801F0004141F0FE4141F470014FF00000EC
S315080087F870BD41F0FE4141F4780170BD70B54FF087
S31508008808FF0C4CF4E06C1CEA11541DBF1CEA135506
S3150800881894EA0C0F95EA0C0F00F0A7F8A4EB0504E8
S3150800882881EA030E52EA03354FEA013100F08880DF
S315080088384FEA03334FF0805545EA131343EA1263A8
S315080088484FEA022245EA111545EA10654FEA00265D
S315080088580EF000419D4208BF964244F1FD0404F516
S31508008868407402D25B084FEA3202B61A65EB030572
S315080088785B084FEA32024FF480104FF4002CB6EB2F
S31508008888020E75EB030E22BFB61A754640EA0C00AF
S315080088985B084FEA3202B6EB020E75EB030E22BFEF
S315080088A8B61A754640EA5C005B084FEA3202B6EB30
S315080088B8020E75EB030E22BFB61A754640EA9C00EF
S315080088C85B084FEA3202B6EB020E75EB030E22BFBF
S315080088D8B61A754640EADC0055EA060E18D04FEA7D
S315080088E8051545EA16754FEA06164FEAC30343EA1D
S315080088F852734FEAC2025FEA1C1CC0D111F4801FEA
S315080089080BD141EA00014FF000004FF0004CB6E7E2
S3150800891811F4801F04BF01430020B4F1FD0C88BF81
S31508008928BCF5E06F3FF6AFAEB5EB030C04BFB6EB8C
S31508008938020C5FEA500C50F1000041EB045170BD7F
S315080089480EF0004E4EEA113114EB5C04C2BFD4EBAC
S315080089580C0541EA045170BD41F480114FF0000E30
S31508008968013C90E645EA060E8DE60CEA135594EAAC
S315080089780C0F08BF95EA0C0F3FF43BAF94EA0C0FAF
S315080089880AD150EA01347FF434AF95EA0C0F7FF424
S3150800899825AF104619462CE795EA0C0F06D152EA78
S315080089A803353FF4FDAE1046194622E750EA41065C
S315080089B818BF52EA43067FF4C5AE50EA41047FF46D
S315080089C80DAF52EA43057FF4EBAE12E74FF0FF3CD2
S315080089D806E000BF4FF0010C02E000BF4FF0010CA3
S315080089E84DF804CD4FEA410C7FEA6C5C4FEA430C1C
S315080089F818BF7FEA6C5C1BD001B050EA410C0CBF6B
S31508008A0852EA430C91EA030F02BF90EA020F0020CC
S31508008A18704710F1000F91EA030F58BF994208BF33
S31508008A2890422CBFD8176FEAE37040F001007047F0
S31508008A384FEA410C7FEA6C5C02D150EA013C07D147
S31508008A484FEA430C7FEA6C5CD6D152EA033CD3D092
S31508008A585DF8040B704700BF8446104662468C468C
S31508008A681946634600E000BF01B5FFF7B7FF0028BF
S31508008A7848BF10F1000F01BD4DF808EDFFF7F4FFE8
S31508008A880CBF012000205DF808FB00BF4DF808ED73
S31508008A98FFF7EAFF34BF012000205DF808FB00BF96
S31508008AA84DF808EDFFF7E0FF94BF012000205DF8B8
S31508008AB808FB00BF4DF808EDFFF7CEFF94BF01206D
S31508008AC800205DF808FB00BF4DF808EDFFF7C4FF66
S31508008AD834BF012000205DF808FB00BF4FEA410CAF
S31508008AE87FEA6C5C02D150EA013C0AD14FEA430C92
S31508008AF87FEA6C5C02D152EA033C02D14FF00000CF
S31508008B0870474FF0010070474FEA410212F500120C
S31508008B1815D211D56FF47873B3EB625212D94FEAAE
S31508008B28C12343F0004343EA505311F0004F23FA98
S31508008B3802F018BF404270474FF00000704750EAED
S31508008B48013005D111F0004008BF6FF000407047AA
S31508008B584FF00000704700BF4FEA4102B2F1E04308
S31508008B6824BFB3F5001CDCF1FE5C0DD901F0004CFE
S31508008B784FEAC0024CEA5070B2F1004F40EB83004E
S31508008B8808BF20F00100704711F0804F21D113F17A
S31508008B983872BCBF01F00040704741F480114FEAB3
S31508008BA85252C2F11802C2F1200C10FA0CF320FA3C
S31508008BB802F018BF40F001004FEAC1234FEAD32359
S31508008BC803FA0CFC40EA0C0023FA02F34FEA4303C3
S31508008BD8CCE77FEA625307D150EA01331EBF4FF04C
S31508008BE8FE4040F44000704701F0004040F0FE4067
S31508008BF840F40000704700BF80F0004002E000BF64
S31508008C0881F0004142001FBF5FEA410392EA030F61
S31508008C187FEA226C7FEA236C6AD04FEA1262D2EBAB
S31508008C281363C1BFD218414048404140B8BF5B42B0
S31508008C38192B88BF704710F0004F40F4000020F049
S31508008C487F4018BF404211F0004F41F4000121F05F
S31508008C587F4118BF494292EA030F3FD0A2F10102A9
S31508008C6841FA03FC10EB0C00C3F1200301FA03F1E7
S31508008C7800F0004302D5494260EB4000B0F5000F0A
S31508008C8813D3B0F1807F06D340084FEA310102F1C9
S31508008C980102FE2A51D2B1F1004F40EBC25008BF7B
S31508008CA820F0010040EA03007047490040EB000045
S31508008CB8013A28BFB0F5000FEDD2B0FA80FCACF146
S31508008CC8080CB2EB0C0200FA0CF0AABF00EBC25073
S31508008CD852421843BCBFD0401843704792F0000F61
S31508008CE881F4000106BF80F400000132013BB5E7B4
S31508008CF84FEA41037FEA226C18BF7FEA236C21D02A
S31508008D0892EA030F04D092F0000F08BF084670478E
S31508008D1890EA010F1CBF0020704712F07F4F04D15C
S31508008D28400028BF40F00040704712F100723CBF6F
S31508008D3800F50000704700F0004343F0FE4040F499
S31508008D48000070477FEA226216BF08467FEA236357
S31508008D580146420206BF5FEA412390EA010F40F442
S31508008D68800070474FF0000304E000BF10F000438E
S31508008D7848BF40425FEA000C08BF704743F0964375
S31508008D8801464FF000001CE050EA010208BF704790
S31508008D984FF000030AE000BF50EA010208BF704717
S31508008DA811F0004302D5404261EB41015FEA010C2C
S31508008DB802BF84460146002043F0B64308BFA3F124
S31508008DC88053A3F50003BCFA8CF2083AA3EBC25306
S31508008DD810DB01FA02FC634400FA02FCC2F1200225
S31508008DE8BCF1004F20FA02F243EB020008BF20F05C
S31508008DF80100704702F1200201FA02FCC2F12002C2
S31508008E0850EA4C0021FA02F243EB020008BF20EAB6
S31508008E18DC7070474FF0FF0C1CEAD0521EBF1CEAE4
S31508008E28D15392EA0C0F93EA0C0F6FD01A4480EAD2
S31508008E38010C400218BF5FEA41211ED04FF00063BB
S31508008E4843EA501043EA5111A0FB01310CF00040E7
S31508008E58B1F5000F3EBF490041EAD3715B0040EA0D
S31508008E68010062F17F02FD2A1DD8B3F1004F40EBDD
S31508008E78C25008BF20F00100704790F0000F0CF0B0
S31508008E88004C08BF49024CEA502040EA51207F3A74
S31508008E98C2BFD2F1FF0340EAC250704740F400004F
S31508008EA84FF00003013A5DDC12F1190FDCBF00F040
S31508008EB800407047C2F10002410021FA02F1C2F1EE
S31508008EC8200200FA02FC5FEA310040F1000053EA8A
S31508008ED84C0308BF20EADC70704792F0000F00F0D8
S31508008EE8004C02BF400010F4000F013AF9D040EADE
S31508008EF80C0093F0000F01F0004C02BF490011F472
S31508008F08000F013BF9D041EA0C018FE70CEAD1536F
S31508008F1892EA0C0F18BF93EA0C0F0AD030F0004CEF
S31508008F2818BF31F0004CD8D180EA010000F00040A3
S31508008F38704790F0000F17BF90F0004F084691F061
S31508008F48000F91F0004F14D092EA0C0F01D142029B
S31508008F580FD193EA0C0F03D14B0218BF084608D164
S31508008F6880EA010000F0004040F0FE4040F40000AE
S31508008F78704740F0FE4040F4400070474FF0FF0C41
S31508008F881CEAD0521EBF1CEAD15392EA0C0F93EA88
S31508008F980C0F69D0A2EB030280EA010C49024FEADA
S31508008FA8402037D04FF0805343EA111143EA101393
S31508008FB80CF000408B4238BF5B0042F17D024FF44B
S31508008FC8000C8B4224BF5B1A40EA0C00B3EB510F26
S31508008FD824BFA3EB510340EA5C00B3EB910F24BF0F
S31508008FE8A3EB910340EA9C00B3EBD10F24BFA3EB94
S31508008FF8D10340EADC001B0118BF5FEA1C1CE0D15C
S31508009008FD2A3FF650AF8B4240EBC25008BF20F00E
S31508009018010070470CF0004C4CEA50207F32C2BF62
S31508009028D2F1FF0340EAC250704740F400004FF0FF
S315080090380003013A37E792F0000F00F0004C02BF30
S31508009048400010F4000F013AF9D040EA0C0093F0FA
S31508009058000F01F0004C02BF490011F4000F013B54
S31508009068F9D041EA0C0195E70CEAD15392EA0C0FBC
S3150800907808D142027FF47DAF93EA0C0F7FF470AFF4
S31508009088084676E793EA0C0F04D14B023FF44CAF37
S3150800909808466EE730F0004C18BF31F0004CCAD1CC
S315080090A830F000427FF45CAF31F000437FF43CAF08
S315080090B85FE700BF4FF0FF3C06E000BF4FF0010C2A
S315080090C802E000BF4FF0010C4DF804CD4FEA40020C
S315080090D84FEA41037FEA226C18BF7FEA236C11D056
S315080090E801B052EA530C18BF90EA010F58BFB2EB09
S315080090F8030088BFC81738BF6FEAE17018BF40F089
S31508009108010070477FEA226C02D15FEA402C05D13C
S315080091187FEA236CE4D15FEA412CE1D05DF8040BC1
S31508009128704700BF844608466146FFE70FB5FFF754
S31508009138C9FF002848BF10F1000F0FBD4DF808ED0C
S31508009148FFF7F4FF0CBF012000205DF808FB00BFFD
S315080091584DF808EDFFF7EAFF34BF012000205DF857
S3150800916808FB00BF4DF808EDFFF7E0FF94BF0120A4
S3150800917800205DF808FB00BF4DF808EDFFF7D2FFA1
S3150800918894BF012000205DF808FB00BF4DF808EDE4
S31508009198FFF7C8FF34BF012000205DF808FB00BFB1
S315080091A84FEA4002B2F1FE4F0FD34FF09E03B3EBDE
S315080091B812620DD94FEA002343F0004310F0004F1E
S315080091C823FA02F018BF404270474FF00000704774
S315080091D812F1610F01D1420205D110F0004008BF13
S315080091E86FF0004070474FF0000070477BB972B9BE
S315080091F80029BEBF00204FF0004106E008BF00283E
S315080092081CBF6FF000414FF0FF3000F0D7B9ADF141
S31508009218080C6DE904CE002909DB002B1ADB00F0DF
S315080092284DF8DDF804E0DDE9022304B07047404252
S3150800923861EB4101002B1BDB00F040F8DDF804E088
S31508009248DDE9022304B0404261EB4101524263EB77
S3150800925843037047524263EB430300F02FF8DDF8E7
S3150800926804E0DDE9022304B0404261EB410170479E
S31508009278524263EB430300F021F8DDF804E0DDE928
S31508009288022304B0524263EB4303704753B94AB901
S31508009298002908BF00281CBF4FF0FF314FF0FF30E8
S315080092A800F08CB9ADF1080C6DE904CE00F006F8AB
S315080092B8DDF804E0DDE9022304B070472DE9F0473C
S315080092C8089D8E4604468846002B4AD18A42174688
S315080092D862D9B2FA82F64EB1C6F1200301FA06F847
S315080092E820FA03F3B74043EA0808B4404FEA174E92
S315080092F8B8FBFEF11FFA87FC0EFB118801FB0CF27E
S31508009308230C43EA08439A4209D9FB1801F1FF30AE
S3150800931880F0EB809A4240F2E88002393B449A1A78
S31508009328B2FBFEF00EFB102200FB0CFCA3B243EACC
S3150800933802439C4509D9FB1800F1FF3280F0D78013
S315080093489C4540F2D4803B44023840EA014000215B
S31508009358A3EB0C031DB10022F340C5E90032BDE8B2
S31508009368F0878B4205D90DB1C5E9000100210846E9
S31508009378F5E7B3FA83F1002946D1734502D3824249
S3150800938800F20881841A6EEB030201209046002D2C
S31508009398E5D0C5E90048E2E7002A00F09180B2FA6C
S315080093A882F6002E40F0A5808A1A0121030C4FEA9E
S315080093B8174E80B2BCB2B2FBFEFC0EFB1C2243EA77
S315080093C8024304FB0CF29A4207D9FB180CF1FF3842
S315080093D802D29A4200F2E380C4469B1AB3FBFEF215
S315080093E80EFB123302FB04F440EA03439C4207D9F6
S315080093F8FB1802F1FF3002D29C4200F2CD800246E9
S315080094081B1B42EA0C40A5E7C1F120068B4022FA4D
S3150800941806F71F432EFA06FA4FEA1749BAFBF9F870
S315080094280EFA01FE20FA06F309FB18AA1FFA87FCAA
S3150800943843EA0E0300FA01FE08FB0CF01C0C44EA8A
S315080094480A44A04202FA01F20AD93C1908F1FF3A7D
S3150800945880F09E80A04240F29B80A8F102083C4416
S31508009468241A98B2B4FBF9F309FB134403FB0CFC62
S3150800947840EA0444A44509D93C1903F1FF3080F0B1
S315080094888580A44540F28280023B3C4443EA084072
S31508009498A4EB0C04A0FB028C64454346E14664D35E
S315080094A861D05DB1BEEB030264EB090404FA06F663
S315080094B822FA01F31E43CC40C5E9006400214EE7B1
S315080094C8B1FBF2FC010C41EA0E4180B240EA0142C6
S315080094D83B46B1FBF7F138463C46B846BE46202619
S315080094E8A2EB080241EA0C4165E7014617E7104670
S315080094F82BE7C6F120012EFA01FCB7400EFA06FE44
S3150800950820FA01F141EA0E014FEA174EBCFBFEF8B4
S31508009518BCB20EFB18CC08FB04F90A0C42EA0C424A
S31508009528B04091454FEA104380B23ED9BA1808F1BF
S31508009538FF3C01D291451FD8A2EB0902B2FBFEF9FE
S3150800954809FB04F80EFB192A8AB242EA0A4242457E
S3150800955829D2BA1809F1FF31C2D24245C0D2A9F1B7
S3150800956802013A44BCE7C6459BD2B8EB02036CEB4A
S31508009578070C0138E14694E7A7EB09094A44B2FB08
S31508009588FEF9A8F1020C09FB04F8DBE703467DE7B8
S31508009598D04665E70846FAE63B44023A30E7ACF1B6
S315080095A8020C3B4419E749469AE7A2EB0902B2FBC3
S315080095B8FEF9C44609FB04F8C4E700BF704700BFB4
S315080095C880B584B000AF3B1D00221A605A609A60C5
S315080095D8184B194A1A60174B00229A60154B002235
S315080095E81A73144B00221A75124B4FF46022DA616B
S315080095F8104B00225A600F4B01221A610D4805F0DC
S3150800960897F90346002B01D002F0EAFE08237B608F
S315080096180123BB600023FB603B1D1946054805F07E
S315080096284BFC0346002B01D002F0DAFE00BF1037C8
S31508009638BD4680BD6C0200200024014080B58AB072
S3150800964800AF786007F1180300221A605A609A601A
S31508009658DA607B681B681F4A934237D11E4B9B69A1
S315080096681D4A43F4007393611B4B9B6903F400730B
S315080096787B617B69184B9B69174A43F0040393611E
S31508009688154B9B6903F004033B613B69124B9B69C5
S31508009698114A43F0080393610F4B9B6903F00803CB
S315080096A8FB60FB680823BB610323FB6107F118030A
S315080096B819460A4806F07AFF0323BB610323FB61B0
S315080096C807F118031946064806F070FF00BF283741
S315080096D8BD4680BD00240140001002400008014034
S315080096E8000C014080B582B000AF03460A46FB71FC
S315080096F81346BB71FB79062B47D801A252F823F00B
S3150800970825970008359700084597000855970008D3
S31508009718659700087597000885970008BB791A4663
S315080097284FF480711D4807F0DCF82FE0BB791A461C
S315080097384FF40071194807F0D4F827E0BB791A46A0
S315080097484FF48061154807F0CCF81FE0BB791A4634
S315080097584FF40061114807F0C4F817E0BB791A46B8
S315080097684FF480510D4807F0BCF80FE0BB791A464C
S315080097784FF400410A4807F0B4F807E0BB791A46DF
S315080097880821084807F0ADF800E000BFFB7906494C
S31508009798BA79CA5400BF0837BD4680BD00180140CB
S315080097A800080140001401409C02002080B483B0E0
S315080097B800AF0346FB71FB79034AD35C18460C379E
S315080097C8BD4680BC704700BF9C02002080B582B0A9
S315080097D800AF0346FB71FB79062B3BD801A252F86A
S315080097E823F000BF09980008159800082198000872
S315080097F82D980008399800084598000851980008D7
S315080098080221174807F056F8034624E004211448AD
S3150800981807F050F803461EE08021124807F04AF878
S31508009828034618E08021104807F044F8034612E07A
S3150800983810210E4807F03EF803460CE008210B48AD
S3150800984807F038F8034606E00221064807F032F81A
S31508009858034600E0002318460837BD4680BD00BF0A
S31508009868000801400018014000140140000C01409E
S3150800987880B500AF104805F0B3FC00210020FFF7BB
S3150800988831FF00210120FFF72DFF00210220FFF7F5
S3150800989829FF00210320FFF725FF00210420FFF7F1
S315080098A821FF01210520FFF71DFF00210620FFF7EC
S315080098B819FF00BF80BD00BF6C02002090B587B0B5
S315080098C800AF78600C4B7B610C4B3B617969786813
S315080098D8FFF796F903461C4639697869FFF79AFA35
S315080098E8034619462046FFF749FB0346FB60FB6813
S315080098F818461C37BD4690BD00007A443211803B95
S31508009908B0B586B000AFF860B9607A603B60F868B1
S31508009918FEF7E0FD1CA3D3E90023FEF76FFF024616
S315080099280B4614461D46B868FEF7E6FD02460B4682
S3150800993820462946FEF738FE02460B4610461946C3
S31508009948FFF70AF903467B6179687869FFF714FC1B
S315080099580346002B01D00E4B10E079697868FFF7AB
S315080099684FF9034619467869FFF708FB034619466F
S315080099783868FFF74FFA03463B613B6918461837BC
S31508009988BD46B0BDAFF300800000000000FEAF4042
S31508009998000080BF80B588B000AF0346FB71FB792D
S315080099A8002B03D0082000F03BF802E0092000F05D
S315080099B837F8174805F094F84FF0FF31144805F0C2
S315080099C869F9134805F06CFAF861114805F036F993
S315080099D8FB69B3F57A6F01D9142315E00D4BBB6102
S315080099E80D4B7B610D4B3B61F8693B697A69B9692F
S315080099F8FFF786FF03461846FFF760FFF860F86822
S31508009A08FFF7CEFB03461BB218462037BD4680BD76
S31508009A186C020020333353400000A04000007A440B
S31508009A2880B586B000AF78607B68FB6001233B6130
S31508009A3803237B6107F10C031946064805F03CFA2F
S31508009A480346002B01D002F0CBFC00BF1837BD46F1
S31508009A5880BD00BF6C02002080B500AF174B184ABE
S31508009A681A60164B08225A60144B00229A60134B48
S31508009A780022DA60114B4FF460221A610F4B4FF43B
S31508009A8880125A610D4B00221A760C4B01225A761F
S31508009A980A4B01229A76094B0122DA76074B0022ED
S31508009AA81A77064B01225A77044805F047FC0346FD
S31508009AB8002B01D002F094FC00BF80BDA402002050
S31508009AC80064004080B500AF174B184A1A60164B59
S31508009AD810225A60144B00229A60134B0022DA604F
S31508009AE8114B4FF460221A610F4B4FF480125A61DA
S31508009AF80D4B00221A760C4B01225A760A4B012284
S31508009B089A76094B0122DA76074B00221A77064B12
S31508009B1801225A77044805F011FC0346002B01D0A8
S31508009B2802F05EFC00BF80BDCC0200200068004041
S31508009B3880B58EB000AF786007F1200300221A605E
S31508009B485A609A60DA607B681B68614A934253D107
S31508009B58604B1B6801335F4A13605E4B1B68012B19
S31508009B680BD15D4BDB695C4A43F00073D3615A4BF2
S31508009B78DB6903F00073FB61FB69574B9B69564A1F
S31508009B8843F020039361544B9B6903F02003BB61A0
S31508009B98BB6901233B6200237B620023BB6207F192
S31508009BA8200319464D4806F001FD02233B620223AD
S31508009BB87B620323FB6207F120031946474806F030
S31508009BC8F5FC474B5B683B633B6B23F4C0433B633D
S31508009BD83B6B43F0E0633B633B6B43F4C0433B6337
S31508009BE83F4A3B6B536000220021142006F049FBCC
S31508009BF8142006F062FB67E07B681B68394A9342C3
S31508009C0862D1354BDB69344A43F08063D361324B02
S31508009C18DB6903F080637B617B692E4B1B68013324
S31508009C282C4A13602B4B1B68012B0BD12A4BDB697B
S31508009C38294A43F00073D361274BDB6903F00073A5
S31508009C483B613B69244B9B69234A43F008039361AC
S31508009C58214B9B6903F00803FB60FB6820233B62E2
S31508009C6800237B620023BB6207F1200319461E48BE
S31508009C7806F09CFC40233B6202237B620323FB62BB
S31508009C8807F120031946184806F090FC144B5B6840
S31508009C987B637B6B43F0E0637B637B6B43F48003F6
S31508009CA87B630F4A7B6B5360002200213F2006F036
S31508009CB8E8FA3F2006F001FB00220021412006F0C1
S31508009CC8E0FA412006F0F9FA00BF3837BD4680BDEC
S31508009CD800640040F402002000100240001401400D
S31508009CE80000014000680040000C014080B400AF45
S31508009CF8084B00221A70074B00225A70054B00229F
S31508009D0862F06902DA7300221A7400BFBD4680BC85
S31508009D18704700BFF802002080B500AF1E4B5A787E
S31508009D281E4B1B789A4206D01B4B5A781B4B1A7047
S31508009D38194B00221A701A4B5B78002B03D0164B66
S31508009D4804225A7716E0174B1B7B002B03D0124BBD
S31508009D5807225A770EE0134B5B7B002B03D00E4B7A
S31508009D680A225A7706E00C4B9B7F002B02D10A4B36
S31508009D7800225A77084B5B7F0021184602F0DEF965
S31508009D880346002B06D0044B5B7F1A46002106487B
S31508009D980AF0EEF900BF80BDF8020020170300207C
S31508009DA808000020140A00207865010880B500AF6D
S31508009DB80B4B10221A7000F077FF0A4B42F210720A
S31508009DC81A80084B40F2DC525A80064B40F6B832E5
S31508009DD89A80044B40F69672DA8000BF80BD00BFB1
S31508009DE8180300203003002080B500AF0C4BD3F8C9
S31508009DF80730184603F074FF094B1A78094B5A714D
S31508009E08074B5A78074B9A71054B9A78054BDA71BE
S31508009E18034BD3F80330034AC2F8013000BF80BDAC
S31508009E286C00002038030020B0B584B002AFAB4BF5
S31508009E3893F80A31022B40F0D180A84BD3F80031A9
S31508009E48B3F51C5F47D0B3F51C5F00F2C380B3F5C2
S31508009E58E05F00F0B680B3F5E05F00F2BB80B3F5CB
S31508009E68B85F00F0B280B3F5B85F00F2B380B3F517
S31508009E78B05F00F0AC80B3F5B05F00F2AB80B3F525
S31508009E88A85F00F0A680B3F5A85F00F2A380B3F533
S31508009E98985F00F08680B3F5985F00F29B80B3F56B
S31508009EA8885F6FD0B3F5885F00F29480B3F5805F5A
S31508009EB846D0B3F5805F00F28D80B3F5106F2CD0CD
S31508009EC8B3F5106F00F28680B3F5007F0BD0B3F5B3
S31508009ED8C06F18D07EE0824B01221A707F4B1A8811
S31508009EE8804B1A8076E0804B01221A707F4A7B4B9A
S31508009EF814461D460FCD0FC40FCD0FC40FCD0FC482
S31508009F082B68237066E07A4B01221A70794A734BDC
S31508009F1814460FCB07C423705CE0774B01221A70EE
S31508009F286E4B1B78AA2B03D1744B01221A7002E0D8
S31508009F38724B00221A70694B1A78714B1A7049E0ED
S31508009F4804F0C8FC03466F4A13606F4B634A92E8ED
S31508009F5803001860043319706B4B1B88FB806A4B27
S31508009F685B88C3F57A63BB80FB88684AA2FB032330
S31508009F78DB089AB2664BA3F80F20654BBA88A3F894
S31508009F881B2027E004F0A6FC03465E4A1360614BD3
S31508009F98524A07CA03C31A705E4B9A795C4B9A7081
S31508009FA818E004F097FC0346564A13605A4B4B4A86
S31508009FB892E8030018600433198002330A0C1A70F1
S31508009FC808E0564B01221A7004E000BF02E000BF01
S31508009FD800E000BF414B002283F80A2104F07AFC0E
S31508009FE802464F4B1B68D21A4E4B1B689A42C0F062
S31508009FF8C7844D4B1B78103B122B00F2A28401A292
S3150800A00852F823F059A000084BA900084BA90008E4
S3150800A0187FA0000891A0000841A100088BA10008AC
S3150800A028FDA100089FA20008F1A200087DA4000867
S3150800A03881A5000813A6000869A60008DBA600087B
S3150800A048C3A8000805A9000825A9000837A9000813
S3150800A05800210020FFF746FB00210120FFF742FBFD
S3150800A068324B1B78032B40F0708400F01DFE00F07D
S3150800A078A9FE00F06ABC142000F0B4FC4FF4FA708C
S3150800A08800F068FD00F07CBC144B93F80A31002BED
S3150800A09801D101F0BDFAFA2000F05CFD104B1B78DF
S3150800A0A8002B02D0152000F09DFC0D4B1B78002BC9
S3150800A0B840F04D8400F042FD034642F21072934286
S3150800A0C840F245841A4800F0D3FD114B09225A7705
S3150800A0D81849042001F042FA00F039BC7408002037
S3150800A0E82B030020400300202803002044030020F7
S3150800A0F829030020780300202A0300202D030020C6
S3150800A108BC030020C403002088030020CDCCCCCC97
S3150800A118F802002098030020A40300202C0300203E
S3150800A128200300202403002018030020D103002060
S3150800A138FCC0F0FCC0650108AF4B93F80A31002B48
S3150800A14801D101F065FAFA2000F004FDAB4B5B7A01
S3150800A158002B02D0162000F045FC00F0EFFC034661
S3150800A16842F21072934240F2F4834FF2F04000F044
S3150800A1782BFDA34B0A225A77A249042001F0EEF9CF
S3150800A188FEE39D4B93F80A31002B01D101F040FA02
S3150800A198FA2000F0DFFC9C4B1B889C4AA2FB032391
S3150800A1A8DB089AB2964BA3F80F20954B002242F08B
S3150800A1B80A02DA7600221A77914B0122DA758F4B52
S3150800A1C8DB79052B02D1172000F00CFC00F0B6FC51
S3150800A1D8034642F21072934240F2BD834FF2F040B2
S3150800A1E800F0F2FC864B0A225A778949042001F0C6
S3150800A1F8B5F9C5E3804B93F80A31002B01D101F074
S3150800A20807FAFA2000F0A6FC7D4B5B7F002B03D0EB
S3150800A2184FF2F04000F0D8FC00F090FC034641F2FB
S3150800A2288832934202D9182000F0DCFB794BB3F840
S3150800A23801309BB21946774BB3F907301BB2DA0FD0
S3150800A24813445B101BB2994206DA6D4B01225A7702
S3150800A2587149052001F082F96E4BB3F801309BB2BB
S3150800A26819466C4BB3F907301BB26C4A82FB0302DA
S3150800A2789210DB17D31A1BB2994280F26E83604B91
S3150800A28801225A776649052001F068F94FF2F0402D
S3150800A29800F09AFC61E35A4B0022DA7300221A741A
S3150800A2A8574B0022DA7600221A77554B0022DA75C0
S3150800A2B800F044FC034641F2883293420BD94FF228
S3150800A2C8F04000F081FC4E4B0A225A775549042083
S3150800A2D801F044F954E3494B9B7A002B40F03F833D
S3150800A2E8192000F07FFB3AE3434B93F80A31002B19
S3150800A2F802D1002001F0A0F9FA2000F02BFC4A4B05
S3150800A3081B78002B60D01A2000F06CFB4749072001
S3150800A31801F024F9464B1B781A46454B5B781946D3
S3150800A328434B9B7800930B464249072001F016F9E0
S3150800A3383F4BDB781A464049072001F00FF93C4B9A
S3150800A3489B881A463D49072001F008F9384BDB88EF
S3150800A3581A463B49072001F001F93A4A3A490720C3
S3150800A36801F0FCF8324BDB681A463849072001F039
S3150800A378F5F82F4B9B7C1A462D4B5B7C19462C4BC4
S3150800A3881B7C03F2C17300930B463149072001F081
S3150800A398E5F8274BDA7C9B8A1B0213431A462D4994
S3150800A3A8072001F0DBF8224B9B7D1A462A4907202D
S3150800A3B801F0D4F8294A2A49072001F0CFF8294A92
S3150800A3C82949072001F0CAF800F0B8FB034641F20C
S3150800A3D88832934240F2C582134B1B78002B40F013
S3150800A3E8C082074B09225A77204800F041FC2049C9
S3150800A3F8042001F0B3F8B4E274080020140A002017
S3150800A408F8020020D065010840030020CDCCCCCC4A
S3150800A418F065010860000020106601086766666630
S3150800A4282466010854660108280300207466010892
S3150800A438440300208066010894660108A866010896
S3150800A448C06601084C030020D8660108F0660108B2
S3150800A4580467010830670108446701085C0300209F
S3150800A468546701086D03002064670108FCC0F0FD05
S3150800A47878670108B04B93F80A31002B02D1AA2055
S3150800A48801F0DAF8FA2000F065FBAC4B1B78002BD4
S3150800A4985AD01B2000F0A6FAA949072001F05EF851
S3150800A4A8A84B1B88A84AA2FB03235B099BB21A463A
S3150800A4B8A649072001F052F8A24B5B88A44AA2FBDA
S3150800A4C80323DB089BB21A46A249072001F046F87F
S3150800A4D89C4B9B889E4AA2FB0323DB089BB21A4621
S3150800A4E89D49072001F03AF8964BDB88984AA2FB63
S3150800A4F80323DB089BB21A469449072001F02EF875
S3150800A508904B1B7A323B1A469449072001F026F8E5
S3150800A5188C4BB3F809309BB28D4AA2FB0323DB08A0
S3150800A5289BB21A468E49072001F018F8854BB3F8EE
S3150800A5380B309BB2864AA2FB0323DB089BB21A465A
S3150800A5488849072001F00AF800F0F8FA034641F2AC
S3150800A5588832934240F20782784B1B78002B40F0EA
S3150800A5680282814B09225A77804800F081FB80498C
S3150800A578042000F0F3FFF6E16F4B93F80A31002B3D
S3150800A58801D101F021F8022004F0AEF96A4B93F8DC
S3150800A5980A31002B01D101F02DF8FA2000F0DAFA79
S3150800A5A800F0CCFA034641F2883293420DD9714B32
S3150800A5B81B78002B09D16C4B09225A776E4800F094
S3150800A5C857FB6E49042000F0C9FF6D4B1B78002B1A
S3150800A5D803D01C2000F006FAC7E100F0AFFA0346DC
S3150800A5E84EF66022934240F2C081624B1B78012BDB
S3150800A5F840F0BB815C4B09225A775F4800F038FB6C
S3150800A6086049042000F0AAFFAFE14B4B93F80A31E2
S3150800A618002B02D1002001F025F8FA2000F09AFA5A
S3150800A628594B5B7A002B02D01D2000F0DBF900F0AD
S3150800A63885FA034641F27072934240F29881524B6A
S3150800A6485B7A002B40F093814FF2F04000F0BCFA99
S3150800A658454B0A225A774D49042000F07FFF86E1C8
S3150800A668354B93F80A31002B02D1AA2000F0FAFFDD
S3150800A678FA2000F06FFA464B1B79002B00F0798117
S3150800A6881E2000F0AFF904F025F90346414A136085
S3150800A698082000F0E7FC3E4B5B88C3F57A637B80AD
S3150800A6A83B4B1B883B803B88294AA2FB0323DB08D4
S3150800A6B89AB22D4BA3F80F202B4B7A88A3F81B20A8
S3150800A6C8294B0122DA7503F001FB0346324A136067
S3150800A6D84FE104F0FFF802462E4B1B68D31AB3F570
S3150800A6E8FA6F0BD94FF2F04000F06EFA1E4B0922AA
S3150800A6F85A772A49052000F031FF41E11A4B1B78A1
S3150800A708012B02D1264800F07BFA174B1B78032B3E
S3150800A71802D1234800F074FA224B5B78002B45D007
S3150800A7284FF2F04000F050FA0F4B04225A771E49B0
S3150800A738052000F013FF23E17408002029030020F0
S3150800A74888670108780300201F85EB519867010878
S3150800A758CDCCCCCCA4670108B0670108BC67010852
S3150800A768C8670108D4670108F8020020FCC0F1FC94
S3150800A778E06701082A030020FCC0F4FCF06701081A
S3150800A7882D03002000680108140A0020186801082B
S3150800A79888030020C4030020C00300203468010889
S3150800A7A8F0F00004080000205868010800F036FD9B
S3150800A7B80346032B0BD04FF2F04000F005FA784B0E
S3150800A7C808225A777749052000F0C8FED8E0002005
S3150800A7D8FFF7E0F803465A2B05DC0120FFF7DAF8FD
S3150800A7E803465A2B14DD704800F0EEF96C4B052227
S3150800A7F85A770020FFF7CEF803461C460120FFF7D4
S3150800A808C9F8034622466949052000F0A7FEB7E0BD
S3150800A818674BB3F801309BB21946654BB3F9073055
S3150800A8281BB2644A82FB03029210DB17D31A1BB2C7
S3150800A838994206DA5A4B01225A775F49052000F0F1
S3150800A8488DFE574B5B7F002B03D04FF2F04000F08C
S3150800A858BBF95A4B4FF6FD72DA8003F037FA02460F
S3150800A868574B1B68D31A574AA2FB03235B099AB2AC
S3150800A878524B9A804A4BB3F815309BB2C3F57A63A4
S3150800A8889AB24E4B5A80464BB3F813309BB21A46C7
S3150800A898920013445B009AB2484B1A804A4B93F8C5
S3150800A8A80A31002B05D100F0F1FE312000F052F9EB
S3150800A8B866E00A2000F04EF962E00A2000F04AF93C
S3150800A8C8374B0022DA75414B1B68184600F0ECFE38
S3150800A8D800F034F9034642F21072934206D93C490D
S3150800A8E8042000F03BFE3B4800F0C2F93A4B1B78BF
S3150800A8F8002B40D0202000F075F83CE0FA2000F044
S3150800A90829F900F0F1FE00F019F9034640F6C412D9
S3150800A918934232D9222000F065F82EE02F4B1B68A7
S3150800A928184600F001FF222000F05CF828E02C4BBE
S3150800A9381B780A2B23D0102000F054F800F0B4F93D
S3150800A9481DE0102000F04EF81AE000BF18E000BF1E
S3150800A95816E000BF14E000BF12E000BF10E000BF19
S3150800A9680EE000BF0CE000BF0AE000BF08E000BF29
S3150800A97806E000BF04E000BF02E000BF00E000BF39
S3150800A98800F04CFC0346032B03D1054B01229A77AA
S3150800A99802E0034B00229A7700BF0837BD46B0BDD0
S3150800A9A8F802002074680108F0F0010094680108AC
S3150800A9B8600000206766666624660108AC03002006
S3150800A9C8C00300208988888874080020C8030020E6
S3150800A9D8BC680108FDC0F0FC2C030020CC0300204D
S3150800A9E8D103002080B582B000AF0346FB71424A06
S3150800A9F8FB79137003F06EFF0346404A13603E4B1B
S3150800AA081B78102B03D13E49072000F0A7FD3A4BC7
S3150800AA181B78132B03D13B49072000F09FFD364BC3
S3150800AA281B78142B03D13849072000F097FD324BC1
S3150800AA381B78152B03D13549072000F08FFD2E4BBF
S3150800AA481B78172B03D13249072000F087FD2A4BBC
S3150800AA581B78192B03D12F49072000F07FFD264BB9
S3150800AA681B781A2B03D12C49072000F077FD224BB7
S3150800AA781B781B2B03D12949072000F06FFD1E4BB5
S3150800AA881B781C2B03D12649072000F067FD1A4BB3
S3150800AA981B781D2B03D12349072000F05FFD164BB1
S3150800AAA81B781E2B03D12049072000F057FD124BAF
S3150800AAB81B781F2B03D11D49072000F04FFD0E4BAD
S3150800AAC81B78202B03D11A49072000F047FD0A4BAB
S3150800AAD81B78212B03D11749072000F03FFD064BA9
S3150800AAE81B78222B03D11449072000F037FD00BF35
S3150800AAF80837BD4680BD00BF180300201C03002088
S3150800AB08CC680108D8680108EC68010800690108DA
S3150800AB181869010828690108446901086069010873
S3150800AB28746901088C690108A0690108B8690108EF
S3150800AB38CC690108E8690108F869010880B500AF19
S3150800AB4803F0C8FE0246024B1B68D31A184680BD96
S3150800AB581C03002080B582B000AF786003F0BAFE07
S3150800AB680346044A1360044A7B68136000BF083723
S3150800AB78BD4680BD200300202403002080B582B08E
S3150800AB8800AF78600C4B5B7F002B03D00B4B002281
S3150800AB981A7002E0094B01221A70094A7B68136089
S3150800ABA8084B1B781F2B02D01F20FFF71BFF00BF7F
S3150800ABB80837BD4680BD00BFF8020020D003002034
S3150800ABC8C80300201803002080B582B000AF78605B
S3150800ABD8084B00221A70084A7B681360074B1B78D3
S3150800ABE81F2B02D01F20FFF7FDFE00BF0837BD4602
S3150800ABF880BD00BFD0030020C8030020180300202A
S3150800AC0880B582B000AF7860084B02221A70084AED
S3150800AC187B681360074B1B781F2B02D01F20FFF792
S3150800AC28E1FE00BF0837BD4680BD00BFD00300203F
S3150800AC38C80300201803002080B500AF0A4B01227C
S3150800AC481A700A4B0022DA752220FFF7CBFE00207D
S3150800AC5801F02EF900210020FEF744FD002101200D
S3150800AC68FEF740FD00BF80BDD0030020F802002093
S3150800AC7880B582B000AF7860084B01221A707A68EE
S3150800AC880749042000F06AFC064A7B6813602120FD
S3150800AC98FFF7A8FE00BF0837BD4680BDD0030020D1
S3150800ACA80C6A0108CC03002080B500AF03F012FE39
S3150800ACB80346314A1360314B00221A70304B002282
S3150800ACC81A70304B00221A702F4B00221A702F4B1D
S3150800ACD800221A702E4B00221A702E4B00229A70E8
S3150800ACE82C4B0022DA752B4B0022DA7600221A77CB
S3150800ACF8284B0022DA7300221A74312200212648CA
S3150800AD0809F048FA0D220021244809F043FA0522D9
S3150800AD180021234809F03EFA05220021214809F0B6
S3150800AD2839FA02220021204809F034FA09220021BA
S3150800AD381E4809F02FFA072200211D4809F02AFAA9
S3150800AD48082200211B4809F025FA082200211A487A
S3150800AD5809F020FA134B4FF47A625A80114B4FF4D4
S3150800AD68FA721A80154B00221A60154B00221A70BF
S3150800AD7801F0A8F900BF80BDC403002028030020FD
S3150800AD88290300202A0300202B0300202C03002077
S3150800AD982D030020F8020020440300207803002031
S3150800ADA88803002090030020400300209803002011
S3150800ADB8A4030020AC030020B4030020C00300202D
S3150800ADC8BC03002080B500AF01210020FEF78AFCED
S3150800ADD801210120FEF786FC1320FFF703FE00BFBA
S3150800ADE880BD000080B582B000AF984B1B780C2B4D
S3150800ADF800F2168101A252F823F000BF39AE000806
S3150800AE0877AE000851AE000803AF0008BDAE0008CB
S3150800AE1829B0000829B0000829B0000857AF00086B
S3150800AE2829B00008B9AF0008ABAF00089DAF000805
S3150800AE38002001F03DF8864B1B78002B00F0F480C3
S3150800AE48012000F00FF9EFE0002001F031F8814BFE
S3150800AE585B7F002B02D1012000F004F97D4B1B789B
S3150800AE68032B40F0E380002000F0EEFFDEE0002030
S3150800AE7801F01EF8774B5B7F002B02D0022000F00A
S3150800AE88F1F8744B1B78032B02D1002000F0DCFF85
S3150800AE9800F0C4F90346032B40F0CA806D4B1B78B3
S3150800AEA8032B00F0C580042000F0DCF8002000F031
S3150800AEB8FFFFBDE0002000F0FBFF664B1B78032B65
S3150800AEC802D1002000F0C0FF00F0A8F90346032BC2
S3150800AED80FD1604B1B78022B02D1032000F0C2F871
S3150800AEE85C4B1B78032B40F0A580012000F0BAF8CC
S3150800AEF8A0E0012000F0B6F89CE0012000F0D8FF99
S3150800AF08554B1B78222B1AD1544B1B78002B03D18F
S3150800AF180B2000F0A7F812E0504B1B78012B03D141
S3150800AF280C2000F09FF80AE04C4B1B78022B03D143
S3150800AF380A2000F097F802E00B2000F093F8464B39
S3150800AF481B781E2B78D1082000F08CF874E00120B5
S3150800AF5800F0AEFF404B1B78222B6FD13F4B1B7876
S3150800AF68002B03D10B2000F07DF867E03B4B1B78DC
S3150800AF78012B03D10C2000F075F85FE0374B1B78DE
S3150800AF88022B03D10A2000F06DF857E00B2000F0D9
S3150800AF9869F853E0002000F08BFF0A2000F062F8F9
S3150800AFA84FE0002000F084FF0A2000F05BF848E034
S3150800AFB8002000F07DFF274B1B78032B02D10020C9
S3150800AFC800F042FF0023FB7100F028F90346022B24
S3150800AFD819D1234B1B68002B05D103F07BFC0346CC
S3150800AFE81F4A136012E003F075FC02461C4B1B68E7
S3150800AFF8D31A41F28732934208D90123FB71184BB9
S3150800B00800221A6002E0164B00221A60FB79002B10
S3150800B01816D0002000F04CFF012000F023F80FE0BE
S3150800B028002000F01FF80CE000BF0AE000BF08E0A7
S3150800B03800BF06E000BF04E000BF02E000BF00E072
S3150800B04800BF00BF0837BD4680BD00BFD10300203A
S3150800B0581E0F0020F802002018030020D003002045
S3150800B068D403002080B582B000AF0346FB713D4A81
S3150800B078FB7913703B4B1B78002B03D13A49072001
S3150800B08800F06CFA374B1B78012B03D13749072098
S3150800B09800F064FA334B1B78022B03D13449072096
S3150800B0A800F05CFA2F4B1B78032B03D13149072094
S3150800B0B800F054FA2B4B1B78042B03D12E49072092
S3150800B0C800F04CFA274B1B78052B03D12B49072090
S3150800B0D800F044FA234B1B78062B03D1284907208E
S3150800B0E800F03CFA1F4B1B78072B03D1254907208C
S3150800B0F800F034FA1B4B1B78082B03D1224907208A
S3150800B10800F02CFA174B1B78092B03D11F49072087
S3150800B11800F024FA134B1B780A2B03D11C49072085
S3150800B12800F01CFA0F4B1B780B2B03D11949072083
S3150800B13800F014FA0B4B1B780C2B03D11649072081
S3150800B14800F00CFA074B1B780D2B03D1134907207F
S3150800B15800F004FA124AFB79537000BF0837BD4657
S3150800B16880BD00BFD1030020246A0108386A010897
S3150800B178506A0108686A0108806A01089C6A010819
S3150800B188BC6A0108DC6A0108FC6A0108146B010834
S3150800B1982C6B0108446B0108606B0108786B010881
S3150800B1A8F802002080B582B000AF03F093FB024690
S3150800B1B8164B1B68D31A632B24D903F08BFB03465B
S3150800B1C8124A136000F034F80346FB71104B1B78DB
S3150800B1D8FA799A4208D003F07DFB03460D4A1360B4
S3150800B1E80B4AFB7913700EE003F074FB0246094B11
S3150800B1F81B68D31AB3F5967F05D3054B1A78064B01
S3150800B2081A7000E000BF0837BD4680BDD803002085
S3150800B218DC030020E0030020D203002080B400AF3E
S3150800B228024B1B781846BD4680BC7047D2030020DF
S3150800B23880B582B000AF00F051F878602249786886
S3150800B248FDF786FF0346002B08D020497868FDF7E6
S3150800B2589DFF0346002B01D0012331E01C4978687D
S3150800B268FDF776FF0346002B08D01A497868FDF7DC
S3150800B2788DFF0346002B01D0022321E01549786883
S3150800B288FDF766FF0346002B08D013497868FDF7D3
S3150800B2987DFF0346002B01D0032311E00E49786889
S3150800B2A8FDF756FF0346002B09D04FF07E51786804
S3150800B2B8FDF76CFF0346002B01D0042300E00023AA
S3150800B2C818460837BD4680BD000050410000304189
S3150800B2D86666E6409A9999400000404080B582B073
S3150800B2E800AF0320FEF79CFB0E4803F0F9FB642128
S3150800B2F80C4803F0CFFC0B4803F0D2FD78600948E8
S3150800B30803F09CFC7868FDF72DFD034606491846A8
S3150800B318FDF734FE03463B603B6818460837BD46CA
S3150800B32880BD00BF6C020020CDCCE24280B500AFDC
S3150800B338064B074A1A60054804F0D9FF0346002B4E
S3150800B34801D001F04DF800BF80BD00BFE40300201E
S3150800B3580030024080B485B000AF78607B681B680F
S3150800B368094A93420BD1094B5B69084A43F04003E3
S3150800B3785361064B5B6903F04003FB60FB6800BF3B
S3150800B3881437BD4680BC70470030024000100240A2
S3150800B39880B584B000AFF860B9607A607B689BB204
S3150800B3A81946B86800F006F87B6818461037BD468F
S3150800B3B880BD000080B485B000AF78600B467B80FE
S3150800B3C872B600BF0023FB8145E0284BB3F8043466
S3150800B3D89BB2B3F5806F18D3244BB3F802349BB2EB
S3150800B3E801335A42C3F30903C2F3090258BF534249
S3150800B3F89AB21E4BA3F802241C4BB3F804349BB22A
S3150800B408013B9AB2194BA3F80424FB897A681344BA
S3150800B418164AB2F8002492B21978144B9954134B69
S3150800B428B3F800349BB201335A42C3F30903C2F393
S3150800B438090258BF53429AB20C4BA3F800240B4B87
S3150800B448B3F804349BB201339AB2084BA3F8042420
S3150800B458FB890133FB81FA897B889A42B5D362B6A0
S3150800B46800BF00BF1437BD4680BC7047EC030020F8
S3150800B47880B483B000AF72B600BF064BB3F8043485
S3150800B488FB8062B600BFFB8818460C37BD4680BCF1
S3150800B498704700BFEC03002080B582B000AF72B6D3
S3150800B4A800BF2D4BB3F804349BB2002B02D162B609
S3150800B4B800BF4EE0284BB3F80434FB80FB88802B8A
S3150800B4C801D98023FB80244BB3F802349BB2C3F519
S3150800B4D88063BB80FA88BB889A4201D9BB88FB80FF
S3150800B4E81D4BB3F804349BB2FA889A420CD11A4B0E
S3150800B4F8B3F802349BB21A46174B1344F9885022FC
S3150800B508184602F0D3F80BE0134BB3F802349BB293
S3150800B5181A46114B1344F9885122184602F0C6F800
S3150800B5280D4BB3F802349AB2FB8813449BB2C3F3A3
S3150800B53809039AB2084BA3F80224074BB3F8043454
S3150800B5489AB2FB88D31A9AB2034BA3F8042462B6B4
S3150800B55800BF0837BD4680BDEC0300200EB480B591
S3150800B56885B000AF0346FB71154AFB79137007F1DE
S3150800B5782003BB60BB68FA697E21124808F0CCFD37
S3150800B588F860FB68002B01DAFB6812E0FB687D2B84
S3150800B59801DD7E23FB60FB680133094A0021D1548B
S3150800B5A8FB689BB202339BB219460548FFF702FFB0
S3150800B5B8FB6818461437BD46BDE8804003B0704797
S3150800B5C8F4070020F507002080B582B000AF02F026
S3150800B5D87DFB02463B461946104602F0B5FB3B463C
S3150800B5E8072206214FF4E06000F060FB00BF083729
S3150800B5F8BD4680BD80B500AF044B082206214FF42E
S3150800B608006000F053FB00BF80BD00BF3003002078
S3150800B61880B582B000AF01233B7101237B710023FB
S3150800B628BB713B1D032206214FF4185000F03EFB60
S3150800B63800BF0837BD4680BD80B582B000AF034657
S3150800B648FB71074AFB791370054B082206214FF44C
S3150800B658807000F02BFB00BF0837BD4680BD00BFD1
S3150800B6683803002080B584B000AF0346FB71FB7928
S3150800B6783B7307F10C03012204214FF4206000F004
S3150800B68815FB00BF1037BD4680BD000080B500AF6A
S3150800B698044B082206214FF4905000F007FB00BF20
S3150800B6A880BD00BFAC03002080B584B000AF7860C9
S3150800B6B87B681B0EDBB23B727B681B0CDBB27B72AA
S3150800B6C87B681B0ADBB2BB727B68DBB2FB7207F1CD
S3150800B6D80803042204214FF4D05000F0E7FA00BF0B
S3150800B6E81037BD4680BD000080B500AF0B4BD3F8B8
S3150800B6F801300B4A53600A4B00229A700022DA700E
S3150800B708084B9B889AB2064B1A80054B07220621D6
S3150800B7184FF4E85000F0CAFA00BF80BD380300208D
S3150800B728B4030020AC03002080B584B000AF78606D
S3150800B7387B681B0EDBB23B727B681B0CDBB27B7229
S3150800B7487B681B0ADBB2BB727B68DBB2FB7207F14C
S3150800B7580803042204214FF4F85000F0A7FA00BFA2
S3150800B7681037BD4680BD000080B58AB000AF07F126
S3150800B778140300221A605A609A60DA607D4B9B6946
S3150800B7887C4A43F0100393617A4B9B6903F01003D4
S3150800B7983B613B69774B9B69764A43F0040393619F
S3150800B7A8744B9B6903F00403FB60FB68714B9B6948
S3150800B7B8704A43F0080393616E4B9B6903F00803CC
S3150800B7C8BB60BB686B4B9B696A4A43F0400393614D
S3150800B7D8684B9B6903F040037B607B68654B9B69F4
S3150800B7E8644A43F020039361624B9B6903F0200384
S3150800B7F83B603B68002230215F4805F072F800225A
S3150800B8084FF4F8515D4805F06CF800224FF40041F2
S3150800B8185B4805F066F8002218215A4805F061F8D1
S3150800B82800228021584805F05CF802237B61002332
S3150800B838BB610023FB6107F114031946504804F05D
S3150800B848B5FE04237B610023BB610223FB6107F174
S3150800B858140319464A4804F0A9FE30237B610123DC
S3150800B868BB610023FB6102233B6207F114031946F7
S3150800B878414804F09BFE44F282037B610023BB61C6
S3150800B8880023FB6107F1140319463C4804F08EFEB1
S3150800B8984FF4F8537B610123BB610023FB61022344
S3150800B8A83B6207F114031946344804F07FFE4FF447
S3150800B8B800437B610123BB610023FB6102233B62D2
S3150800B8C807F1140319462E4804F070FE18237B6105
S3150800B8D80123BB610023FB6102233B6207F11403C2
S3150800B8E81946284804F062FE80237B610023BB6161
S3150800B8F80023FB6107F114031946224804F056FE93
S3150800B90818237B610023BB610023FB6107F114033D
S3150800B91819461D4804F04AFE80237B610123BB6152
S3150800B9280023FB6102233B6207F1140319461648F4
S3150800B93804F03CFE4FF440737B611223BB6103237A
S3150800B9483B6207F1140319460F4804F02FFE0F4B04
S3150800B9585B687B627B6A43F0E0637B627B6A43F0E1
S3150800B96802037B62094A7B6A536000BF2837BD46D3
S3150800B97880BD00BF001002400010014000180140B9
S3150800B9880008014000140140000C01400000014075
S3150800B99890B5CDB040AF786007F10C0300221A6065
S3150800B9A85A6007F10C0307F114020021786804F0BD
S3150800B9B831F80346002B40F05381BB699BB245F228
S3150800B9C8F462934240F04C81BB691B0A03F47F4337
S3150800B9D8B3F56C4F13D0B3F56C4F00F20C81B3F581
S3150800B9E86B4F57D0B3F56B4F00F20581B3F5C85FB7
S3150800B9F800F0DD80B3F5F05F00F0B680FBE03B7B36
S3150800BA08102B3ED17B7B1AB2BB7B1BB21B021BB227
S3150800BA1813431BB29AB2944BA3F80421924B012202
S3150800BA2883F80721FA7B904B83F806218E4B02226E
S3150800BA3883F808218C4B93F808218B4B83F8092146
S3150800BA48FB7C1A04BB7C1B0213437A7C13431A46F5
S3150800BA58854BC3F80021844BB3F80431FF2B10D863
S3150800BA68814C684604F110034FF48072194608F0B1
S3150800BA789FFC94E80F0000F041F97B4B012283F8FC
S3150800BA880A213B7BFF2B40F0E680774B002283F8A0
S3150800BA980A21E0E0744B93F80A31012B40F0DD8067
S3150800BAA83B7B002B00F0DB803B7B222B00F2D78008
S3150800BAB86D4B93F807213B7B9A4240F0D0803B7B3D
S3150800BAC85A1E1346DB009B1A674A981807F10C0397
S3150800BAD801330722194608F06BFC634B93F80731C4
S3150800BAE80133DAB2604B83F807215F4B93F80721D5
S3150800BAF85D4B93F806319A4211D95B4C684604F1B6
S3150800BB0810034FF48072194608F052FC94E80F00A7
S3150800BB1800F03AF9544B022283F80A219FE0524B67
S3150800BB2893F80931002B07D04F4B93F80931013B9D
S3150800BB38DAB24D4B83F809214B4B93F80931002BA0
S3150800BB4840F08D80484C684604F110034FF4807223
S3150800BB58194608F02DFC94E80F0000F0CFF8424B80
S3150800BB68022283F809217AE040490420FFF7F6FC07
S3150800BB783B7B19467B7B1846BB7BFA7B0192009375
S3150800BB8803460A463A490420FFF7E8FC3B7C19466F
S3150800BB987B7C1846BB7CFA7C0192009303460A46CE
S3150800BBA834490420FFF7DAFCFFF746F858E032492B
S3150800BBB80720FFF7D3FC3B7B19467B7B1846BB7BE4
S3150800BBC8FA7B0192009303460A462C490720FFF799
S3150800BBD8C5FC3B7C19467B7C1846BB7CFA7C0192E3
S3150800BBE8009303460A4623490720FFF7B7FC24486B
S3150800BBF8FEF7C4FF34E01C4B93F80A31002B2FD10B
S3150800BC087B6A9AB2184BA3F80421174B012283F8CA
S3150800BC180721154B012283F80621134B012283F8C5
S3150800BC280821114B002283F80921BB691B0A03F472
S3150800BC387F430D4AC2F800310B4B022283F80A21CA
S3150800BC48094BB3F804311A4607F10C031946064896
S3150800BC5808F0AEFB04E000BF02E000BF00E000BF4A
S3150800BC6800BF3437BD4690BD74080020906B0108A4
S3150800BC78B46B0108D06B0108E86B0108046C01086D
S3150800BC88F0F0004080B500AF074803F077FDFDF7F0
S3150800BC98E3FE00F0B3F8044803F02CFD022102483D
S3150800BCA803F0D9FF00BF80BDA402002080B58CB080
S3150800BCB800AFF8607B600B46FB721346BB72FB7AD3
S3150800BCC89A06FB681B02134343F4744343F056036E
S3150800BCD8FB6100237B6204233B62BB7ABB6207F1E4
S3150800BCE8140307F118017A68034803F090FD00BFAA
S3150800BCF83037BD4680BD00BFA402002084B080B599
S3150800BD0882B000AF07F1100C8CE80F0011233B70C6
S3150800BD1897F818317B7097F818311A4697F816313C
S3150800BD28194697F81731CB1A01339A4208DD97F85E
S3150800BD38162197F81731D31ADBB20133DBB27B70B9
S3150800BD4897F81731BB70FF23FB70FF233B71D7F8B1
S3150800BD581031DBB27B71D7F810311B0ADBB2BB7125
S3150800BD68D7F810311B0CDBB2FB713B4608220721BA
S3150800BD784FF46C40FFF79AFF00BF0837BD46BDE889
S3150800BD88804004B07047000084B080B582B000AF28
S3150800BD9807F1100C8CE80F0013233B70164BB3F809
S3150800BDA80431DBB27B70144BB3F804311B0A9BB21F
S3150800BDB8DBB2BB70104B93F80631FB70FF233B715F
S3150800BDC8D7F81031DBB27B71D7F810311B0ADBB212
S3150800BDD8BB71D7F810311B0CDBB2FB713B46082246
S3150800BDE807214FF46C40FFF761FF00BF0837BD46CF
S3150800BDF8BDE8804004B070477408002080B58AB052
S3150800BE0800AF00237B610023BB610123FB6100238C
S3150800BE183B6000237B600023BB600023FB60002394
S3150800BE283B6101233B623B461946064803F082FB01
S3150800BE380346002B01D000F0D3FA00BF2837BD46C9
S3150800BE4880BD00BFA402002080B483B000AF0346BB
S3150800BE58FB71FB79002B14BF01230023DBB21A46BA
S3150800BE68044B9A70034B00221A7200BF0C37BD4662
S3150800BE7880BC70470800002080B500AF0A4B1B78C5
S3150800BE88002B05D08021094804F014FD034609E073
S3150800BE988021064804F00EFD0346002B0CBF01233B
S3150800BEA80023DBB2184680BD0400002000180140B4
S3150800BEB880B483B000AF0346FB71044AFB7913705C
S3150800BEC800BF0C37BD4680BC704700BF080000207D
S3150800BED880B582B000AF02F0FDFC786000F004F986
S3150800BEE8724B5B78002B40F0DD80FFF7C5FF0346F1
S3150800BEF8002B0CBF01230023FB706C4B1B78002B0F
S3150800BF080CBF01230023BB70684B9B78FF2B04D119
S3150800BF18FA78BB789A4200F0AD80644B9B78FF2B81
S3150800BF2809D1BB7883F00103DBB21A465F4B9A70D6
S3150800BF385E4B00221A725D4BDB78022B4AD0022B25
S3150800BF4800F3B180002B02D0012B2AD0ABE0584B66
S3150800BF581B78002B0FD0554B9B78012B05D1012256
S3150800BF682021544804F0BDFC14E001221021514850
S3150800BF7804F0B7FC0EE04D4B9B78012B05D1012246
S3150800BF8810214C4804F0ADFC04E001222021494860
S3150800BF9804F0A7FC454B0122DA70444A7B685360D3
S3150800BFA867E0424B5B687A68D31A434A1288934219
S3150800BFB85CD3002210213F4804F093FC002220217C
S3150800BFC83C4804F08EFC394B0222DA70374A7B6803
S3150800BFD853604BE0354B5B687A68D31A312B47D9DF
S3150800BFE8FFF74AFF0346002B0CBF01230023FB700B
S3150800BFF8FB782E4A9278002A0CBF01220022D2B278
S3150800C00893420CBF012300237B707B78002B09D051
S3150800C018264BFF229A70254B0022DA70234B002202
S3150800C0281A7225E0214B1B7A0133DAB21F4B1A72B2
S3150800C0381E4B1A7A214B1B789A4213D31B4B0122A3
S3150800C0485A701A4A7B68D360184B00229A70174BA5
S3150800C0580022DA70154B00221A7219490420FFF7D4
S3150800C0687DFA05E0114B0022DA7001E000BF1AE0FC
S3150800C07800BF18E00D4BDB78002B0CD000221021EE
S3150800C0880C4804F02EFC002220210A4804F029FC5A
S3150800C098064B0022DA70054BFF229A70034B0022E2
S3150800C0A81A7200E000BF0837BD4680BD08000020A8
S3150800C0B8050000200010014006000020136D010845
S3150800C0C8206C010880B500AF054B00225A70044B56
S3150800C0D80022DA6003490720FFF740FA00BF80BD4F
S3150800C0E8080000202C6C010880B500AF0A4B5B7865
S3150800C0F8002B0FD0084BDB68002B0BD002F0EAFBAD
S3150800C1080246054BDB68D21A044B1B689A4201D3D0
S3150800C118FFF7D8FF00BF80BD08000020146D01088E
S3150800C12880B400AF034B044A9A6000BFBD4680BC82
S3150800C138704700BF00ED00E00080000880B485B0B5
S3150800C14800AF03460A46FB711346BB71BB791F2B22
S3150800C15801D900230EE00023FB73BB79084AD35C98
S3150800C168FA799A4201D00123FB73BB790449FA7913
S3150800C178CA54FB7B18461437BD4680BC704700BFB7
S3150800C1888409002080B584B000AF786002F0A2FB6D
S3150800C198B8607B68FB60FB68B3F1FF3F12D0104BB1
S3150800C1A81B781A46FB681344FB600BE0FEF7FAFF98
S3150800C1B8FFF78EFEFEF716FEFDF736FE00F0F4FFD3
S3150800C1C801F008F902F086FB0246BB68D31AFA683A
S3150800C1D89A42EBD800BF00BF1037BD4680BD00BFE6
S3150800C1E88000002080B500AF0320FDF7EFFA03466C
S3150800C1F8002B02D1024B01221A7000BF80BD00BF76
S3150800C208F802002080B582B002AFFFF789FF02F076
S3150800C21809FB04F08BFB00F073F8FFF7A5FAFDF7A6
S3150800C228CFF9FDF719FCFDF74DFC01F05BF801F0B5
S3150800C238EFFF02F02FF9FFF779F802F0D7F802F0C6
S3150800C248FFF802F051F9FDF713FB00F08DFF4FF4E4
S3150800C258967002F049FBFDF7A9FD01F0A7F800233F
S3150800C268012222490720FFF779F901F07BF8204BCC
S3150800C2781B889BB21A461F490720FFF76FF91C4B04
S3150800C2889B781A461C490720FFF768F9184B9B88BC
S3150800C2989BB21A46164BDB889BB21946144B1B8968
S3150800C2A89BB200930B4615490720FFF757F9FDF788
S3150800C2B89BFDFFF7E7FC00F07DFAFDF717FD00F098
S3150800C2C887FB00F023FC0A20FFF75CFF00F08EF8D6
S3150800C2D8FDF722FD00F00EFE0A20FFF753FFFFF7D1
S3150800C2E881FF3220FFF74EFF00BFE8E7406C0108E0
S3150800C2F8140F0020546C0108686C01087C6C01084E
S3150800C30880B59CB000AF07F13803382200211846DB
S3150800C31807F040FF07F1240300221A605A609A6062
S3150800C328DA601A613B1D20220021184607F032FF01
S3150800C3380523BB634FF480333B6404237B640123E2
S3150800C348BB640123FB644FF48033FB630223BB659C
S3150800C3584FF48033FB654FF4E0133B6602237B6694
S3150800C3684FF4C063BB664023FB6607F138031846DB
S3150800C37804F0ACFB0346002B01D000F031F80F237C
S3150800C3887B620223BB620023FB624FF480633B6334
S3150800C39800237B6307F124030221184604F0ACFE48
S3150800C3A80346002B01D000F01BF803237B604FF4EB
S3150800C3B88073BB604FF40043FB603B1D184605F0CD
S3150800C3C891F80346002B01D000F00AF8034B012226
S3150800C3D81A6000BF7037BD4680BD00BF7000424274
S3150800C3E880B400AF72B600BF00BFFDE72DE9B043C1
S3150800C3F884B000AF2E4B00221A712E4B5B78082B9F
S3150800C40804D12B4B012283F8242003E0284B002271
S3150800C41883F8242002F05EFAF860254B9B68FA68D0
S3150800C428D31ABB60224AFB689360224BD3F80330C1
S3150800C438BA6802FB03F3204AA2FB03239B097B6025
S3150800C4481B4BD3E90423796800200C46054612EBF2
S3150800C458040843EB0509164BC3E90489144BD3E9C9
S3150800C4680423164BA3FB0223DB0A114A9361104BDC
S3150800C47893F82430002B08D00D4B9A690C4BDB69CE
S3150800C488D31A0C4AC2F807300CE00A4B0022DA71B4
S3150800C49800221A7200225A7200229A72044B9B6969
S3150800C4A8034AD36100BF1037BD46BDE8B08300BF55
S3150800C4B8A8090020F8020020D34D6210C5B3A2913E
S3150800C4C880B582B000AF0346FB71064AFB79D37183
S3150800C4D802F000FA0346034A136100BF0837BD464F
S3150800C4E880BD00BF140A002080B500AF02F0F2F93B
S3150800C4F80246024B1B69D31A184680BD140A002047
S3150800C50880B584B000AF7860884B894A012178687D
S3150800C51803F080FA0346002B40F00481844B5B68DD
S3150800C528BB603B7A002B40F0FC8002F0D3F9034647
S3150800C538804A1360BB7A03F03F03DBB2022B05D1AE
S3150800C5487D4B7A4A92E8030083E80300BB7A03F036
S3150800C5583F03DBB2042B19D1784B744A92E80300DF
S3150800C56883E80300754B1B791A46754BDA61734BDA
S3150800C5781A7A734B83F82020704BDA79704B83F854
S3150800C58821206E4B9A796E4B83F82220BB7A03F0EA
S3150800C5983F03DBB2062B23D16A4B644A92E80300B1
S3150800C5A883E80300674B5B781A46664B1B781B02C1
S3150800C5B813441A46634B9A60624BDB781A46614BFA
S3150800C5C89B781B0213441A465E4BDA605D4B5B790F
S3150800C5D81A465C4B1B791B0213441A46594B1A61B7
S3150800C5E8BB7A03F03F03DBB2082B05D1564B4F4AFB
S3150800C5F892E8030083E80300BB7A03F03F03DBB243
S3150800C608092B40F08F80514B484A92E8030083E88B
S3150800C61803004E4BDB791A464C4BDA604B4BDA680B
S3150800C6284A4B9B791B021343484AD360474BDA683F
S3150800C638464B5B791B041343444AD360434BDA6879
S3150800C648424B1B791B061343404AD3603F4BDB78A2
S3150800C6581A463E4B9A603D4B9A683C4B9B781B02A0
S3150800C66813433A4A9360394B9A68384B5B781B04EC
S3150800C6781343364A9360354B9A68344B1B781B0626
S3150800C6881343324A9360314B9B68314AA2FB032312
S3150800C6989B09FB812D4BDB682E4AA2FB03235B090A
S3150800C6A8BB81274AFB895380254ABB899380FB8926
S3150800C6B8132B8CBF01230023DBB21A46204B9A7230
S3150800C6C81F4B01221A721D4B1A791D4B9A711C4B66
S3150800C6D8DB79012B26D91A4B5A881F4BA3F8132046
S3150800C6E8174BB3F904309AB21B4BA3F815201A4B0B
S3150800C6F8B3F815309BB21A46174BB3F813309BB2EA
S3150800C70802FB03F3154A82FB03129210DB17D31AAE
S3150800C7181A46114BC3F80320094B9A7A0E4B1A7618
S3150800C72800E000BF1037BD4680BD00BF580A00208C
S3150800C7383C0A0020380A0020D0090020DC0900201D
S3150800C748140A0020E8090020FC090020040A002031
S3150800C758D34D62101F85EB51F8020020676666669E
S3150800C76880B58AB000AF0E237B610023BB61012325
S3150800C778FB6100233B6000237B600023BB6000232A
S3150800C788FB6000233B6101233B6201233B610E23C7
S3150800C7987B623B461946064802F0CCFE0346002B48
S3150800C7A801D0FFF71DFE00BF2837BD4680BD00BF74
S3150800C7B8CC02002080B500AF134802F0DFFFFDF772
S3150800C7C881F9FFF7CDFF104802F094FF10210E48B3
S3150800C7D803F041FA242200210C4807F0DBFC0B4B36
S3150800C7E80022DA7102F076F80346084A1361074B05
S3150800C7F847F230525A61054B00221A76002100206A
S3150800C80800F006F800BF80BDCC020020140A0020FC
S3150800C81880B584B000AF03460A46FB711346BB7160
S3150800C82807F1080308220021184607F0B3FCFB792C
S3150800C838002B15D10D4B1B7A002B13D0BB79002B77
S3150800C8480CBF01230023DBB23B72F97907F1080311
S3150800C8581A22F02000F066F81420FFF793FC02E08D
S3150800C86800BF00E000BF1037BD4680BD140A00208F
S3150800C87880B586B000AF0346FB710B46BB801346EE
S3150800C8887B8007F1080308220021184607F082FC76
S3150800C898FB79002B40D1BB88952B01D89623BB8002
S3150800C8A81F4B1B7E002B06D1BB88B3F5FA7F02D334
S3150800C8B840F2F313BB807B88642202FB03F37B6197
S3150800C8C8BB884FF47A7202FB03F33B617B691B0E44
S3150800C8D8DBB23B737B691B0CDBB27B737B691B0A78
S3150800C8E8DBB2BB737B69DBB2FB733B691B0EDBB23E
S3150800C8F83B723B691B0CDBB27B723B691B0ADBB2DA
S3150800C908BB723B69DBB2FB72F97907F108031C2293
S3150800C918F02000F007F800E000BF1837BD4680BDD4
S3150800C928140A002080B58CB000AF3B600346FB7143
S3150800C9380B46BB7113467B71FB7987F82830BB79A0
S3150800C94887F829307B7903F03F03DAB297F82A305B
S3150800C95862F3050387F82A307B8D0A2262F3891366
S3150800C9687B850A2387F82F30BB6A7B610023FB6126
S3150800C9780423BB6108233B621EE0144803F016F83B
S3150800C9880346002B0ED007F10C0307F110013A688D
S3150800C9980E4802F03CFF034687F82E3097F82E30EB
S3150800C9A8002B0ED00120FFF7EDFB97F92F30DBB2ED
S3150800C9B8013BDBB287F82F3097F92F30002BDCDCE8
S3150800C9C800E000BF3037BD4680BD00BFCC0200205E
S3150800C9D880B582B000AF3B4600221A605A603B46D3
S3150800C9E804220021F020FFF79DFF1420FFF7CAFB59
S3150800C9F83B4606220021F020FFF794FF1420FFF794
S3150800CA08C1FB3B4609220021F020FFF78BFF1420C3
S3150800CA18FFF7B8FB394BB3F81B309BB2384AA2FB71
S3150800CA280323DB089BB21A46344BB3F813309BB280
S3150800CA3802FB03F31A46334B5B699A4211D9314B09
S3150800CA485A6913469B0013445B001A462B4BB3F8E6
S3150800CA5813309BB2B2FBF3F39AB2284BA3F8112012
S3150800CA6806E0264BB3F81B309AB2244BA3F81120DC
S3150800CA78224BB3F811309BB2B3F57A7F08D91F4B0E
S3150800CA88002262F017025A74002242F003029A74CE
S3150800CA981A4BB3F811309BB21A46184BB3F80F3035
S3150800CAA89BB202FB03F3184A82FB03129210DB17A8
S3150800CAB8D31A1A46114BC3F80B20124B5B7A002B74
S3150800CAC818D00E4BB3F80F309BB20C4AB2F81120A7
S3150800CAD892B219460020FFF7CBFE1420FFF752FB47
S3150800CAE8064BB3F813309BB2B3F5F57F02D9054B5D
S3150800CAF801221A7600BF0837BD4680BDF802002015
S3150800CB08CDCCCCCC140A00206766666698B500AF0B
S3150800CB1801F0E0FE0246B44B1B68D31AB3F5FA7F58
S3150800CB2820D9B24B00221A72B04B00229A72B04B27
S3150800CB3800221A71AE4B00221A72AD4B0022DA7126
S3150800CB48AB4B00229A71AB4B00229A60A94B002284
S3150800CB58DA60A84B00221A61A74B0022DA60A64BB6
S3150800CB6800229A60A14B1B7A002B03D09F4B1B7897
S3150800CB78002B0CD1A14B0022DA7400221A759F4BA0
S3150800CB8800225A7500229A759C4B00221A769B4BEE
S3150800CB989B7F002B0CD001210420FCF7A3FD01F094
S3150800CBA899FE0346964A1360904B01221A7010E0C4
S3150800CBB801F090FE0246924B1B68D31A4EF6602285
S3150800CBC8934206D900210420FCF78CFD874B0022E6
S3150800CBD81A700520FCF7FAFD03461A46834BDA72E3
S3150800CBE8824B1B7A002B07D0804B1B7B002B03D16B
S3150800CBF87E4B1B78002B02D17C4B00225A727B4B4A
S3150800CC08DB79092B00F2558101A252F823F000BFFF
S3150800CC1841CC000875CC000891CC0008C9CC00089E
S3150800CC2817CD000859CD0008C3CD00086DCE0008F9
S3150800CC381DCE0008A7CE00086C4B00225A700021AA
S3150800CC480320FCF74FFD694B1B7A002B00F0358152
S3150800CC58664B1B78002B00F03081644B1B7B002B3E
S3150800CC6840F02B810120FFF72BFC26E1FFF73CFC5F
S3150800CC780346B3F57A6F40F222815C4B01225A7259
S3150800CC880220FFF71DFC1AE1584B00221A760021EC
S3150800CC980320FCF727FD554B5B7A002B03D10020B0
S3150800CCA8FFF70EFC1CE1554BDB7D002B00F00981D4
S3150800CCB801210020FFF7ACFD0320FFF701FC00E186
S3150800CCC84A4B9B7A002B0CD0484B5B7A002B08D032
S3150800CCD801F000FE03464B4A13600420FFF7F0FBF9
S3150800CCE8F1E0FFF701FC034642F21072934240F264
S3150800CCF8EA803E4B01225A73404B0A225A77002093
S3150800CD08FFF7DEFB40490420FEF728FCDBE001219B
S3150800CD180320FCF7E7FC354BDB7A002B03D005200C
S3150800CD28FFF7CEFBD1E0FFF7DFFB0346B3F57A7FC3
S3150800CD3840F2CB802D4B01221A73304B07225A77C3
S3150800CD480620FFF7BDFB31490420FEF707FCBCE0C7
S3150800CD582A4BDB7D002B03D0244B5B7A002B03D1AF
S3150800CD680620FFF7ADFBBBE00520FCF72FFD0346C1
S3150800CD781C460320FCF71AFD03469C4217D001F00F
S3150800CD88A9FD0246224B1B68D31AB3F57A7F40F2EF
S3150800CD989E801A4B07225A77144B01221A730620CB
S3150800CDA8FFF78EFB19490420FEF7D8FB8FE001F040
S3150800CDB891FD0346164A136089E0104B00225A74FF
S3150800CDC800229A740D4BB3F815309BB21D2B06D961
S3150800CDD8FFF78AFB034641F28832934279D908203D
S3150800CDE8FFF76EFB75E000BF380A0020140A00201A
S3150800CDF8DC090020E8090020040A0020F8020020BF
S3150800CE08600A0020640A0020946C0108A46C0108D2
S3150800CE18680A002000210320FCF764FC314BDB7A02
S3150800CE28002B07D100210020FFF7F2FC0720FFF7A7
S3150800CE3847FB50E0FFF758FB0346B3F57A7F4AD914
S3150800CE48284B01221A73284B07225A7700210020FB
S3150800CE58FFF7DEFC0720FFF733FB24490420FEF71B
S3150800CE687DFB38E01F4B9B7A002B03D10920FFF77F
S3150800CE7827FB32E0FFF738FB034642F2107293426B
S3150800CE882BD9184B01225A73174B0A225A770020B6
S3150800CE98FFF716FB16490420FEF760FB1DE0FFF7AF
S3150800CEA823FB0346B3F57A6F19D90220FFF708FB67
S3150800CEB815E00020FFF704FB12E000BF10E000BFF2
S3150800CEC80EE000BF0CE000BF0AE000BF08E000BFA4
S3150800CED806E000BF04E000BF02E000BF00E000BFB4
S3150800CEE800BF98BD140A0020F8020020A46C0108A7
S3150800CEF8C46C010880B500AF344B5B7F002B03D0A8
S3150800CF08334800F01FF95FE0304B5B780D2B57D894
S3150800CF1801A252F823F000BF59CF000861CF0008D4
S3150800CF2869CF000871CF000879CF000881CF0008BB
S3150800CF3889CF000891CF000899CF0008A1CF00082B
S3150800CF48A9CF0008B1CF0008B9CF0008C1CF00089B
S3150800CF58204800F0F7F837E01F4800F0F3F833E008
S3150800CF681B4800F0EFF82FE01C4800F0EBF82BE020
S3150800CF781A4800F0E7F827E0194800F0E3F823E034
S3150800CF88174800F0DFF81FE0154800F0DBF81BE04B
S3150800CF98134800F0D7F817E0124800F0D3F813E062
S3150800CFA8104800F0CFF80FE00E4800F0CBF80BE079
S3150800CFB80C4800F0C7F807E0084800F0C3F803E093
S3150800CFC8044800F0BFF800BF80BD00BFF802002083
S3150800CFD854000020180000202400002030000020FB
S3150800CFE83C0000204800002080B487B000AFF860F5
S3150800CFF8B96011461A460B46FB801346BB80FA8869
S3150800D008BB889A4201D9BB88FB80BB88002B01D113
S3150800D0180123BB80FA8813461B029A1ABB8892FB1F
S3150800D028F3F3FB82FB681B781A46FB8AC3F1FF03F6
S3150800D03803FB02F2BB681B781946FB8A01FB03F35C
S3150800D0481344204A82FB03121A44D211DB17D31A57
S3150800D058DAB23B6A1A70FB685B781A46FB8AC3F130
S3150800D068FF0303FB02F2BB685B781946FB8A01FBE0
S3150800D07803F31344134A82FB03121A44D211DB172B
S3150800D088D31ADAB23B6A5A70FB689B781A46FB8A47
S3150800D098C3F1FF0303FB02F2BB689B781946FB8AB8
S3150800D0A801FB03F31344074A82FB03121A44D211FD
S3150800D0B8DB17D31ADAB23B6A9A7000BF1C37BD462B
S3150800D0C880BC70478180808080B483B000AF786068
S3150800D0D87B681B781A46642302FB03F3174A82FB0C
S3150800D0E803121A44D211DB17D21A154B1B689A6316
S3150800D0F87B685B781A46642302FB03F30F4A82FBB4
S3150800D10803121A44D211DB17D21A0D4B1B68DA63BD
S3150800D1187B689B781A46642302FB03F3074A82FB5B
S3150800D12803121A44D211DB17D21A054B1B681A6464
S3150800D13800BF0C37BD4680BC704700BF8180808021
S3150800D148240F002080B483B000AF7860054B7A6856
S3150800D1581068516803C312891A8000BF0C37BD4688
S3150800D16880BC7047740A002080B582B000AF0023DF
S3150800D1783B7100237B710023BB710421094804F025
S3150800D188E5FD0821074804F0E1FD0C21054804F0EF
S3150800D198DDFD3B1D1846FFF797FF00BF0837BD465C
S3150800D1A880BD00BF240F002080B582B002AF01F011
S3150800D1B891FB0246464B1B68D31A142B40F285800E
S3150800D1C801F088FB0346424A1360424B5B880133E9
S3150800D1D89AB2404B5A803F4B1B78032B67D801A25B
S3150800D1E852F823F0FDD100082FD200085BD20008B8
S3150800D1F88DD20008374B5A88374BDB781946374B98
S3150800D20800930B4634493648FFF7EEFE314B5B88E8
S3150800D218314AD27893424ED92E4B01221A702D4B99
S3150800D22800225A8047E02B4B2B4A043312681146D2
S3150800D23819800233120C1A70264B5B88264A127913
S3150800D24893423AD9234B02221A70224B00225A805B
S3150800D25833E0204B5A88204B5B7919461F4B0093BD
S3150800D2680B461F491C48FFF7BFFE1A4B5B881A4A2C
S3150800D2785279934223D9174B03221A70154B002269
S3150800D2885A801CE0134B144A0433073211889278E3
S3150800D29819809A700F4B5B880F4A9279934210D976
S3150800D2A80C4B00221A700B4B00225A8009E0094BD6
S3150800D2B800221A7006E000BF04E000BF02E000BFC3
S3150800D2C800E000BF0548FFF7FFFE00BFBD4680BD6A
S3150800D2D8800A00206C0A0020740A0020700A0020C0
S3150800D2E87B0A002080B500AF0A4B0B4A1A60094B27
S3150800D2F84FF0FF325A60074B4FF480729A60054820
S3150800D30804F074FB0346002B01D0FFF769F800BF49
S3150800D31880BD00BF840A00200028004080B584B07C
S3150800D32800AF78607B681B680B4A934210D103F0FC
S3150800D338F1FA0A4BDB69094A43F00063D361074BE4
S3150800D348DB6903F00063FB60FB68054B01221A6082
S3150800D35800BF1037BD4680BD0028004000100240B7
S3150800D3683C04424280B400AF0E4B1B681B689AB255
S3150800D3780D4B1A800B4B1B685A790B4B9A70094B45
S3150800D3881B681A79084BDA70074B01229A80064BF4
S3150800D3980022DA80044B01221A8100BFBD4680BCF0
S3150800D3A8704700BF00000020140F002080B500AFAA
S3150800D3B84FF404720021054806F0ECFE4FF4047297
S3150800D3C80021034806F0E6FE00BF80BD980A002043
S3150800D3D8A80C002080B500AF2A4B93F84230DBB280
S3150800D3E8202B0AD1284B93F80832DBB2002B04D13C
S3150800D3F8FF222649234805F082FA254B93F842303E
S3150800D408DBB2202B04D1FF222249214805F077FAFE
S3150800D4181C4B93F84130DBB2212B19D11A4BD3F8A0
S3150800D4280C32002B14D001F055FA0246164BD3F8E5
S3150800D4380C32D31A642B0BD9124805F0BDFA002210
S3150800D4481021154803F04DFA0F4B0022C3F80C2299
S3150800D4580D4B93F80832DBB2002B11D0094B93F821
S3150800D4684130DBB2212B0BD00C4800F0DFF9FF2244
S3150800D4780649044805F043FA034B002283F80822B4
S3150800D48800BF80BDFC0F0020980A0020980B0020DA
S3150800D4986C0F0020A80D002000140140980C0020ED
S3150800D4A880B582B000AF78600B467B807B681A68C7
S3150800D4B81C4B1B689A4216D17B881A461A491B4880
S3150800D4C800F080F90346002B04D11422002100201D
S3150800D4D800F0ECF8164B00221A70FF221249114880
S3150800D4E805F00DFA19E07B681A68124B1B689A4210
S3150800D4F813D17B881A461049104800F063F9034689
S3150800D508002B05D00A4B01221A700D4800F08EF937
S3150800D518FF220949074805F0F2F900BF0837BD4652
S3150800D52880BD00BFFC0F0020980B0020980A002039
S3150800D538B80E00206C0F0020A80D0020A80C0020AB
S3150800D548A80E002080B582B000AF78607B681A689C
S3150800D558084B1B689A4208D100221021064803F096
S3150800D568C0F9064B0022C3F80C2200BF0837BD468F
S3150800D57880BD00BFFC0F002000140140980A002057
S3150800D58880B485B000AF78600B467B804FF0FF33D8
S3150800D598FB6000237B8121E07B897A6813441B782A
S3150800D5A81A46FB685340FB6000237B7210E0FB6851
S3150800D5B803F00103002B05D0FB685A080D4B5340AE
S3150800D5C8FB6002E0FB685B08FB607B7A01337B72D1
S3150800D5D87B7A072BEBD97B8901337B817A897B8810
S3150800D5E89A42D9D3FB68DB4318461437BD4680BC34
S3150800D5F8704700BF2083B8ED80B588B000AFF860E3
S3150800D6087A601A460B467B8113467B720023FB8396
S3150800D618FB8B5A1CFA831A467B6813447A7A1A7063
S3150800D628FB68002B19D00023BB8312E0BB8BFA6872
S3150800D6381A44FB8B591CF98319467B680B441278E4
S3150800D6481A70FB8BFA2B01D900232AE0BB8B01330E
S3150800D658BB83BA8B7B899A42E8D3FB8B19467868D1
S3150800D668FFF78EFF03463B6107F110037B61002332
S3150800D678BB6112E0BB697A691A44FB8B591CF983AA
S3150800D68819467B680B4412781A70FB8BFE2B01D956
S3150800D698002306E0BB690133BB61BB69032BE9DDDF
S3150800D6A8FB8B18462037BD4680BD000080B584B080
S3150800D6B800AF78600B467B8013467B707B78798849
S3150800D6C8154A7868FFF798FF0346FB81FB89002B04
S3150800D6D81ED0124B93F84130DBB2212B07D10F48E5
S3150800D6E805F06AF9002210210D4803F0FAF801221C
S3150800D6F810210B4803F0F5F8FB891A46064907482E
S3150800D70805F0C8F801F0E6F80346034AC2F80C32F1
S3150800D71800BF1037BD4680BD980A0020FC0F0020C0
S3150800D7280014014080B588B000AFF8600B467A60EF
S3150800D7387B817B89042B01D800233FE07B89B3F5DD
S3150800D748807F01D9002339E07B89043BFB83FB8B67
S3150800D758FA6813441B781946FB8B0133FA68134495
S3150800D7681B781B0241EA0302FB8B0233F9680B4458
S3150800D7781B781B041A43FB8B0333F9680B441B7885
S3150800D7881B061343BB61FB8B1946F868FFF7F8FEBF
S3150800D7987861BA697B699A4201D000230EE0FB6872
S3150800D7A85A1C7B685A60FB681A787B681A70FB8B68
S3150800D7B8DBB2013BDAB27B685A7001231846203778
S3150800D7C8BD4680BD80B584B000AFF860B960134621
S3150800D7D8FB80FB6803F50072FB881946B868FFF7F3
S3150800D7E8A1FF0346002B01D1002304E0FB680122B0
S3150800D7F883F80822012318461037BD4680BD000065
S3150800D80880B400AFBFF34F8F00BF064BDB6803F445
S3150800D818E0620449044B1343CB60BFF34F8F00BF44
S3150800D82800BFFDE700ED00E00400FA0580B584B006
S3150800D83800AF78601323FB737B681B78C22B00F351
S3150800D848D080B02B0FDA602B42D0602B00F3C9804A
S3150800D858502B43D0502B00F3C480012B00F0AA802C
S3150800D868402B2DD0BDE0B03B122B00F2BA8001A2A6
S3150800D87852F823F0EBD80008EBD90008EBD90008D2
S3150800D888EBD90008EBD900089BD90008EBD90008A2
S3150800D898EBD90008EBD90008EBD90008EBD9000842
S3150800D8A8EBD90008EBD90008EBD90008EBD9000832
S3150800D8B8EBD9000831D9000895D9000869D90008B4
S3150800D8C800F0B6F8402258214D48FFF7EFFE93E0DE
S3150800D8D860220A214B48FFF7E9FE8DE0FDF7DCFDDB
S3150800D8E88AE07B685B780B2B1BD17B685A68464BAA
S3150800D8F81068516803C31189927A19809A70FCF7DF
S3150800D90873FA424B01221A70FCF76EFA3E4BD3F8AB
S3150800D91803303D4A3E490720FDF720FE1223FB73D4
S3150800D92862E01323FB735FE07B685B78012B14D1F5
S3150800D9387B685B681B781A464FF47A7302FB03F315
S3150800D9481A46344B5A61334B5B691A4632490720E3
S3150800D958FDF704FE1223FB7346E01323FB7343E02B
S3150800D9687B685B78012B0ED17B685B681A782B4B32
S3150800D9781A702A4B1B781A4629490720FDF7EEFD27
S3150800D9881223FB7330E01323FB732DE01323FB7379
S3150800D9982AE0122200210020FFF788FE00BF214B4B
S3150800D9A893F84130DBB2212BF9D00A2000F09CFF0E
S3150800D9B8FFF726FF7B685B78092B0FD17B685A68C7
S3150800D9C8194B1068516803C3127A1A70174B1B78DB
S3150800D9D8DBB2012B0FD01223FB7305E01323FB736D
S3150800D9E802E01323FB7300BFFB7B1A4600210020C5
S3150800D9F8FFF75CFE00E000BF1037BD4680BD00BFDC
S3150800DA08BC0E0020140F00206C0000201E0F0020FA
S3150800DA18D86C0108140A0020EC6C0108F8020020EA
S3150800DA28006D0108FC0F002060000020B80E0020D9
S3150800DA38B0B500AF9D4B9A789D4B9A709B4BD3F81F
S3150800DA4807309B4AC2F80330984BB3F80F309AB29E
S3150800DA58974BA3F80720954BB3F81B309AB2944B0B
S3150800DA68A3F80920914BB3F813309AB2904BA3F850
S3150800DA780B208E4BB3F815309AB28D4BA3F80D20B0
S3150800DA888A4B1A7E8A4BDA73884B5A7F884B5A70A8
S3150800DA98864B5A78864B1A70854B00221A740022D0
S3150800DAA85A74834B00229A74814B0022DA74002236
S3150800DAB81A750420FBF77AFE034603F00103D9B268
S3150800DAC87B4A537D61F3000353750320FBF76EFE0B
S3150800DAD8034603F00103D9B2754A537D61F341033E
S3150800DAE853750020FBF762FE034603F00103D9B21B
S3150800DAF86F4A537D61F382035375FEF7BDF90346F2
S3150800DB0803F00103D9B26A4A537D61F3C303537517
S3150800DB180320FBF75BFE0346002B0CBF01230023FB
S3150800DB28D9B2634A537D61F304135375FDF7A0FC14
S3150800DB380346002B14BF01230023D9B25C4A537D40
S3150800DB4861F3451353755B4B1B7803F00103D9B290
S3150800DB58574A537D61F386135375574B1B7A03F05F
S3150800DB680103D9B2524A537D61F3C713537500208E
S3150800DB78FBF710FF03465AB24D4B5A760120FBF7BE
S3150800DB8809FF03465AB24A4B9A764B4BDB695AB297
S3150800DB98474BDA76494B5B785AB2454B1A77474B67
S3150800DBA8DB785AB2424B5A77454B9B889AB2404B18
S3150800DBB8DA83424B9A793E4B83F82020414B9B687F
S3150800DBC89AB23B4BA3F821203E4BDB689AB2384BF6
S3150800DBD8A3F823203B4B1B699AB2354BA3F825209B
S3150800DBE8334B394A27331832156854689068D16810
S3150800DBF81D605C609860D960127C1A74324BDA78BA
S3150800DC082B4B83F83820304B9B889AB2284BA3F8BD
S3150800DC1839202D4BDB889AB2254BA3F83B202A4B93
S3150800DC289B681A46224BC3F83D20274BDB68204AD7
S3150800DC38C2F84130244B9A7C1D4B83F84720224B67
S3150800DC485A7C1B4B83F846201F4B1A7C184B83F8C3
S3150800DC5845201D4BDA7C197D09020A435B7D1B04A6
S3150800DC6813439AB2124BA3F84820174B9A7D104BC8
S3150800DC7883F84A200E4B144A4B33293211685268E6
S3150800DC8819605A600A4B002283F85320084B002271
S3150800DC9883F85420002283F85520054B002283F880
S3150800DCA85620002283F8572000BFB0BDF80200208E
S3150800DCB8BC0E002029030020140A0020A403002013
S3150800DCC898030020E80900204403002080B500AF27
S3150800DCD8024800F0A5F80346184680BD840A0020C5
S3150800DCE880B582B000AF78607968034800F0C8F854
S3150800DCF800BF0837BD4680BD840A002080B483B0BB
S3150800DD0800AF78607B680F4A82FB03129210DB1714
S3150800DD18D31A5BB21B0158B27A680A4B83FB021303
S3150800DD289910D317C91A0B469B000B445B00D11AE6
S3150800DD384BB203435BB2DBB218460C37BD4680BC10
S3150800DD48704700BF6766666690B587B000AF7860AB
S3150800DD583960796800200A460346C7E9022307F1AD
S3150800DD680803184606F01EFA78617B691B68184688
S3150800DD78FFF7C4FF03461A463B681A707B695A6858
S3150800DD883B685C1C1046FFF7B9FF034623707B699E
S3150800DD989A683B689C1C1046FFF7B0FF0346237039
S3150800DDA87B69DA683B68DC1C1046FFF7A7FF034661
S3150800DDB823707B691B695A1C3B681C1D1046FFF7B4
S3150800DDC89DFF034623707B695B6903F26C73134AEC
S3150800DDD882FB03125111DA178A1A642101FB02F22F
S3150800DDE89A1A3B685C1D1046FFF788FF034623709E
S3150800DDF87B695B6903F26C73084A82FB031252114A
S3150800DE08DB17D21A3B689C1D1046FFF777FF0346B7
S3150800DE18237000BF1C37BD4690BD00BF1F85EB5158
S3150800DE2880B487B000AF786000237B8200233B82EA
S3150800DE380023FB8100237B617B681B689B697B82C7
S3150800DE487B681B68DB69FB817B681B689B693B826F
S3150800DE587A8A3B8A9A4208D03B8A1A047B681B68E6
S3150800DE68DB699BB213437B6104E07B8A1A04FB894E
S3150800DE7813437B617B6918461C37BD4680BC7047CF
S3150800DE8880B584B000AF786039600023FB73786882
S3150800DE9800F01DF80346002B02D00123FB7311E09E
S3150800DEA87B681B683A68120C9A617B681B683A6833
S3150800DEB892B2DA61786800F032F80346002B01D08E
S3150800DEC80123FB73FB7B18461037BD4680BD80B51A
S3150800DED884B000AF78600023FB6000F0FBFCF860B4
S3150800DEE809E000F0F7FC0246FB68D31AB3F57A7F17
S3150800DEF801D903230FE07B681B685B6803F02003DE
S3150800DF08002BEED07B681B685A687B681B6842F052
S3150800DF1810025A60002318461037BD4680BD80B5E2
S3150800DF2884B000AF78600023FB607B681B685A687A
S3150800DF387B681B6822F010025A6000F0CBFCF86078
S3150800DF4809E000F0C7FC0246FB68D31AB3F57A7FE6
S3150800DF5801D9032307E07B681B685B6803F0200385
S3150800DF68002BEED0002318461037BD4680BD0000AA
S3150800DF7880B485B000AF154B9B69144A43F001037A
S3150800DF889361124B9B6903F00103BB60BB680F4B97
S3150800DF98DB690E4A43F08053D3610C4BDB6903F007
S3150800DFA880537B607B680A4B5B68FB60FB6823F0E1
S3150800DFB8E063FB60FB6843F00073FB60044AFB6898
S3150800DFC8536000BF1437BD4680BC70470010024036
S3150800DFD80000014080B400AF00BFFDE780B400AF81
S3150800DFE800BFFDE780B400AF00BFFDE780B400AF0F
S3150800DFF800BFFDE780B400AF00BFFDE780B400AFFF
S3150800E00800BFBD4680BC704780B400AF00BFBD46A0
S3150800E01880BC704780B400AF00BFBD4680BC70475F
S3150800E02880B500AF00F044FC00BF80BD80B500AFE6
S3150800E038024801F035FE00BF80BD00BFA4020020DB
S3150800E04880B500AF024804F0CBFD00BF80BD00BF15
S3150800E058B40F002080B500AF024804F0C1FD00BF28
S3150800E06880BD00BFFC0F002080B500AF024804F051
S3150800E078B7FD00BF80BD00BF4410002080B500AFC3
S3150800E088024804F0ADFD00BF80BD00BF6C0F00203C
S3150800E09880B500AF024801F003FE00BF80BD00BF8F
S3150800E0A8CC02002080B500AF024801F0F9FD00BF98
S3150800E0B880BD00BFCC02002080B400AF01231846FB
S3150800E0C8BD4680BC704780B582B000AF78603960BD
S3150800E0D806F02EF9034616221A604FF0FF33184643
S3150800E0E80837BD4680BD80B582B000AF78604FF06E
S3150800E0F8FF317868FFF7E7FF00BFFDE780B586B010
S3150800E10800AFF860B9607A6000237B610AE0AFF374
S3150800E11800800146BB685A1CBA60CAB21A707B6985
S3150800E12801337B617A697B689A42F0DB7B6818461B
S3150800E1381837BD4680BD80B483B000AF78604FF00D
S3150800E148FF3318460C37BD4680BC704780B483B089
S3150800E15800AF786039603B684FF400525A60002374
S3150800E16818460C37BD4680BC704780B483B000AFEC
S3150800E1787860012318460C37BD4680BC704780B4C2
S3150800E18885B000AFF860B9607A600023184614377E
S3150800E198BD4680BC7047000080B586B000AF786081
S3150800E1A8144A154BD31A7B617B693B61134B1B6871
S3150800E1B8002B02D1114B124A1A60104B1A687B6859
S3150800E1C813443A699A4207D206F0B2F803460C2273
S3150800E1D81A604FF0FF3309E0084B1B68FB60074BD2
S3150800E1E81A687B681344054A1360FB68184618378B
S3150800E1F8BD4680BD0000012000040000200F002055
S3150800E208E011002080B400AF00BFBD4680BC70474F
S3150800E21880B58EB000AF07F1280300221A605A604D
S3150800E2289A60DA6007F1200300221A605A603B1DDB
S3150800E23800221A605A609A60DA601A615A619A610D
S3150800E248374B384A1A60364B4FF434725A60344B97
S3150800E25800229A60324B6422DA60314B00221A6136
S3150800E2682F4B00229A612E4803F0C9FC0346002B5F
S3150800E27801D0FEF7B5F84FF48053BB6207F12803BF
S3150800E2881946274803F0CEFE0346002B01D0FEF7B1
S3150800E298A7F8234803F002FD0346002B01D0FEF732
S3150800E2A89FF800233B6200237B6207F12003194687
S3150800E2B81B4804F039FA0346002B01D0FEF790F8FC
S3150800E2C860237B600023BB600023FB6000237B611F
S3150800E2D83B1D04221946124803F0E2FD0346002BAB
S3150800E2E801D0FEF77DF83B1D082219460C4803F0B5
S3150800E2F8D7FD0346002B01D0FEF772F83B1D0C220A
S3150800E3081946074803F0CCFD0346002B01D0FEF753
S3150800E31867F8034800F026F800BF3837BD4680BDC1
S3150800E328240F00200008004080B485B000AF78604C
S3150800E3387B681B68094A93420BD1094BDB69084A73
S3150800E34843F00403D361064BDB6903F00403FB605F
S3150800E358FB6800BF1437BD4680BC704700080040FC
S3150800E3680010024080B588B000AF786007F10C034A
S3150800E37800221A605A609A60DA607B681B68174A36
S3150800E388934226D1164B9B69154A43F0200393619D
S3150800E398134B9B6903F02003BB60BB684FF46043CB
S3150800E3A8FB6002233B610223BB6107F10C03194694
S3150800E3B80C4802F0FBF80C4B5B68FB61FB6943F001
S3150800E3C8E063FB61FB6943F48053FB61064AFB691A
S3150800E3D8536000BF2037BD4680BD00BF0008004017
S3150800E3E800100240001401400000014080B500AF4B
S3150800E3F8114B124A1A60104B4FF416525A600E4BBC
S3150800E40800229A600C4B0022DA600B4B00221A6134
S3150800E418094B0C225A61084B00229A61064B0022C6
S3150800E428DA61054804F0E6F90346002B01D0FDF742
S3150800E438D7FF00BF80BD00BF6C0F0020005000400A
S3150800E44880B500AF114B124A1A60104B4FF4E132EF
S3150800E4585A600E4B00229A600C4B0022DA600B4B6E
S3150800E46800221A61094B0C225A61084B00229A614C
S3150800E478064B0022DA61054804F0BCF90346002B6E
S3150800E48801D0FDF7ADFF00BF80BD00BFB40F002067
S3150800E4980038014080B500AF114B124A1A60104B7C
S3150800E4A84FF4E1325A600E4B00229A600C4B002258
S3150800E4B8DA600B4B00221A61094B0C225A61084B89
S3150800E4C800229A61064B0022DA61054804F092F99F
S3150800E4D80346002B01D0FDF783FF00BF80BD00BFB0
S3150800E4E8FC0F00200044004080B500AF114B124ACB
S3150800E4F81A60104B4FF4E1325A600E4B00229A60AC
S3150800E5080C4B0022DA600B4B00221A61094B0C22CD
S3150800E5185A61084B00229A61064B0022DA610548BF
S3150800E52804F068F90346002B01D0FDF759FF00BF30
S3150800E53880BD00BF441000200048004080B592B056
S3150800E54800AF786007F1300300221A605A609A60B3
S3150800E558DA607B681B68954A934245D1944BDB6918
S3150800E568934A43F48013D361914BDB6903F4801310
S3150800E578FB62FB6A8E4B9B698D4A43F010039361D5
S3150800E5888B4B9B6903F01003BB62BB6A884B9B697C
S3150800E598874A43F020039361854B9B6903F0200360
S3150800E5A87B627B6A4FF480533B6302237B630323B6
S3150800E5B8FB6307F1300319467E4801F0F7FF042389
S3150800E5C83B6300237B630023BB6307F130031946CB
S3150800E5D8794801F0EBFF00220021352001F051FEB1
S3150800E5E8352001F06AFEDCE07B681B68734A9342B3
S3150800E5F83AD16F4B9B696E4A43F4804393616C4BDF
S3150800E6089B6903F480433B623B6A694B9B69684A8A
S3150800E61843F004039361664B9B6903F00403FB61AB
S3150800E628FB694FF400733B6302237B630323FB6395
S3150800E63807F130031946624801F0B8FF4FF48063C2
S3150800E6483B6300237B630023BB6307F1300319464A
S3150800E6585B4801F0ABFF00220021252001F011FEDE
S3150800E668252001F02AFE9CE07B681B68554A9342E0
S3150800E67846D14F4BDB694E4A43F40033D3614C4BC2
S3150800E688DB6903F40033BB61BB69494B9B69484A9C
S3150800E69843F020039361464B9B6903F020037B6193
S3150800E6A87B6920233B6302237B630323FB6307F110
S3150800E6B830031946404801F079FF40233B6300239D
S3150800E6C87B630023BB6307F1300319463A4801F018
S3150800E6D86DFF3D4B5B683B643B6C43F0E0633B6412
S3150800E6E83B6C43F008033B64374A3B6C5360002293
S3150800E6F80021262001F0C5FD262001F0DEFD50E0A8
S3150800E7087B681B68314A93424BD1294BDB69284AF7
S3150800E71843F48023D361264BDB6903F480233B61EA
S3150800E7283B69234B9B69224A43F010039361204BAC
S3150800E7389B6903F01003FB60FB684FF480633B6337
S3150800E74802237B630323FB6307F130031946194841
S3150800E75801F02CFF4FF400633B6300237B6300231F
S3150800E768BB6307F130031946124801F01FFF164B21
S3150800E7785B687B647B6C23F030037B647B6C43F0BB
S3150800E788E0637B647B6C43F010037B640E4A7B6C06
S3150800E798536000220021272001F073FD272001F08D
S3150800E7A88CFD00BF4837BD4680BD00BF00500040FD
S3150800E7B800100240001001400014014000380140D2
S3150800E7C8000801400044004000000140004800409D
S3150800E7D8DFF834D0FFF716FD0C480D490D4A00231B
S3150800E7E802E0D458C4500433C4188C42F9D30A4AF0
S3150800E7F80A4C002301E013600432A242FBD305F059
S3150800E8089DFDFDF7FFFC7047000001200000002071
S3150800E8184C0200204C71010850020020DC1100202F
S3150800E828FEE7000080B500AF084B1B68074A43F0AF
S3150800E83810031360032001F019FD0F2000F008F8F3
S3150800E848FFF796FB0023184680BD00BF002002404C
S3150800E85880B582B000AF7860124B1A68124B1B78E5
S3150800E86819464FF47A73B3FBF1F3B2FBF3F3184680
S3150800E87801F031FD0346002B01D001230EE07B6829
S3150800E8880F2B0AD8002279684FF0FF3001F0F9FCFF
S3150800E898064A7B681360002300E0012318460837F8
S3150800E8A8BD4680BD78000020800000207C0000203E
S3150800E8B880B400AF054B1B781A46054B1B681344F2
S3150800E8C8034A136000BFBD4680BC7047800000201D
S3150800E8D88C10002080B400AF024B1B681846BD4652
S3150800E8E880BC70478C10002080B584B000AF786073
S3150800E8F8FFF7F0FFB8607B68FB60FB68B3F1FF3F82
S3150800E90805D00A4B1B781A46FB681344FB6000BF00
S3150800E918FFF7E0FF0246BB68D31AFA689A42F7D8A7
S3150800E92800BF00BF1037BD4680BD00BF800000206D
S3150800E93880B586B000AF78600023FB7500233B617D
S3150800E9480023BB600023FB607B68002B01D10123F1
S3150800E958BEE07B689B68002B7B689B6A002B09D105
S3150800E9687B680022DA627B68002283F824207868AC
S3150800E978FAF764FE786800F0F1FB0346FB757B68D6
S3150800E9889B6A03F01003002B40F09980FB7D002B4F
S3150800E99840F095807B689B6A23F4885323F002032A
S3150800E9A843F002027B689A627B685A687B68DB696F
S3150800E9B81A437B681B7B5B001343BA681343BB6027
S3150800E9C87B689B68B3F5807F03D07B689B68012BBF
S3150800E9D802D14FF4807300E000233A6913433B6180
S3150800E9E87B681B7D012B19D17B681B7B002B09D102
S3150800E9F87B689B69013B5A033B69134343F40063ED
S3150800EA083B610BE07B689B6A43F020027B689A624D
S3150800EA187B68DB6A43F001027B68DA627B681B68FD
S3150800EA285B6823F469417B681B683A690A435A603C
S3150800EA387B681B689A68284B13407A681268B96815
S3150800EA480B4393607B689B68B3F5807F03D07B682C
S3150800EA589B68012B04D17B681B69013B1B05FB607E
S3150800EA687B681B68DB6A23F470017B681B68FA6895
S3150800EA780A43DA627B681B689A68184B1340BA68B7
S3150800EA889A420BD17B680022DA627B689B6A23F07C
S3150800EA98030343F001027B689A6218E07B689B6A65
S3150800EAA823F0120343F010027B689A627B68DB6ADC
S3150800EAB843F001027B68DA620123FB7507E07B688D
S3150800EAC89B6A43F010027B689A620123FB75FB7DFB
S3150800EAD818461837BD4680BDFDF7E1FFFE0E1FFF35
S3150800EAE880B584B000AF78600023FB737B6893F821
S3150800EAF82430012B01D1022398E07B68012283F890
S3150800EB082420786800F0D0FA0346FB73FB7B002BB9
S3150800EB1840F087807B689B6A23F4407323F00103DF
S3150800EB2843F480727B689A627B681B68414A934201
S3150800EB3805D1414B5B6803F47023002B15D17B681C
S3150800EB489B6A23F480127B689A627B681B685B68F9
S3150800EB5803F48063002B26D07B689B6A23F4405312
S3150800EB6843F480527B689A621DE07B689B6A43F48B
S3150800EB7880127B689A627B681B682F4A934204D086
S3150800EB887B681B682B4A93420DD12B4B5B6803F4B1
S3150800EB988063002B07D07B689B6A23F4405343F4B1
S3150800EBA880527B689A627B689B6A03F48053002BC1
S3150800EBB806D07B68DB6A23F006027B68DA6202E025
S3150800EBC87B680022DA627B68002283F824207B6847
S3150800EBD81B686FF002021A607B681B689B6803F45F
S3150800EBE86023B3F5602F13D17B681B68114A9342DB
S3150800EBF805D1114B5B6803F47023002B08D17B6899
S3150800EC081B689A687B681B6842F4A0029A600CE045
S3150800EC187B681B689A687B681B6842F480129A604E
S3150800EC2803E07B68002283F82420FB7B184610370C
S3150800EC38BD4680BD002801400024014080B584B047
S3150800EC4800AF78600023FB737B6893F82430012BA8
S3150800EC5801D102231AE07B68012283F82420786808
S3150800EC6800F07CFA0346FB73FB7B002B09D17B6813
S3150800EC789B6A23F4885323F0010343F001027B6857
S3150800EC889A627B68002283F82420FB7B1846103793
S3150800EC98BD4680BD90B587B000AF7860396000235F
S3150800ECA87B610023FB6000233B61FFF713FE786155
S3150800ECB87B681B689B6803F48073002B0BD07B6802
S3150800ECC89B6A43F020027B689A627B68002283F875
S3150800ECD824200123D3E07B681B685B6803F48073F0
S3150800ECE8002B31D17B681B68DB6A03F47003002BA1
S3150800ECF82AD121E03B68B3F1FF3F1DD03B68002BC2
S3150800ED0807D0FFF7E7FD02467B69D31A3A689A42A5
S3150800ED1812D27B681B681B6803F00203002B0BD111
S3150800ED287B689B6A43F004027B689A627B680022C8
S3150800ED3883F824200323A2E07B681B681B6803F07A
S3150800ED480203002BD6D070E04F4B1C68022002F055
S3150800ED58FBFC0346B4FBF3F27B681B6819694B4B4B
S3150800ED680B40002B18D17B681B68D968484B0B40A9
S3150800ED78002B11D17B681B681969464B0B40002B81
S3150800ED8808D17B681B68D968434B0B40002B01D117
S3150800ED98142320E029231EE07B681B6819693D4B6C
S3150800EDA80B40002B06D17B681B68D9683A4B0B4089
S3150800EDB8002B0DD07B681B681969384B0B40002B54
S3150800EDC808D17B681B68D968344B0B40002B01D1E6
S3150800EDD8542300E0FC2302FB03F33B6121E03B6874
S3150800EDE8B3F1FF3F1AD03B68002B07D0FFF772FD37
S3150800EDF802467B69D31A3A689A420FD2FB683A697F
S3150800EE089A420BD97B689B6A43F004027B689A622C
S3150800EE187B68002283F82420032330E0FB6801334B
S3150800EE28FB60FB683A699A42D9D87B681B686FF019
S3150800EE3812021A607B689B6A43F400727B689A62BE
S3150800EE487B681B689B6803F46023B3F5602F15D1AC
S3150800EE587B681B7B002B11D17B689B6A23F4807225
S3150800EE687B689A627B689B6A03F48053002B05D1FA
S3150800EE787B689B6A43F001027B689A6200231846FE
S3150800EE881C37BD4690BD00BF78000020244992244F
S3150800EE98244992009224491292244900499224004E
S3150800EEA880B483B000AF78607B681B68DB6C184653
S3150800EEB80C37BD4680BC704780B485B000AF786013
S3150800EEC839600023FB730023BB607B6893F8243002
S3150800EED8012B01D10223DCE07B68012283F8242078
S3150800EEE83B685B68062B1CD87B681B68596B3B68B4
S3150800EEF85A6813469B001344053B1F2202FA03F37C
S3150800EF08DB4319403B6818683B685A6813469B00F8
S3150800EF181344053B00FA03F27B681B680A435A63E5
S3150800EF283CE03B685B680C2B1CD87B681B68196B34
S3150800EF383B685A6813469B001344233B1F2202FA70
S3150800EF4803F3DB4319403B6818683B685A6813465D
S3150800EF589B001344233B00FA03F27B681B680A43A9
S3150800EF681A631BE07B681B68D96A3B685A681346AC
S3150800EF789B001344413B1F2202FA03F3DB43194063
S3150800EF883B6818683B685A6813469B001344413B1C
S3150800EF9800FA03F27B681B680A43DA623B681B6857
S3150800EFA8092B1CD97B681B68D9683B681A681346FD
S3150800EFB85B0013441E3B072202FA03F3DB4319409E
S3150800EFC83B6898683B681A6813465B0013441E3BFF
S3150800EFD800FA03F27B681B680A43DA6019E07B6863
S3150800EFE81B6819693B681A6813465B0013440722AD
S3150800EFF802FA03F3DB4319403B6898683B681A68CA
S3150800F00813465B00134400FA03F27B681B680A433D
S3150800F0181A613B681B68102B03D03B681B68112BC9
S3150800F02832D17B681B681D4A934225D17B681B68C9
S3150800F0389B6803F40003002B26D17B681B689A6833
S3150800F0487B681B6842F400029A603B681B68102BB1
S3150800F0581AD1134B1B68134AA2FB03239A0C1346AF
S3150800F0689B0013445B00BB6002E0BB68013BBB60C6
S3150800F078BB68002BF9D107E07B689B6A43F020023E
S3150800F0887B689A620123FB737B68002283F8242035
S3150800F098FB7B18461437BD4680BC704700240140E0
S3150800F0A87800002083DE1B4380B584B000AF786003
S3150800F0B80023FB600023BB607B681B689B6803F022
S3150800F0C80103012B40D07B681B689A687B681B681C
S3150800F0D842F001029A601F4B1B681F4AA2FB0323D2
S3150800F0E89B0CBB6002E0BB68013BBB60BB68002B9E
S3150800F0F8F9D1FFF7EFFBF8601FE0FFF7EBFB0246D5
S3150800F108FB68D31A022B18D97B681B689B6803F01F
S3150800F1180103012B11D07B689B6A43F010027B68B8
S3150800F1289A627B68DB6A43F001027B68DA627B686D
S3150800F138002283F82420012307E07B681B689B6864
S3150800F14803F00103012BD8D1002318461037BD4612
S3150800F15880BD00BF7800002083DE1B4380B584B0DD
S3150800F16800AF78600023FB607B681B689B6803F028
S3150800F1780103012B2ED17B681B689A687B681B687C
S3150800F18822F001029A60FFF7A5FBF8601BE0FFF77B
S3150800F198A1FB0246FB68D31A022B14D97B681B68A5
S3150800F1A89B6803F00103012B0DD17B689B6A43F02A
S3150800F1B810027B689A627B68DB6A43F001027B6807
S3150800F1C8DA62012307E07B681B689B6803F0010382
S3150800F1D8012BDCD0002318461037BD4680BD000039
S3150800F1E890B587B000AF78600023FB750023FB60F5
S3150800F1F87B6893F82430012B01D1022397E07B68BA
S3150800F208012283F824207868FFF7A8FF0346FB75D0
S3150800F2187868FFF749FF0346FB75FB7D002B40F02E
S3150800F22881807B689B6A23F4885323F0020343F0A2
S3150800F23802027B689A62404B1C68022002F084FA34
S3150800F2480346B4FBF3F35B00FB6002E0FB68013B93
S3150800F258FB60FB68002BF9D17B681B689A687B689A
S3150800F2681B6842F008029A60FFF734FB38611BE016
S3150800F278FFF730FB02463B69D31A0A2B14D97B6879
S3150800F2881B689B6803F00803002B0DD07B689B6AF4
S3150800F29823F0120343F010027B689A627B68002207
S3150800F2A883F82420012342E07B681B689B6803F0E7
S3150800F2B80803002BDCD17B681B689A687B681B6887
S3150800F2C842F004029A60FFF705FB38611BE0FFF776
S3150800F2D801FB02463B69D31A0A2B14D97B681B68BB
S3150800F2E89B6803F00403002B0DD07B689B6A23F008
S3150800F2F8120343F010027B689A627B68002283F83F
S3150800F3082420012313E07B681B689B6803F0040329
S3150800F318002BDCD17B689B6A23F0030343F00102C8
S3150800F3287B689A627B68002283F82420FB7D18464E
S3150800F3381C37BD4690BD00BF7800002080B584B054
S3150800F34800AF78607B68002B01D10123EDE07B686C
S3150800F35893F82030DBB2002B02D17868FAF7E8FB7D
S3150800F3687B681B681A687B681B6842F001021A608A
S3150800F378FFF7B0FAF86012E0FFF7ACFA0246FB6846
S3150800F388D31A0A2B0BD97B685B6A43F400327B686D
S3150800F3985A627B68052283F820200123C5E07B682A
S3150800F3A81B685B6803F00103002BE5D07B681B68C4
S3150800F3B81A687B681B6822F002021A60FFF78AFA45
S3150800F3C8F86012E0FFF786FA0246FB68D31A0A2B9A
S3150800F3D80BD97B685B6A43F400327B685A627B68A0
S3150800F3E8052283F8202001239FE07B681B685B6859
S3150800F3F803F00203002BE5D17B681B7E012B08D19D
S3150800F4087B681B681A687B681B6842F080021A606A
S3150800F41807E07B681B681A687B681B6822F080020D
S3150800F4281A607B685B7E012B08D17B681B681A68A3
S3150800F4387B681B6842F040021A6007E07B681B6815
S3150800F4481A687B681B6822F040021A607B689B7EF4
S3150800F458012B08D17B681B681A687B681B6842F011
S3150800F46820021A6007E07B681B681A687B681B68B5
S3150800F47822F020021A607B68DB7E012B08D17B68A4
S3150800F4881B681A687B681B6822F010021A6007E076
S3150800F4987B681B681A687B681B6842F010021A604A
S3150800F4A87B681B7F012B08D17B681B681A687B68F9
S3150800F4B81B6842F008021A6007E07B681B681A682E
S3150800F4C87B681B6822F008021A607B685B7F012B41
S3150800F4D808D17B681B681A687B681B6842F00402B7
S3150800F4E81A6007E07B681B681A687B681B6822F045
S3150800F4F804021A607B689A687B68DB681A437B682B
S3150800F5081B691A437B685B6942EA03017B685B6887
S3150800F5185A1E7B681B680A43DA617B6800225A62AE
S3150800F5287B68012283F82020002318461037BD4639
S3150800F53880BD000080B487B000AF786039607B680A
S3150800F5481B687B617B6893F82030FB74FB7C012B76
S3150800F55803D0FB7C022B40F0BE80654B7B617B6940
S3150800F568D3F8003243F001027B69C3F800227B69AD
S3150800F578D3F8003223F47C527B69C3F800227B69EE
S3150800F588D3F800223B685B6A1B021A437B69C3F8F7
S3150800F59800223B685B6903F01F03012202FA03F3A2
S3150800F5A8FB607B69D3F81C22FB68DB431A407B693E
S3150800F5B8C3F81C223B68DB69002B23D17B69D3F887
S3150800F5C80C22FB68DB431A407B69C3F80C223B68AC
S3150800F5D8DB6819043B685B689BB23A685269194349
S3150800F5E87B69483243F832103B689B6819043B68C4
S3150800F5F81B689AB23B685B690A4379694833DB003A
S3150800F6080B445A603B68DB69012B22D17B69D3F826
S3150800F6180C22FB681A437B69C3F80C223B681B68F3
S3150800F62819043B685B689BB23A68526919437B6957
S3150800F638483243F832103B689B6819043B68DB6814
S3150800F6489AB23B685B690A4379694833DB000B441D
S3150800F6585A603B689B69002B09D17B69D3F8042259
S3150800F668FB68DB431A407B69C3F8042207E07B6919
S3150800F678D3F80422FB681A437B69C3F804223B685B
S3150800F6881B69002B09D17B69D3F81422FB68DB4375
S3150800F6981A407B69C3F8142207E07B69D3F8142259
S3150800F6A8FB681A437B69C3F814223B681B6A012B5B
S3150800F6B807D17B69D3F81C22FB681A437B69C3F810
S3150800F6C81C227B69D3F8003223F001027B69C3F850
S3150800F6D80022002306E07B685B6A43F480227B6885
S3150800F6E85A62012318461C37BD4680BC704700BFBE
S3150800F6F80064004080B584B000AF78607B6893F8F2
S3150800F7082030DBB2012B2ED17B68022283F8202019
S3150800F7187B681B681A687B681B6822F001021A60F6
S3150800F728FFF7D8F8F86012E0FFF7D4F80246FB6846
S3150800F738D31A0A2B0BD97B685B6A43F400327B68B9
S3150800F7485A627B68052283F82020012312E07B6829
S3150800F7581B685B6803F00103002BE5D17B68002270
S3150800F7685A62002306E07B685B6A43F400227B68DA
S3150800F7785A62012318461037BD4680BD80B584B045
S3150800F78800AF78607B6893F82030DBB2022B33D160
S3150800F7987B681B681A687B681B6842F001021A6056
S3150800F7A8FFF798F8F86012E0FFF794F80246FB6846
S3150800F7B8D31A0A2B0BD97B685B6A43F400327B6839
S3150800F7C85A627B68052283F8202001231BE07B68A0
S3150800F7D81B685B6803F00103002BE5D07B681B6890
S3150800F7E81A687B681B6822F002021A607B68012285
S3150800F7F883F82020002306E07B685B6A43F48012BE
S3150800F8087B685A62012318461037BD4680BD80B406
S3150800F81889B000AFF860B9607A603B60FB6893F816
S3150800F8282030FB77FB681B689B68BB61FB7F012B55
S3150800F83803D0FB7F022B40F0AD80BB6903F08063E1
S3150800F848002B0AD1BB6903F00063002B05D1BB69FD
S3150800F85803F08053002B00F09580BB691B0E03F05C
S3150800F86803037B6101227B699A403B681A60BB687F
S3150800F8789B68002B0DD1BB681B685A05BB68DB68FB
S3150800F888F96809681A437B6918331B010B441A601F
S3150800F8980FE0BB685B68DA00BB689B681A43BB68FD
S3150800F8A8DB68F96809681A437B6918331B010B4436
S3150800F8B81A60FB681968BB681A697B6918331B01E3
S3150800F8C80B4404331A60BB681B7D012B11D1FB68F6
S3150800F8D81A687B6918331B01134404331B68FA68D2
S3150800F8E8116843F480727B6918331B010B4404338F
S3150800F8F81A607B6807331B781A067B6806331B78F9
S3150800F9081B041A437B6805331B781B0213437A6862
S3150800F918043212781046FA68116843EA00027B69CD
S3150800F9281B010B4403F5C6731A607B6803331B78FF
S3150800F9381A067B6802331B781B041A437B68013353
S3150800F9481B781B0213437A6812781046FA681168FE
S3150800F95843EA00027B691B010B4403F5C4731A606A
S3150800F968FB681A687B6918331B0113441B68FA6815
S3150800F978116843F001027B6918331B010B441A60AE
S3150800F98800230EE0FB685B6A43F40012FB685A62C0
S3150800F998012306E0FB685B6A43F48022FB685A6227
S3150800F9A8012318462437BD4680BC704780B485B005
S3150800F9B800AF78600023FB607B6893F82030FB7201
S3150800F9C8FB7A012B02D0FB7A022B1DD17B681B68B8
S3150800F9D89B6803F08063002B02D0FB680133FB6049
S3150800F9E87B681B689B6803F00063002B02D0FB68E2
S3150800F9F80133FB607B681B689B6803F08053002B08
S3150800FA0802D0FB680133FB60FB6818461437BD460D
S3150800FA1880BC704780B487B000AFF860B9607A6078
S3150800FA283B60FB6893F82030FB75FB7D012B03D000
S3150800FA38FB7D022B40F00381BB68002B0ED1FB68C7
S3150800FA481B68DB6803F00303002B16D1FB685B6AA7
S3150800FA5843F40012FB685A620123F7E0FB681B6847
S3150800FA681B6903F00303002B07D1FB685B6A43F4A1
S3150800FA780012FB685A620123E8E0FB681A68BB684B
S3150800FA881B331B0113441B6803F004027B689A6046
S3150800FA987B689B68002B0CD1FB681A68BB681B330C
S3150800FAA81B0113441B685B0DC3F30A027B681A60C3
S3150800FAB80BE0FB681A68BB681B331B0113441B68F9
S3150800FAC8DB0823F060427B685A60FB681A68BB68E3
S3150800FAD81B331B0113441B6803F002027B68DA60B8
S3150800FAE8FB681A68BB681B331B01134404331B687D
S3150800FAF803F00803002B03D07B6808221A610BE081
S3150800FB08FB681A68BB681B331B01134404331B685C
S3150800FB1803F00F027B681A61FB681A68BB681B3317
S3150800FB281B01134404331B681B0ADAB27B689A6103
S3150800FB38FB681A68BB681B331B01134404331B682C
S3150800FB481B0C9AB27B685A61FB681A68BB681B016A
S3150800FB58134403F5DC731B68DAB23B681A70FB6852
S3150800FB681A68BB681B01134403F5DC731B681A0A79
S3150800FB783B680133D2B21A70FB681A68BB681B0166
S3150800FB88134403F5DC731B681A0C3B680233D2B2BC
S3150800FB981A70FB681A68BB681B01134403F5DC7303
S3150800FBA81B681A0E3B680333D2B21A70FB681A68C8
S3150800FBB8BB681B01134403F5DE731A683B680433F4
S3150800FBC8D2B21A70FB681A68BB681B01134403F59E
S3150800FBD8DE731B681A0A3B680533D2B21A70FB68CB
S3150800FBE81A68BB681B01134403F5DE731B681A0CF5
S3150800FBF83B680633D2B21A70FB681A68BB681B01E1
S3150800FC08134403F5DE731B681A0E3B680733D2B232
S3150800FC181A70BB68002B08D1FB681B68DA68FB6892
S3150800FC281B6842F02002DA6007E0FB681B681A695D
S3150800FC38FB681B6842F020021A61002306E0FB688D
S3150800FC485B6A43F48022FB685A62012318461C370C
S3150800FC58BD4680BC704780B485B000AF786039600F
S3150800FC687B6893F82030FB73FB7B012B02D0FB7B68
S3150800FC78022B09D17B681B6859697B681B683A6837
S3150800FC880A435A61002306E07B685B6A43F48022CC
S3150800FC987B685A62012318461437BD4680BC7047EC
S3150800FCA880B58AB000AF786000237B627B681B68E2
S3150800FCB85B693B627B681B685B68FB617B681B68E2
S3150800FCC89B68BB617B681B68DB687B617B681B6814
S3150800FCD81B693B617B681B689B69FB603B6A03F091
S3150800FCE80103002B7CD0BB6903F00103002B23D04A
S3150800FCF87B681B6801229A60BB6903F00203002B24
S3150800FD0803D0786800F083F916E0BB6903F00403AA
S3150800FD18002B04D07B6A43F400637B620CE0BB6962
S3150800FD2803F00803002B04D07B6A43F480537B62F4
S3150800FD3802E0786800F086F9BB6903F48073002B43
S3150800FD4824D07B681B684FF480729A60BB6903F4F9
S3150800FD580073002B03D0786800F062F916E0BB69D7
S3150800FD6803F48063002B04D07B6A43F400537B6258
S3150800FD780CE0BB6903F40063002B04D07B6A43F4E8
S3150800FD8880437B6202E0786800F065F9BB6903F492
S3150800FD988033002B24D07B681B684FF480329A6026
S3150800FDA8BB6903F40033002B03D0786800F041F9E7
S3150800FDB816E0BB6903F48023002B04D07B6A43F45E
S3150800FDC800437B620CE0BB6903F40023002B04D0D4
S3150800FDD87B6A43F480337B6202E0786800F044F972
S3150800FDE83B6A03F00803002B0CD07B6903F0100369
S3150800FDF8002B07D07B6A43F400737B627B681B6819
S3150800FE081022DA603B6A03F00403002B0BD07B69E7
S3150800FE1803F00803002B06D07B681B680822DA6003
S3150800FE28786800F02AF93B6A03F00203002B09D028
S3150800FE387B681B68DB6803F00303002B02D078682D
S3150800FE48FBF7A6FD3B6A03F04003002B0CD03B6981
S3150800FE5803F01003002B07D07B6A43F480637B62A8
S3150800FE687B681B6810221A613B6A03F02003002B83
S3150800FE780BD03B6903F00803002B06D07B681B6888
S3150800FE8808221A61786800F001F93B6A03F0100342
S3150800FE98002B09D07B681B681B6903F00303002B3A
S3150800FEA802D07868FCF72CFB3B6A03F40033002B76
S3150800FEB80BD0FB6903F01003002B06D07B681B6880
S3150800FEC810225A60786800F0EAF83B6A03F480332F
S3150800FED8002B0BD0FB6903F00803002B06D07B68C0
S3150800FEE81B6808225A60786800F0E2F83B6A03F44F
S3150800FEF80043002B7BD0FB6903F00403002B72D068
S3150800FF083B6A03F48073002B08D0FB6803F00103EF
S3150800FF18002B03D07B6A43F001037B623B6A03F438
S3150800FF280073002B08D0FB6803F00203002B03D0EC
S3150800FF387B6A43F002037B623B6A03F48063002B07
S3150800FF4808D0FB6803F00403002B03D07B6A43F050
S3150800FF5804037B623B6A03F40063002B43D0FB6807
S3150800FF6803F07003002B3ED0FB6803F07003602B88
S3150800FF782BD0602B2ED8502B22D0502B2AD8402B8A
S3150800FF8819D0402B26D8302B10D0302B22D8102B3E
S3150800FF9802D0202B05D01DE07B6A43F008037B625C
S3150800FFA819E07B6A43F010037B6214E07B6A43F02E
S3150800FFB820037B620FE07B6A43F040037B620AE01A
S3150800FFC87B6A43F080037B6205E07B6A43F48073AF
S3150800FFD87B6200E000BF7B681B689A697B681B68C0
S3150800FFE822F070029A617B681B6804225A607B6A51
S3150800FFF8002B08D07B685A6A7B6A1A437B685A6260
S31508010008786800F05EF800BF2837BD4680BD80B421
S3150801001883B000AF786000BF0C37BD4680BC704717
S3150801002880B483B000AF786000BF0C37BD4680BC8A
S31508010038704780B483B000AF786000BF0C37BD46FF
S3150801004880BC704780B483B000AF786000BF0C37B6
S31508010058BD4680BC704780B483B000AF786000BFE6
S315080100680C37BD4680BC704780B483B000AF786052
S3150801007800BF0C37BD4680BC704780B483B000AF5B
S31508010088786000BF0C37BD4680BC704780B483B022
S3150801009800AF786000BF0C37BD4680BC704780B496
S315080100A883B000AF786000BF0C37BD4680BC704787
S315080100B880B483B000AF786000BF0C37BD4680BCFA
S315080100C8704780B483B000AF786000BF0C37BD466F
S315080100D880BC704780B485B000AF78607B6803F050
S315080100E80703FB600C4BDB68BB60BA684FF6FF0376
S315080100F81340BB60FB681A02BB68134343F0BF632E
S3150801010843F40033BB60044ABB68D36000BF1437A5
S31508010118BD4680BC704700BF00ED00E080B400AF63
S31508010128044BDB681B0A03F007031846BD4680BC67
S31508010138704700BF00ED00E080B483B000AF034606
S31508010148FB7197F90730002B0BDBFB7903F01F02CC
S31508010158064997F907305B09012000FA02F241F8C6
S31508010168232000BF0C37BD4680BC704700E100E07C
S3150801017880B483B000AF03463960FB7197F907303D
S31508010188002B0ADB3B68DAB20C4997F907301201EA
S31508010198D2B20B4483F800230AE03B68DAB208496D
S315080101A8FB7903F00F03043B1201D2B20B441A760A
S315080101B800BF0C37BD4680BC704700BF00E100E0B0
S315080101C800ED00E080B489B000AFF860B9607A60E4
S315080101D8FB6803F00703FB61FB69C3F10703042BFB
S315080101E828BF0423BB61FB690433062B02D9FB69C3
S315080101F8033B00E000237B614FF0FF32BB6902FA3B
S3150801020803F3DA43BB681A407B699A404FF0FF311A
S315080102187B6901FA03F3D9437B680B4013431846F4
S315080102282437BD4680BC704780B582B000AF786078
S315080102387B68013BB3F1807F01D301230FE00A4AAA
S315080102487B68013B53600F214FF0FF30FFF790FFA2
S31508010258054B00229A60044B07221A6000231846A8
S315080102680837BD4680BD00BF10E000E080B582B002
S3150801027800AF78607868FFF72DFF00BF0837BD46DD
S3150801028880BD80B586B000AF0346B9607A60FB7356
S3150801029800237B61FFF742FF78617A68B968786954
S315080102A8FFF790FF024697F90F3011461846FFF7F0
S315080102B85FFF00BF1837BD4680BD80B582B000AF65
S315080102C80346FB7197F907301846FFF735FF00BF54
S315080102D80837BD4680BD80B582B000AF78607868BA
S315080102E8FFF7A2FF034618460837BD4680BD80B505
S315080102F882B000AF78607B68002B01D101230EE03C
S315080103087B685B79DBB2002B05D17B6800221A7101
S315080103187868FBF71FF87B6801225A71002318468B
S315080103280837BD4680BD80B485B000AF7860002324
S31508010338FB737B6893F82130DBB2022B08D07B6804
S3150801034804229A637B68002283F82020012320E08F
S315080103587B681B681A687B681B6822F00E021A609C
S315080103687B681B681A687B681B6822F001021A6099
S315080103787B681A6C7B68DB6B012101FA02F25A6009
S315080103887B68012283F821207B68002283F82020D4
S31508010398FB7B18461437BD4680BC704780B584B0C8
S315080103A800AF78600023FB737B6893F82130DBB2D2
S315080103B8022B05D07B6804229A630123FB73D6E0D6
S315080103C87B681B681A687B681B6822F00E021A602C
S315080103D87B681B681A687B681B6822F001021A6029
S315080103E87B681B681A46644B9A4258D97B681B680E
S315080103F8624A93424FD07B681B68614A934248D048
S315080104087B681B685F4A934240D07B681B685E4AD3
S31508010418934238D07B681B685C4A934230D07B6824
S315080104281B685B4A934228D07B681B68524A9342E9
S3150801043820D07B681B68574A934219D07B681B688A
S31508010448554A934212D07B681B68544A93420AD08C
S315080104587B681B68524A934202D14FF480531BE0CA
S315080104684FF4803318E04FF4807315E0102313E036
S31508010478012311E04FF080730EE04FF480130BE06F
S315080104884FF4803308E04FF4805305E04FF4807346
S3150801049802E0102300E00123424A536057E07B68D3
S315080104A81B68364A93424FD07B681B68344A934285
S315080104B848D07B681B68334A934240D07B681B68DF
S315080104C8314A934238D07B681B68304A934230D008
S315080104D87B681B682E4A934228D07B681B68264A84
S315080104E8934220D07B681B682A4A934219D07B68B5
S315080104F81B68294A934212D07B681B68274A93428C
S315080105080AD07B681B68264A934202D14FF4805366
S315080105181BE04FF4803318E04FF4807315E010237D
S3150801052813E0012311E04FF080730EE04FF48013B6
S315080105380BE04FF4803308E04FF4805305E04FF49D
S31508010548807302E0102300E00123174A53607B6891
S31508010558012283F821207B68002283F820207B6802
S315080105685B6B002B03D07B685B6B78689847FB7BD2
S3150801057818461037BD4680BD800002400800024073
S315080105881C00024030000240440002405800024064
S315080105986C000240080402401C0402403004024070
S315080105A844040240000402400000024080B48BB0B3
S315080105B800AF7860396000237B6200233B6269E1FA
S315080105C801227B6A02FA03F3FB613B681B68FA6935
S315080105D81340BB61BA69FB699A4240F058813B6886
S315080105E85B689A4A93425ED0984A934275D8984A64
S315080105F8934258D0964A93426FD8964A934252D014
S31508010608944A934269D8944A93424CD0924A93425F
S3150801061863D8924A934246D0904A93425DD8122BA0
S315080106282AD8122B59D801A252F823F0AF06010885
S31508010638890601089B060108DD060108E306010883
S31508010648E3060108E3060108E3060108E3060108CB
S31508010658E3060108E3060108E3060108E3060108BB
S31508010668E3060108E3060108E3060108E3060108AB
S3150801067891060108A5060108794A934213D02CE088
S315080106883B68DB683B6229E03B68DB6804333B620D
S3150801069824E03B68DB6808333B621FE03B68DB689C
S315080106A80C333B621AE03B689B68002B02D1042392
S315080106B83B6213E03B689B68012B05D108233B6223
S315080106C87B68FA691A6109E008233B627B68FA695B
S315080106D85A6103E000233B6200E000BFBB69FF2BB8
S315080106E801D87B6801E07B6804337B61BB69FF2B12
S315080106F802D87B6A9B0002E07B6A083B9B003B6148
S315080107087B691A680F213B6901FA03F3DB431A402F
S31508010718396A3B6901FA03F31A437B691A603B682C
S315080107285B6803F08053002B00F0B1804D4B9B6941
S315080107384C4A43F0010393614A4B9B6903F0010351
S31508010748BB60BB68484A7B6A9B08023352F8233068
S31508010758FB607B6A03F003039B000F2202FA03F38B
S31508010768DB43FA681340FB607B68404A934213D01F
S315080107787B683F4A93420DD07B683E4A934207D02D
S315080107887B683D4A934201D1032306E0042304E02A
S31508010798022302E0012300E000237A6A02F0030239
S315080107A892009340FA681343FB602F497B6A9B08BA
S315080107B80233FA6841F823203B685B6803F480131F
S315080107C8002B06D02D4B9A682C49BB6913438B60BD
S315080107D806E02A4B9A68BB69DB43284913408B60B4
S315080107E83B685B6803F40013002B06D0234BDA68D1
S315080107F82249BB691343CB6006E0204BDA68BB691B
S31508010808DB431E491340CB603B685B6803F400333E
S31508010818002B06D0194B5A681849BB6913434B6014
S3150801082806E0164B5A68BB69DB43144913404B600B
S315080108383B685B6803F48033002B21D00F4B1A6899
S315080108480E49BB6913430B6021E000BF0000321053
S3150801085800003110000022100000211000001210BB
S315080108680000111000100240000001400008014074
S31508010878000C014000100140001401400004014029
S315080108880B4B1A68BB69DB43094913400B607B6A42
S3150801089801337B623B681A687B6A22FA03F3002BE9
S315080108A87FF48EAE00BF00BF2C37BD4680BC7047AB
S315080108B80004014080B485B000AF78600B467B80A0
S315080108C87B689A687B881340002B02D00123FB7347
S315080108D801E00023FB73FB7B18461437BD4680BC31
S315080108E8704780B483B000AF78600B467B801346A7
S315080108F87B707B78002B03D07A887B681A6103E0C2
S315080109087B881A047B681A6100BF0C37BD4680BC10
S315080109187047000080B400AF034B01221A6000BF7C
S31508010928BD4680BC704700BF20000E4280B582B024
S3150801093800AFFDF7CFFF7860604B1B685F4A43F04D
S315080109480103136008E0FDF7C5FF02467B68D31A61
S31508010958022B01D90323ACE0584B1B6803F00203A9
S31508010968002BF0D0554B1B6823F0F803534A43F084
S3150801097880031360FDF7AEFF7860504B00225A607A
S315080109880AE0FDF7A7FF02467B68D31A41F28832C7
S31508010998934201D903238CE0484B5B6803F00C03A7
S315080109A8002BEED1464B474A1A60474B1B68184637
S315080109B8FDF74EFF0346002B01D0012379E0FDF729
S315080109C889FF78603D4B1B683C4A23F080731360A6
S315080109D808E0FDF77FFF02467B68D31A022B01D987
S315080109E8032366E0354B1B6803F00073002BF0D12F
S315080109F8324B00225A60FDF76DFF78602F4B1B6852
S31508010A082E4A23F41023136008E0FDF763FF024614
S31508010A187B68D31A642B01D903234AE0274B1B6841
S31508010A2803F40033002BF0D1244B1B68234A23F423
S31508010A3880231360FDF74EFF7860204B1B681F4A19
S31508010A4823F08063136008E0FDF744FF02467B68DC
S31508010A58D31A642B01D903232BE0184B1B6803F01F
S31508010A680063002BF0D1FDF735FF7860134B1B683F
S31508010A78124A23F08053136008E0FDF72BFF02465C
S31508010A887B68D31A642B01D9032312E00B4B1B6825
S31508010A9803F00053002BF0D1084B0022DA62074B0A
S31508010AA85B6A064A43F080735362044B00229A60D4
S31508010AB8002318460837BD4680BD00BF001002400E
S31508010AC87800002000127A007C00002080B586B0E4
S31508010AD800AF78607B68002B01D1012304E37B68AA
S31508010AE81B6803F00103002B00F08780924B5B68B3
S31508010AF803F00C03042B0CD08F4B5B6803F00C0333
S31508010B08082B12D18C4B5B6803F48033B3F5803F0D
S31508010B180BD1894B1B6803F40033002B6CD07B6817
S31508010B289B68002B68D10123DEE27B689B68B3F5D5
S31508010B38803F06D1804B1B687F4A43F48033136094
S31508010B482EE07B689B68002B0CD17B4B1B687A4A85
S31508010B5823F480331360784B1B68774A23F4802380
S31508010B6813601DE07B689B68B3F5A02F0CD1724B07
S31508010B781B68714A43F4802313606F4B1B686E4ADE
S31508010B8843F4803313600BE06B4B1B686A4A23F402
S31508010B9880331360684B1B68674A23F48023136004
S31508010BA87B689B68002B13D0FDF794FE386108E033
S31508010BB8FDF790FE02463B69D31A642B01D9032334
S31508010BC892E25D4B1B6803F40033002BF0D014E066
S31508010BD8FDF780FE386108E0FDF77CFE02463B69B1
S31508010BE8D31A642B01D903237EE2534B1B6803F4FA
S31508010BF80033002BF0D100E000BF7B681B6803F0C7
S31508010C080203002B63D04C4B5B6803F00C03002BE3
S31508010C180BD0494B5B6803F00C03082B1CD1464BD8
S31508010C285B6803F48033002B16D1434B1B6803F02A
S31508010C380203002B05D07B685B69012B01D00123D0
S31508010C4852E23D4B1B6823F0F8027B689B69DB007F
S31508010C58394913430B603AE07B685B69002B20D05E
S31508010C68364B01221A60FDF735FE386108E0FDF7B3
S31508010C7831FE02463B69D31A022B01D9032333E213
S31508010C882D4B1B6803F00203002BF0D02A4B1B6877
S31508010C9823F0F8027B689B69DB00274913430B603D
S31508010CA815E0264B00221A60FDF714FE386108E0A4
S31508010CB8FDF710FE02463B69D31A022B01D9032315
S31508010CC812E21D4B1B6803F00203002BF0D17B6867
S31508010CD81B6803F00803002B3AD07B68DB69002BF5
S31508010CE819D0174B01221A60FDF7F4FD386108E09F
S31508010CF8FDF7F0FD02463B69D31A022B01D90323F6
S31508010D08F2E10D4B5B6A03F00203002BF0D00120D8
S31508010D1800F0CAFB1CE00A4B00221A60FDF7DAFD4F
S31508010D2838610FE0FDF7D6FD02463B69D31A022B57
S31508010D3808D90323D8E100BF001002400000424247
S31508010D48800442429B4B5B6A03F00203002BE9D1FC
S31508010D587B681B6803F00403002B00F0A6800023B8
S31508010D68FB75944BDB6903F08053002B0DD1914B2E
S31508010D78DB69904A43F08053D3618E4BDB6903F0F4
S31508010D888053BB60BB680123FB758B4B1B6803F457
S31508010D988073002B18D1884B1B68874A43F48073E4
S31508010DA81360FDF797FD386108E0FDF793FD0246E4
S31508010DB83B69D31A642B01D9032395E17E4B1B683A
S31508010DC803F48073002BF0D07B681B69012B06D1CD
S31508010DD8784B1B6A774A43F0010313622DE07B6857
S31508010DE81B69002B0CD1734B1B6A724A23F001034A
S31508010DF81362704B1B6A6F4A23F0040313621CE0E3
S31508010E087B681B69052B0CD16A4B1B6A694A43F037
S31508010E1804031362674B1B6A664A43F001031362AC
S31508010E280BE0644B1B6A634A23F001031362614BA7
S31508010E381B6A604A23F0040313627B681B69002B4B
S31508010E4815D0FDF747FD38610AE0FDF743FD02466F
S31508010E583B69D31A41F28832934201D9032343E104
S31508010E68544B1B6A03F00203002BEED014E0FDF77E
S31508010E7831FD38610AE0FDF72DFD02463B69D31AB3
S31508010E8841F28832934201D903232DE1494B1B6A62
S31508010E9803F00203002BEED1FB7D012B05D1454B4F
S31508010EA8DB69444A23F08053D3617B68DB6A002BEC
S31508010EB800F08C803F4B5B6803F48033B3F5803FC1
S31508010EC80ED13C4B5B6803F00C03082B08D1394B50
S31508010ED8DB6A03F48033B3F5803F01D1012303E1CB
S31508010EE87B68DB6A022B4ED1324B1B6803F08053B1
S31508010EF8002B09D02F4BDB6A03F0F0027B685B6B8A
S31508010F089A4201D00123EFE02C4B00221A60FDF723
S31508010F18E1FC386108E0FDF7DDFC02463B69D31AB6
S31508010F28642B01D90323DFE0224B1B6803F0006316
S31508010F38002BF0D11F4BDB6A23F0F0027B685B6B51
S31508010F481C491343CB621B4BDB6A23F470627B682B
S31508010F581B6B18491343CB62184B01221A60FDF71C
S31508010F68B9FC386108E0FDF7B5FC02463B69D31AB6
S31508010F78642B01D90323B7E00E4B1B6803F0006302
S31508010F88002BF0D022E00B4BDB6A0A4A23F48033A4
S31508010F98D3620A4B00221A60FDF79CFC38610FE000
S31508010FA8FDF798FC02463B69D31A642B08D9032333
S31508010FB89AE000BF001002400070004068004242F3
S31508010FC84B4B1B6803F00063002BE9D17B681B6A4E
S31508010FD8002B00F08880464B5B6803F00C03082B4E
S31508010FE868D07B681B6A022B4DD1424B00221A60D6
S31508010FF8FDF770FC386108E0FDF76CFC02463B69B1
S31508011008D31A022B01D903236EE0394B1B6803F067
S315080110180073002BF0D17B685B6AB3F5803F0FD16B
S31508011028334BDA6A7B685B6831491343CB62304BC9
S31508011038DB6A23F00F027B68DB682D491343CB6211
S315080110482B4B5B6823F474127B68596A7B689B6A25
S315080110580B43274913434B60264B01221A60FDF7B8
S3150801106839FC386108E0FDF735FC02463B69D31AB5
S31508011078022B01D9032337E01D4B1B6803F00073C4
S31508011088002BF0D02FE01B4B00221A60FDF722FC3B
S31508011098386108E0FDF71EFC02463B69D31A022BA4
S315080110A801D9032320E0124B1B6803F00073002BB8
S315080110B8F0D118E07B681B6A012B01D1012313E0E3
S315080110C80B4B5B68FB60FB6803F480327B685B6AE1
S315080110D89A4206D1FB6803F470127B689B6A9A42A6
S315080110E801D0012300E0002318461837BD4680BD04
S315080110F8001002406000424280B584B000AF7860B3
S3150801110839607B68002B01D10123D0E06A4B1B6843
S3150801111803F007033A689A4210D9674B1B6823F00C
S31508011128070265493B6813430B60634B1B6803F069
S3150801113807033A689A4201D00123B8E07B681B681D
S3150801114803F00203002B20D07B681B6803F0040315
S31508011158002B05D0594B5B68584A43F4E063536042
S315080111687B681B6803F00803002B05D0534B5B68A3
S31508011178524A43F460535360504B5B6823F0F002BC
S315080111887B689B684D4913434B607B681B6803F072
S315080111980103002B40D07B685B68012B07D1474BBD
S315080111A81B6803F40033002B15D101237FE07B6804
S315080111B85B68022B07D1414B1B6803F00073002BB0
S315080111C809D1012373E03D4B1B6803F00203002B89
S315080111D801D101236BE0394B5B6823F003027B6875
S315080111E85B68364913434B60FDF774FBF8600AE000
S315080111F8FDF770FB0246FB68D31A41F2883293421F
S3150801120801D9032353E02D4B5B6803F00C027B6875
S315080112185B689B009A42EBD1274B1B6803F00703CF
S315080112283A689A4210D2244B1B6823F007022249CE
S315080112383B6813430B60204B1B6803F007033A68A6
S315080112489A4201D0012332E07B681B6803F0040344
S31508011258002B08D0194B5B6823F4E0627B68DB68CE
S31508011268164913434B607B681B6803F00803002B78
S3150801127809D0124B5B6823F460527B681B69DB0053
S315080112880E4913434B6000F021F802460B4B5B6885
S315080112981B0903F00F030A49CB5C22FA03F3094A2F
S315080112A81360094B1B681846FDF7D2FA002318463E
S315080112B81037BD4680BD00BF00200240001002401D
S315080112C8186D0108780000207C0000202DE9B04F30
S315080112D88EB000AF0023FB620023BB6200237B6349
S315080112E800237B6200233B6300233B620023FB61E7
S315080112F84E4B5B68FB62FB6A03F00C03042B02D0B6
S31508011308082B03D089E04A4B3B6389E0FB6A9B0CAF
S3150801131803F00F02474B9B5C7B62FB6A03F480333D
S31508011328002B72D0414BDB6A03F00F02424B9B5CE0
S31508011338BB623E4BDB6A03F48033002B53D03B4B2D
S31508011348DB6A1B0903F00F0301333B62374BDB6A80
S315080113581B0A03F00F030233FB61FB6900229A4655
S3150801136893467B6A00223B617A613B6903FB0BF270
S315080113787B690AFB03F313443A69AAFB02010B4486
S3150801138819462B4B03FB01F2002300FB03F3134415
S31508011398274AA0FB02452B441D463B6A0022BB602F
S315080113A8FA60BB6A00223B607A60D7E902010B46FC
S315080113B8D7E900AB524602FB03F25B4684460CFBAF
S315080113C803F3134402465146A2FB01894B44994645
S315080113D842464B4620462946F7F758FF02460B462A
S315080113E813467B6307E07B6A114A03FB02F2BB6A71
S315080113F8B2FBF3F37B630F4B5B7B1A467B6A93421B
S3150801140808D17B6B5B087B6304E07B6A0B4A02FBAA
S3150801141803F37B637B6B3B6302E0094B3B6300BFCA
S315080114283B6B18463837BD46BDE8B08F00100240F9
S3150801143840787D01306D0108406D010800093D00BD
S3150801144800127A0080B400AF024B1B681846BD46E5
S3150801145880BC70477800002080B500AFFFF7F2FF1F
S315080114680246054B5B681B0A03F007030349CB5C75
S3150801147822FA03F3184680BD00100240286D0108B8
S3150801148880B500AFFFF7DEFF0246054B5B68DB0A4E
S3150801149803F007030349CB5C22FA03F3184680BD18
S315080114A800100240286D010880B485B000AF786045
S315080114B80A4B1B680A4AA2FB03235B0A7A6802FBE2
S315080114C803F3FB6000BFFB685A1EFA60002BF9D1CB
S315080114D800BF00BF1437BD4680BC7047780000209E
S315080114E8D34D621080B588B000AF786000237B6160
S315080114F800233B610023FB617B681B6803F001033A
S31508011508002B7DD00023FB768B4BDB6903F08053D8
S31508011518002B0DD1884BDB69874A43F08053D36189
S31508011528854BDB6903F08053FB60FB680123FB7677
S31508011538824B1B6803F48073002B18D17F4B1B68F9
S315080115487E4A43F480731360FDF7C4F9786108E0AD
S31508011558FDF7C0F902467B69D31A642B01D903231F
S31508011568E5E0764B1B6803F48073002BF0D0724BC9
S315080115781B6A03F440733B613B69002B2ED07B68D9
S315080115885B6803F440733A699A4227D06A4B1B6A27
S3150801159823F440733B616A4B01221A60684B0022A7
S315080115A81A60654A3B6913623B6903F00103002B1C
S315080115B814D0FDF78FF978610AE0FDF78BF9024631
S315080115C87B69D31A41F28832934201D90323AEE0E3
S315080115D8594B1B6A03F00203002BEED0564B1B6AC4
S315080115E823F440727B685B68534913430B62FB7E9D
S315080115F8012B05D1504BDB694F4A23F08053D36140
S315080116087B681B6803F00203002B08D04A4B5B680A
S3150801161823F440427B689B68474913434B607B68C0
S315080116281B6803F00403002B08D0434BDB6A23F439
S3150801163800327B68DB6840491343CB627B681B68C9
S3150801164803F00803002B08D03B4BDB6A23F48022FE
S315080116587B681B6938491343CB62374BDB6A03F44A
S315080116680033002B05D1344BDB6A03F48023002BA6
S3150801167801D00123FB61FB69012B48D12E4B1B685D
S3150801168803F08053002B38D12B4B1B6803F080637A
S31508011698002B09D0284BDB6A03F0F0027B689B69AB
S315080116A89A4201D0012342E0234BDB6A23F0F00278
S315080116B87B689B6920491343CB621F4BDB6A23F47A
S315080116C870427B685B691C491343CB621D4B012237
S315080116D81A60FDF7FFF8786108E0FDF7FBF802469E
S315080116E87B69D31A642B01D9032320E0124B1B68A3
S315080116F803F00053002BF0D009E00F4BDB6A03F423
S3150801170870427B685B699A4201D001230FE07B68C6
S315080117181B6803F01003002B08D0074B5B6823F4FA
S3150801172880027B68DB69044913434B60002318462A
S315080117382037BD4680BD00BF00100240007000403A
S31508011748400442427000424280B58AB000AF7860D0
S315080117580023FB6100237B620023BB6100237B61B5
S3150801176800233B610023FB600023BB6000233B6227
S315080117787B68013B0F2B00F21D8101A252F823F069
S315080117883D190108A1190108BD1901089B18010885
S31508011798BD190108BD190108BD190108ED18010887
S315080117A8BD190108BD190108BD190108BD190108A6
S315080117B8BD190108BD190108BD190108C91701088C
S315080117C8834B5B68BB60824B1B6803F08073002BF5
S315080117D800F0F280BB689B0C03F00F037D4AD35CCB
S315080117E8BB61BB6803F48033002B3BD0784BDB6ABB
S315080117F803F00F03784AD35CFB61754BDB6A03F484
S315080118088033002B1CD0724BDB6A1B0903F00F03CC
S315080118180133FB606E4BDB6A1B0A03F00F030233C5
S315080118287B616E4AFB68B2FBF3F37A6903FB02F242
S31508011838FB69B2FBF3F2BB6902FB03F37B6207E0C0
S31508011848664AFB69B2FBF3F2BB6902FB03F37B62E7
S31508011858604B5B7B1A46BB69934208D17B6A5B0876
S315080118687B6204E0BB695E4A02FB03F37B62584B61
S315080118785B6803F48003B3F5800F02D17B6A3B6288
S315080118889AE07B6A5B00574AA2FB03235B083B6223
S3150801189892E04F4BDB6A03F40033002B03D1FFF7C1
S315080118A815FD38628AE04A4B1B6803F08053002B02
S315080118B800F08480464BDB6A1B0903F00F030133EA
S315080118C8FB60434BDB6A1B0B03F00F0302333B61D7
S315080118D8424AFB68B2FBF3F33A6902FB03F35B007E
S315080118E83B626BE03A4BDB6A03F48023002B03D196
S315080118F8FFF7ECFC386263E0354B1B6803F080534D
S31508011908002B5DD0324BDB6A1B0903F00F03013349
S31508011918FB602F4BDB6A1B0B03F00F0302333B619A
S315080119282E4AFB68B2FBF3F33A6902FB03F35B0041
S315080119383B6245E0264B1B6ABB60BB6803F44073F0
S31508011948B3F5807F08D1BB6803F00203002B03D0E7
S315080119584FF400433B621EE0BB6803F44073B3F5DA
S31508011968007F09D11A4B5B6A03F00203002B03D0E7
S3150801197849F640433B620EE0BB6803F44073B3F58E
S31508011988407F1FD1124B1B6803F40033002B19D073
S31508011998154B3B6216E015E0FFF772FD02460C4B44
S315080119A85B689B0B03F0030301335B00B2FBF3F39C
S315080119B83B6208E000BF06E000BF04E000BF02E0A2
S315080119C800BF00E000BF3B6A18462837BD4680BD00
S315080119D800100240506D0108606D010840787D01CC
S315080119E800093D00ABAAAAAAF0FA020080B584B09C
S315080119F800AF78600023FB607B68002B01D10123C7
S31508011A087AE07B685B7CDBB2002B05D17B68002218
S31508011A181A747868FBF782FC7B6802225A7478681C
S31508011A2800F070F80346002B04D07B6804225A7428
S31508011A38012361E0786800F092F80346002B04D088
S31508011A487B6804225A74012356E07B681B685A6826
S31508011A587B681B6822F007025A607B689B68002B23
S31508011A6805D0274B1B6B264A23F001031363244B26
S31508011A78DB6A23F460727B689B6821491343CB624E
S31508011A887B685B68B3F1FF3F03D07B685B68FB60E3
S31508011A980EE00120FFF758FEF860FB68002B04D119
S31508011AA87B6804225A74012326E0FB68013BFB6024
S31508011AB8FB681A0C7B681B6802F00F029A607B6840
S31508011AC81B68FA6892B2DA60786800F070F803461B
S31508011AD8002B04D07B6804225A7401230CE07B6826
S31508011AE80022DA737B6801225A737B6801229A738A
S31508011AF87B6801225A74002318461037BD4680BDF3
S31508011B08006C004080B584B000AF78600023FB60A4
S31508011B187B68002B01D101231DE07B681B685A6885
S31508011B287B681B6822F008025A60FCF7D3FEF86046
S31508011B3809E0FCF7CFFE0246FB68D31AB3F57A7FAC
S31508011B4801D9032307E07B681B685B6803F0080370
S31508011B58002BEED0002318461037BD4680BD80B548
S31508011B6884B000AF78600023FB60FCF7B3FEF86029
S31508011B7809E0FCF7AFFE0246FB68D31AB3F57A7F8C
S31508011B8801D903230FE07B681B685B6803F0200310
S31508011B98002BEED07B681B685A687B681B6842F085
S31508011BA810025A60002318461037BD4680BD80B515
S31508011BB884B000AF78600023FB607B681B685A68AD
S31508011BC87B681B6822F010025A60FCF783FEF860EE
S31508011BD809E0FCF77FFE0246FB68D31AB3F57A7F5C
S31508011BE801D9032307E07B681B685B6803F02003B8
S31508011BF8002BEED0002318461037BD4680BD80B5A8
S31508011C0882B000AF78607B68002B01D1012341E0DF
S31508011C187B6893F83D30DBB2002B06D17B6800223E
S31508011C2883F83C207868FCF77FFB7B68022283F8F7
S31508011C383D207B681A687B6804331946104600F00C
S31508011C48B9FA7B68012283F846207B68012283F862
S31508011C583E207B68012283F83F207B68012283F8AE
S31508011C6840207B68012283F841207B68012283F89A
S31508011C7842207B68012283F843207B68012283F886
S31508011C8844207B68012283F845207B68012283F872
S31508011C983D20002318460837BD4680BD80B582B069
S31508011CA800AF78607B68002B01D1012341E07B688E
S31508011CB893F83D30DBB2002B06D17B68002283F806
S31508011CC83C20786800F039F87B68022283F83D20C1
S31508011CD87B681A687B6804331946104600F06AFA65
S31508011CE87B68012283F846207B68012283F83E2017
S31508011CF87B68012283F83F207B68012283F840200C
S31508011D087B68012283F841207B68012283F84220F7
S31508011D187B68012283F843207B68012283F84420E3
S31508011D287B68012283F845207B68012283F83D20D8
S31508011D38002318460837BD4680BD80B483B000AF76
S31508011D48786000BF0C37BD4680BC704780B584B043
S31508011D5800AF786039603B68002B09D17B6893F836
S31508011D683E30DBB2012B14BF01230023DBB222E08C
S31508011D783B68042B09D17B6893F83F30DBB2012B0A
S31508011D8814BF01230023DBB215E03B68082B09D1F0
S31508011D987B6893F84030DBB2012B14BF012300237B
S31508011DA8DBB208E07B6893F84130DBB2012B14BF3C
S31508011DB801230023DBB2002B01D0012363E03B6832
S31508011DC8002B04D17B68022283F83E2013E03B6886
S31508011DD8042B04D17B68022283F83F200BE03B6879
S31508011DE8082B04D17B68022283F8402003E07B682C
S31508011DF8022283F841207B681B6801223968184644
S31508011E0800F06EFC7B681B68214A934207D17B6800
S31508011E181B685A6C7B681B6842F400425A647B68E3
S31508011E281B681B4A934213D07B681B68B3F1804F22
S31508011E380ED07B681B68174A934209D07B681B68D2
S31508011E48154A934204D07B681B68144A934211D1F8
S31508011E587B681B689B6803F00703FB60FB68062B16
S31508011E6810D07B681B681A687B681B6842F00102F8
S31508011E781A6007E07B681B681A687B681B6842F06A
S31508011E8801021A60002318461037BD4680BD00BFF7
S31508011E98002C01400004004000080040000C0040E6
S31508011EA880B586B000AFF860B9607A600023FB7523
S31508011EB8FB6893F83C30012B01D10223AEE0FB689D
S31508011EC8012283F83C207B680C2B00F29F8001A233
S31508011ED852F823F0111F01081520010815200108D9
S31508011EE815200108511F01081520010815200108A8
S31508011EF815200108931F0108152001081520010856
S31508011F0815200108D31F0108FB681B68B96818461C
S31508011F1800F0C8F9FB681B689A69FB681B6842F0F8
S31508011F2808029A61FB681B689A69FB681B6822F0B4
S31508011F3804029A61FB681B689969BB681A69FB6898
S31508011F481B680A439A6164E0FB681B68B968184606
S31508011F5800F00EFAFB681B689A69FB681B6842F46D
S31508011F6800629A61FB681B689A69FB681B6822F418
S31508011F7880629A61FB681B689969BB681B691A02C2
S31508011F88FB681B680A439A6143E0FB681B68B968E2
S31508011F98184600F057FAFB681B68DA69FB681B687C
S31508011FA842F00802DA61FB681B68DA69FB681B6894
S31508011FB822F00402DA61FB681B68D969BB681A69E9
S31508011FC8FB681B680A43DA6123E0FB681B68B96882
S31508011FD8184600F0A1FAFB681B68DA69FB681B68F2
S31508011FE842F40062DA61FB681B68DA69FB681B68F8
S31508011FF822F48062DA61FB681B68D969BB681B69C8
S315080120081A02FB681B680A43DA6102E00123FB75B9
S3150801201800BFFB68002283F83C20FB7D1846183769
S31508012028BD4680BD80B584B000AF786039600023AD
S31508012038FB737B6893F83C30012B01D10223B4E08A
S315080120487B68012283F83C207B68022283F83D20BD
S315080120587B681B689B68BB60BB6823F07703BB601A
S31508012068BB6823F47F43BB607B681B68BA689A60C0
S315080120783B681B68B3F5005F3ED0B3F5005F00F215
S315080120888780B3F5805F00F08680B3F5805F7FD8D7
S31508012098702B1AD0702B7BD8602B50D0602B77D831
S315080120A8502B3CD0502B73D8402B58D0402B6FD887
S315080120B8302B64D0302B6BD8202B60D0202B67D8D7
S315080120C8002B5CD0102B5AD062E07B6818683B68F5
S315080120D899683B685A683B68DB6800F0E2FA7B68EE
S315080120E81B689B68BB60BB6843F07703BB607B686A
S315080120F81B68BA689A604FE07B6818683B689968F4
S315080121083B685A683B68DB6800F0CBFA7B681B6852
S315080121189A687B681B6842F480429A603CE07B684F
S3150801212818683B6859683B68DB681A4600F042FA42
S315080121387B681B685021184600F099FA2CE07B68E1
S3150801214818683B6859683B68DB681A4600F060FA04
S315080121587B681B686021184600F089FA1CE07B68D1
S3150801216818683B6859683B68DB681A4600F022FA22
S315080121787B681B684021184600F079FA0CE07B68F1
S315080121881A683B681B681946104600F070FA03E09E
S315080121980123FB7300E000BF7B68012283F83D2019
S315080121A87B68002283F83C20FB7B18461037BD461E
S315080121B880BD000080B485B000AF786039607B685F
S315080121C81B68FB607B68334A93420FD07B68B3F17F
S315080121D8804F0BD07B68304A934207D07B682F4AD9
S315080121E8934203D07B682E4A934208D1FB6823F0B1
S315080121F87003FB603B685B68FA681343FB607B689E
S31508012208244A93420FD07B68B3F1804F0BD07B6881
S31508012218214A934207D07B68204A934203D07B68B8
S315080122281F4A934208D1FB6823F44073FB603B6855
S31508012238DB68FA681343FB60FB6823F080023B6896
S315080122485B691343FB607B68FA681A603B689A689E
S315080122587B68DA623B681A687B689A627B680D4A0A
S31508012268934203D13B681A697B681A637B68012222
S315080122785A617B681B6903F00103002B05D07B684B
S315080122881B6923F001027B681A6100BF1437BD4632
S3150801229880BC7047002C014000040040000800403B
S315080122A8000C004080B487B000AF786039607B685D
S315080122B81B6A7B617B681B6A23F001027B681A62C9
S315080122C87B685B683B617B689B69FB60FB6823F0FD
S315080122D87003FB60FB6823F00303FB603B681B681C
S315080122E8FA681343FB607B6923F002037B613B6849
S315080122F89B687A6913437B617B681C4A93420CD1B4
S315080123087B6923F008037B613B68DB687A691343B9
S315080123187B617B6923F004037B617B68134A9342DB
S3150801232811D13B6923F480733B613B6923F400733C
S315080123383B613B685B693A6913433B613B689B6947
S315080123483A6913433B617B683A695A607B68FA685C
S315080123589A613B685A687B685A637B687A691A6224
S3150801236800BF1C37BD4680BC704700BF002C014022
S3150801237880B487B000AF786039607B681B6A7B6177
S315080123887B681B6A23F010027B681A627B685B68A4
S315080123983B617B689B69FB60FB6823F4E043FB6050
S315080123A8FB6823F44073FB603B681B681B02FA68E9
S315080123B81343FB607B6923F020037B613B689B68B9
S315080123C81B017A6913437B617B681D4A93420DD1C8
S315080123D87B6923F080037B613B68DB681B017A69AB
S315080123E813437B617B6923F040037B617B68144A4D
S315080123F8934213D13B6923F480633B613B6923F418
S3150801240800633B613B685B699B003A6913433B611F
S315080124183B689B699B003A6913433B617B683A6948
S315080124285A607B68FA689A613B685A687B689A6356
S315080124387B687A691A6200BF1C37BD4680BC70473B
S31508012448002C014080B487B000AF786039607B689A
S315080124581B6A7B617B681B6A23F480727B681A6234
S315080124687B685B683B617B68DB69FB60FB6823F01B
S315080124787003FB60FB6823F00303FB603B681B687A
S31508012488FA681343FB607B6923F400737B613B6835
S315080124989B681B027A6913437B617B681D4A9342D1
S315080124A80DD17B6923F400637B613B68DB681B02FA
S315080124B87A6913437B617B6923F480637B617B6853
S315080124C8144A934213D13B6923F480533B613B6910
S315080124D823F400533B613B685B691B013A69134363
S315080124E83B613B689B691B013A6913433B617B68FE
S315080124F83A695A607B68FA68DA613B685A687B68A0
S31508012508DA637B687A691A6200BF1C37BD4680BCE4
S31508012518704700BF002C014080B487B000AF7860CF
S3150801252839607B681B6A3B617B681B6A23F48052A6
S315080125387B681A627B685B687B617B68DB69FB6021
S31508012548FB6823F4E043FB60FB6823F44073FB60F4
S315080125583B681B681B02FA681343FB603B6923F453
S3150801256800533B613B689B681B033A6913433B610C
S315080125787B680F4A934209D17B6923F480437B61BF
S315080125883B685B699B017A6913437B617B687A6956
S315080125985A607B68FA68DA613B685A687B681A6424
S315080125A87B683A691A6200BF1C37BD4680BC70470A
S315080125B8002C014080B487B000AFF860B9607A6032
S315080125C8FB681B6A7B61FB681B6A23F00102FB68CF
S315080125D81A62FB689B693B613B6923F0F0033B611F
S315080125E87B681B013A6913433B617B6923F00A033C
S315080125F87B617A69BB6813437B61FB683A699A61AF
S31508012608FB687A691A6200BF1C37BD4680BC7047E9
S3150801261880B487B000AFF860B9607A60FB681B6A56
S315080126287B61FB681B6A23F01002FB681A62FB6868
S315080126389B693B613B6923F470433B617B681B03D8
S315080126483A6913433B617B6923F0A0037B61BB6845
S315080126581B017A6913437B61FB683A699A61FB68CE
S315080126687A691A6200BF1C37BD4680BC704780B4B8
S3150801267885B000AF786039607B689B68FB60FB684A
S3150801268823F07003FB603A68FB68134343F00703BA
S31508012698FB607B68FA689A6000BF1437BD4680BC40
S315080126A8704780B487B000AFF860B9607A603B605C
S315080126B8FB689B687B617B6923F47F437B613B6885
S315080126C81A027B681A43BB6813437A6913437B6109
S315080126D8FB687A699A6000BF1C37BD4680BC70479B
S315080126E880B487B000AFF860B9607A60BB6803F058
S315080126F81F03012202FA03F37B61FB681A6A7B69E5
S31508012708DB431A40FB681A62FB681A6ABB6803F05E
S315080127181F03796801FA03F31A43FB681A6200BFB3
S315080127281C37BD4680BC704780B485B000AF786059
S3150801273839607B6893F83C30012B01D102234BE0C1
S315080127487B68012283F83C207B68022283F83D20B6
S315080127587B681B685B68FB607B681B689B68BB605A
S31508012768FB6823F07003FB603B681B68FA68134330
S31508012778FB607B681B68FA685A607B681B68194A9C
S31508012788934213D07B681B68B3F1804F0ED07B68E0
S315080127981B68154A934209D07B681B68134A9342FA
S315080127A804D07B681B68124A93420CD1BB6823F094
S315080127B88003BB603B685B68BA681343BB607B6888
S315080127C81B68BA689A607B68012283F83D207B6892
S315080127D8002283F83C20002318461437BD4680BCDE
S315080127E8704700BF002C0140000400400008004063
S315080127F8000C004080B582B000AF78607B68002B7A
S3150801280801D1012342E07B6893F84130DBB2002B02
S3150801281806D17B68002283F840207868FBF78EFE8C
S315080128287B68242283F841207B681B68DA687B6801
S315080128381B6822F40052DA60786800F0B3FE7B68F8
S315080128481B681A697B681B6822F490421A617B68BF
S315080128581B685A697B681B6822F02A025A617B68D9
S315080128681B68DA687B681B6842F40052DA607B6881
S3150801287800225A647B68202283F841207B6820223B
S3150801288883F842207B6800225A63002318460837D2
S31508012898BD4680BD80B485B000AFF860B9601346FF
S315080128A8FB80FB6893F84130DBB2202B21D1BB684A
S315080128B8002B02D0FB88002B01D101231AE0FB6803
S315080128C8BA681A62FB68FA889A84FB68FA88DA840D
S315080128D8FB6800225A64FB68212283F84120FB68B9
S315080128E81B68DA68FB681B6842F08002DA60002315
S315080128F800E0022318461437BD4680BC704780B5E8
S315080129088CB000AFF860B9601346FB80FB6893F892
S315080129184230DBB2202B4AD1BB68002B02D0FB8898
S31508012928002B01D1012343E0FB6801221A63FB68E6
S3150801293800225A63FB881A46B968F86800F0FDFB55
S31508012948034687F82F3097F82F30002B2CD1FB68D0
S315080129581B6B012B25D100233B61FB681B681B6890
S315080129683B61FB681B685B683B613B69FB681B68E5
S315080129780C33BB61BB6953E8003F7B617B6943F054
S315080129881003BB62FB681B680C33BA6A7A623B623E
S31508012998396A7A6A41E80023FB61FB69002BE5D1AC
S315080129A802E0012387F82F3097F82F3000E0022339
S315080129B818463037BD4680BD80B5A2B000AF7860ED
S315080129C80123C7F884307B681B680C333B663B6E6A
S315080129D853E8003FFB65FB6D23F4F073C7F88030B5
S315080129E87B681B680C33D7F88020FA66BB66B96E14
S315080129F8FA6E41E800237B667B6E002BE3D17B6880
S31508012A081B681433FB64FB6C53E8003FBB64BB6C5F
S31508012A1823F00103FB677B681B681433FA6FBA65F1
S31508012A287B65796DBA6D41E800233B653B6D002BE3
S31508012A38E5D17B681B6B012B19D17B681B680C33A5
S31508012A48BB63BB6B53E8003F7B637B6B23F01003C7
S31508012A58BB677B681B680C33BA6F7A643B64396C4D
S31508012A687A6C41E80023FB63FB6B002BE5D17B6895
S31508012A789B6B002B0FD07B681B685B6903F080038F
S31508012A88002B04D07B689B6B534A5A6303E07B6827
S31508012A989B6B00225A637B68DB6B002B0FD07B6824
S31508012AA81B685B6903F04003002B04D07B68DB6B6A
S31508012AB84A4A5A6303E07B68DB6B00225A637B68E0
S31508012AC81B685B6903F08003002B2DD07B681B68A4
S31508012AD814337B627B6A53E8003F3B623B6A23F007
S31508012AE880037B677B681B6814337A6F3A63FB62DA
S31508012AF8F96A3A6B41E80023BB62BB6A002BE5D148
S31508012B087B689B6B002B0FD07B689B6B1846FDF780
S31508012B1845FC0346002B04D07B689B6B00225A634D
S31508012B2802E00023C7F884307B681B685B6903F0F9
S31508012B384003002B30D07B681B6814333B613B6923
S31508012B4853E8003FFB60FB6823F040033B677B685B
S31508012B581B6814333A6FFA61BB61B969FA6941E8C6
S31508012B6800237B617B69002BE5D17B68DB6B002B36
S31508012B7812D07B68DB6B1846FDF710FC0346002B61
S31508012B8807D07B68DB6B00225A630123C7F88430B8
S31508012B9802E00023C7F88430D7F88430012B16D110
S31508012BA87B680022DA847B680022DA857B68002242
S31508012BB85A647B68202283F841207B68202283F89F
S31508012BC842207B6800221A63786800F0ADFA002370
S31508012BD818468837BD4680BDA13201080133010868
S31508012BE880B5BAB000AF78607B681B681B68C7F800
S31508012BF8E4307B681B68DB68C7F8E0307B681B68CC
S31508012C085B69C7F8DC300023C7F8D8300023C7F852
S31508012C18D430D7F8E43003F00F03C7F8D830D7F81B
S31508012C28D830002B0FD1D7F8E43003F02003002B56
S31508012C3809D0D7F8E03003F02003002B03D07868D1
S31508012C4800F0F1FB5BE2D7F8D830002B00F0DE8004
S31508012C58D7F8DC3003F00103002B06D1D7F8E030AA
S31508012C6803F49073002B00F0D180D7F8E43003F011
S31508012C780103002B0BD0D7F8E03003F48073002B3F
S31508012C8805D07B685B6C43F001027B685A64D7F808
S31508012C98E43003F00403002B0BD0D7F8DC3003F03B
S31508012CA80103002B05D07B685B6C43F002027B6845
S31508012CB85A64D7F8E43003F00203002B0BD0D7F88F
S31508012CC8DC3003F00103002B05D07B685B6C43F00D
S31508012CD804027B685A64D7F8E43003F00803002B2A
S31508012CE811D0D7F8E03003F02003002B05D1D7F827
S31508012CF8DC3003F00103002B05D07B685B6C43F0DD
S31508012D0808027B685A647B685B6C002B00F0F281C9
S31508012D18D7F8E43003F02003002B08D0D7F8E030C1
S31508012D2803F02003002B02D0786800F07CFB7B684F
S31508012D381B685B6903F04003002B14BF01230023BA
S31508012D48DBB2C7F8D4307B685B6C03F00803002B49
S31508012D5803D1D7F8D430002B4FD0786800F026FA7B
S31508012D687B681B685B6903F04003002B41D07B68CD
S31508012D781B681433C7F89C30D7F89C3053E8003FD2
S31508012D88C7F89830D7F8983023F04003C7F8D030F9
S31508012D987B681B681433D7F8D020C7F8A820C7F86A
S31508012DA8A430D7F8A410D7F8A82041E80023C7F813
S31508012DB8A030D7F8A030002BD9D17B68DB6B002B64
S31508012DC813D07B68DB6B7E4A5A637B68DB6B1846D4
S31508012DD8FDF7E4FA0346002B16D07B68DB6B5B6BC1
S31508012DE87A68D26B104698470EE0786800F093F92E
S31508012DF80AE0786800F08FF906E0786800F08BF940
S31508012E087B6800225A6475E100BF73E17B681B6B16
S31508012E18012B40F04F81D7F8E43003F01003002B5B
S31508012E2800F04881D7F8E03003F01003002B00F0D2
S31508012E3841810023BB607B681B681B68BB607B6894
S31508012E481B685B68BB60BB687B681B685B6903F0CA
S31508012E584003002B00F0B6807B68DB6B1B685B6858
S31508012E68A7F8BE30B7F8BE30002B00F045817B685D
S31508012E789B8DB7F8BE209A4280F03E817B68B7F8E9
S31508012E88BE20DA857B68DB6B9B69202B00F088807E
S31508012E987B681B680C33C7F88830D7F8883053E83D
S31508012EA8003FC7F88430D7F8843023F48073C7F80D
S31508012EB8B8307B681B680C33D7F8B820C7F8942054
S31508012EC8C7F89030D7F89010D7F8942041E800232E
S31508012ED8C7F88C30D7F88C30002BD9D17B681B689A
S31508012EE814337B677B6F53E8003F3B673B6F23F0DF
S31508012EF80103C7F8B4307B681B681433D7F8B420C4
S31508012F08C7F88020FB67F96FD7F8802041E80023C6
S31508012F18BB67BB6F002BE1D17B681B6814333B6623
S31508012F283B6E53E8003FFB65FB6D23F04003C7F88A
S31508012F38B0307B681B681433D7F8B020FA66BB66CD
S31508012F48B96EFA6E41E800237B667B6E002BE3D1E6
S31508012F587B68202283F842207B6800221A637B68F3
S31508012F681B680C33FB64FB6C53E8003FBB64BB6C02
S31508012F7823F01003C7F8AC307B681B680C33D7F805
S31508012F88AC20BA657B65796DBA6D41E800233B6566
S31508012F983B6D002BE3D17B68DB6B1846FDF7C3F95C
S31508012FA87B6802225A637B689A8D7B68DB8D9BB2A4
S31508012FB8D31A9BB219467868FAF772FA9CE000BFE9
S31508012FC8793201087B689A8D7B68DB8D9BB2D31AA7
S31508012FD8A7F8CE307B68DB8D9BB2002B00F08E807C
S31508012FE8B7F8CE30002B00F089807B681B680C3354
S31508012FF8BB63BB6B53E8003F7B637B6B23F490731E
S31508013008C7F8C8307B681B680C33D7F8C8207A64B8
S315080130183B64396C7A6C41E80023FB63FB6B002B34
S31508013028E3D17B681B6814337B627B6A53E8003FEC
S315080130383B623B6A23F00103C7F8C4307B681B6807
S315080130481433D7F8C4203A63FB62F96A3A6B41E844
S315080130580023BB62BB6A002BE3D17B68202283F875
S3150801306842207B6800221A637B681B680C333B6124
S315080130783B6953E8003FFB60FB6823F01003C7F878
S31508013088C0307B681B680C33D7F8C020FA61BB616E
S31508013098B969FA6941E800237B617B69002BE3D1A9
S315080130A87B6802225A63B7F8CE3019467868FAF768
S315080130B8F7F923E0D7F8E43003F08003002B09D0A9
S315080130C8D7F8E03003F08003002B03D0786800F0C6
S315080130D843F914E0D7F8E43003F04003002B0ED087
S315080130E8D7F8E03003F04003002B08D0786800F0E1
S315080130F882F904E000BF02E000BF00E000BFE8373C
S31508013108BD4680BD80B483B000AF786000BF0C3778
S31508013118BD4680BC704780B483B000AF786000BFF5
S315080131280C37BD4680BC704780B483B000AF786061
S3150801313800BF0C37BD4680BC704780B485B000AF68
S31508013148F860B9601346FB80FB68BA689A62FB683F
S31508013158FA889A85FB68FA88DA85FB6800225A6430
S31508013168FB68222283F84220FB681B69002B07D0DB
S31508013178FB681B68DA68FB681B6842F48072DA60C8
S31508013188FB681B685A69FB681B6842F001025A61A9
S31508013198FB681B68DA68FB681B6842F02002DA607C
S315080131A8002318461437BD4680BC704780B495B0CD
S315080131B800AF78607B681B680C337B637B6B53E8CD
S315080131C8003F3B633B6B23F49073FB647B681B6886
S315080131D80C33FA6C3A64FB63F96B3A6C41E80023E1
S315080131E8BB63BB6B002BE5D17B681B6814333B6259
S315080131F83B6A53E8003FFB61FB6923F00103BB64A3
S315080132087B681B681433BA6CFA62BB62B96AFA6AD4
S3150801321841E800237B627B6A002BE5D17B681B6B3F
S31508013228012B19D17B681B680C33FB60FB6853E8D3
S31508013238003FBB60BB6823F010037B647B681B688F
S315080132480C337A6CBA617B617969BA6941E80023FA
S315080132583B613B69002BE5D17B68202283F8422034
S315080132687B6800221A6300BF5437BD4680BC704785
S3150801327880B584B000AF78607B685B6AFB60FB68E1
S315080132880022DA85FB680022DA84F868FFF743FF2B
S3150801329800BF1037BD4680BD80B584B000AF7860E1
S315080132A87B685B6AFB60FB689B6B00225A63FB6859
S315080132B8DB6B002B04D0FB68DB6B5B6B002B17D130
S315080132C8FB680022DA84FB680022DA85FB6800229B
S315080132D85A64FB68202283F84120FB68202283F878
S315080132E84220FB6800221A63F868FFF71DFF00E011
S315080132F800BF1037BD4680BD80B584B000AF786081
S315080133087B685B6AFB60FB68DB6B00225A63FB68B8
S315080133189B6B002B04D0FB689B6B5B6B002B17D14F
S31508013328FB680022DA84FB680022DA85FB6800223A
S315080133385A64FB68202283F84120FB68202283F817
S315080133484220FB6800221A63F868FFF7EDFE00E0E1
S3150801335800BF1037BD4680BD80B485B000AF786020
S315080133687B6893F84130DBB2212B3ED17B689B6899
S31508013378B3F5805F14D17B681B69002B10D17B6874
S315080133881B6AFB60FB681B881A467B681B68C2F3C5
S3150801339808025A607B681B6A9A1C7B681A6208E0ED
S315080133A87B681B6A591C7A6811621A787B681B68DC
S315080133B85A607B68DB8C9BB2013B9BB27A681946DB
S315080133C8D184002B0FD17B681B68DA687B681B6878
S315080133D822F08002DA607B681B68DA687B681B68FA
S315080133E842F04002DA60002300E002231846143747
S315080133F8BD4680BC704780B582B000AF78607B68EF
S315080134081B68DA687B681B6822F04002DA607B6809
S31508013418202283F841207868FAF794F80023184699
S315080134280837BD4680BD80B58CB000AF78607B682B
S3150801343893F84230DBB2222B40F0AE807B689B685A
S31508013448B3F5805F17D17B681B69002B13D100235D
S31508013458FB627B689B6ABB627B681B685B689BB27D
S31508013468C3F308039AB2BB6A1A807B689B6A9A1CDB
S315080134787B689A6226E07B689B6AFB620023BB62CB
S315080134887B689B68B3F5805F07D07B689B68002BD0
S315080134980AD17B681B69002B06D17B681B685B68A8
S315080134A8DAB2FB6A1A7008E07B681B685B68DBB2EC
S315080134B803F07F03DAB2FB6A1A707B689B6A5A1CA7
S315080134C87B689A627B68DB8D9BB2013B9BB27A6803
S315080134D81946D185002B5DD17B681B68DA687B683C
S315080134E81B6822F02002DA607B681B68DA687B6849
S315080134F81B6822F48072DA607B681B685A697B68E4
S315080135081B6822F001025A617B68202283F842204F
S315080135187B6800225A637B681B6B012B35D17B6854
S3150801352800221A637B681B680C337B617B6953E845
S31508013538003F3B613B6923F010037B627B681B688C
S315080135480C337A6A3A62FB61F9693A6A41E80023F7
S31508013558BB61BB69002BE5D17B681B681B6803F057
S315080135681003102B0AD10023FB607B681B681B68B4
S31508013578FB607B681B685B68FB60FB687B689B8DE7
S3150801358819467868F9F78CFF02E07868FFF7BAFDFB
S31508013598002302E0002300E0022318463037BD461F
S315080135A880BD000080B584B000AF78607B681B6871
S315080135B81B6923F440517B68DA687B681B680A43F0
S315080135C81A617B689A687B681B691A437B685B6919
S315080135D81343BB607B681B68DB6823F4B05323F08D
S315080135E80C037A681268B9680B43D3607B681B6851
S315080135F85B6923F440717B689A697B681B680A438F
S315080136085A617B681B682C4A934203D1FDF738FF38
S31508013618F86002E0FDF720FFF860FA6813469B0098
S3150801362813449A001A447B685B689B00B2FBF3F360
S31508013638224AA2FB03235B091901FA6813469B0070
S3150801364813449A001A447B685B689B00B2FBF3F241
S315080136581A4BA3FB02035B09642000FB03F3D31A85
S315080136681B013233154AA2FB03235B0903F0F00356
S315080136781944FA6813469B0013449A001A447B684E
S315080136885B689B00B2FBF3F20C4BA3FB02035B09D5
S31508013698642000FB03F3D31A1B013233074AA2FB42
S315080136A803235B0903F00F027B681B680A449A60C7
S315080136B800BF1037BD4680BD003801401F85EB5154
S315080136C8002B2DE9F0471D46BBBF03F100431D46F4
S315080136D800232D2388B01446B8BF1446129A109EA3
S315080136E81370149BDDF84CA023F02008B8F1460F97
S315080136F805D0B8F1450F00D10136022300E00323AE
S3150801370807AA049206AACDE902A2CDE900362246FD
S315080137182B4600F001FFB8F1470F074619D1119B4F
S31508013728DB070ED500EB06090022002320462946A9
S31508013738F5F7A2F908B1CDF81C903022079B4B453D
S315080137481ED33846079B159ADB1B136008B0BDE8DC
S31508013758F087B8F1460F00EB0609E5D10378302B57
S315080137680AD10022002320462946F5F785F918B912
S31508013778C6F10106CAF80060DAF800309944D3E7B9
S31508013788591C07911A70D9E7F7B50029B6BF2D2331
S315080137982B23494209290270437029DD0DF10703D4
S315080137A81D460A27B1FBF7F61A4607FB16143034E5
S315080137B802F8014C0C46632C314603F1FF33F1DC60
S315080137C83031941E03F8011C2346411CAB420AD327
S315080137D80DF109039B1AAC4288BF0023023303443F
S315080137E8181A03B0F0BD13F8016B01F8016FEDE77C
S315080137F8302330318370C170031DF1E72DE9F04F8D
S3150801380891B00C46DDF8688016461F46054600F055
S31508013818BDFD036818460893F4F702FD00230E93C5
S31508013828D8F800300990073323F0070303F1080293
S3150801383894F818A0D4F800B0C8F80020D3E900898C
S3150801384829F000430B93CDF828804FF0FF32DDE9C4
S315080138580A01C4E912899C4BF5F740F970BBDDE901
S315080138680A014FF0FF32984BF5F71AF930BB0022D7
S31508013878002340464946F5F709F910B12D2384F87E
S315080138884330924A924BBAF1470F8CBF90469846F5
S3150801389803234FF0000923612BF004032360334601
S315080138A82146284600970FAA00F0D4F9013040F0BE
S315080138B890804FF0FF3011B0BDE8F08F42464B4675
S315080138C840464946F5F70AF948B14B46002BB8BFB1
S315080138D82D23804AB8BF84F843307F4BD3E7636802
S315080138E80AF0DF015A1C3FD10623636000224BF414
S315080138F88063236006920EAACDE904A20DAA039253
S315080139080DF13302CDE90132636842460093284630
S315080139184B460A91FFF7D4FE0A99804647290D991D
S3150801392828D1C81C02DB6368994240DDAAF1020A5C
S315080139385FFA8AFA5246013904F150000D91FFF7E8
S3150801394823FF0E9A81461318012A236102DC22688D
S31508013958D20701D5013323619DF83330002B9ED058
S315080139682D2384F843309AE74729BFD1002BBDD1C7
S315080139780123BAE7BAF1650FDCD9BAF1660F18D18E
S31508013988002963680BDD216113B92268D00702D5BE
S3150801399801330B4423614FF00009A165DCE713B92C
S315080139A82268D20701D50233F4E70123F2E74FF07B
S315080139B8670A0E9B994205DB23682161D807EAD570
S315080139C84B1CE7E70029CCBF0122C1F102021344C7
S315080139D8E0E723685A0507D423694246314628464B
S315080139E8B84701302BD164E7BAF1650F40F2DC809C
S315080139F8D4E9120100220023F5F73EF8002833D04E
S31508013A08012331462846354AB84701303FF451AFB4
S31508013A18DDE90D38434502DB2368D8070FD5DDE90B
S31508013A28082331462846B84701303FF442AF4FF0DC
S31508013A38000908F1FF3804F11A0AC84509DC2368A0
S31508013A489B0700F10281E0680F9B9842B8BF1846A8
S31508013A5831E70123524631462846B84701303FF433
S31508013A6828AF09F10109E8E70D9B002B38DC01238A
S31508013A7831462846194AB84701303FF41AAFDDE9F5
S31508013A880D3959EA030302D12368D907D7D5DDE9E0
S31508013A98082331462846B84701303FF40AAF4FF0A4
S31508013AA8000A04F11A0B0D9B5B42534501DC4B4690
S31508013AB893E701235A4631462846B84701303FF469
S31508013AC8F8AE0AF1010AEEE7FFFFEF7F746D010808
S31508013AD8706D01087C6D0108786D0108806D010813
S31508013AE8A36DDDF838A05345A8BF5346002B994660
S31508013AF836DC4FF0000B29EAE97904F11A02A36DBD
S31508013B080A93A3EB09035B4531DC0D9B9A453ADC1D
S31508013B182368DA0737D40D9BAAEB03090A9BAAEB94
S31508013B2803039945A8BF9946B9F1000F33DC4FF04D
S31508013B38000829EAE97904F11A0B0D9BAAEB030394
S31508013B48A3EB090343457FF77AAF01235A46314662
S31508013B582846B84701303FF4ACAE08F10108ECE74E
S31508013B68424631462846B8470130C2D1A1E6012363
S31508013B78314628460A92B84701303FF49AAE0A9A5E
S31508013B880BF1010BBBE73146DDE908232846B8479F
S31508013B980130C0D18DE60A9A4B4631462846424439
S31508013BA8B8470130C3D184E6DDF838A0BAF1010F68
S31508013BB801DCDB0736D50123424631462846B84794
S31508013BC801303FF476AEDDE9082331462846B84781
S31508013BD801303FF46EAED4E91201002200230AF13E
S31508013BE8FF3AF4F749FFC0B9534608F101023146CD
S31508013BF82846B84701300CD15BE601235A463146B7
S31508013C082846B84701303FF454AE08F10108D045B3
S31508013C18F3DB4B4604F15002E0E64FF0000804F1E5
S31508013C281A0BF4E701234246E1E701234A463146DE
S31508013C382846B84701303FF43CAE08F10108E36865
S31508013C480F995B1A4345F0DCFDE64FF0000804F1CD
S31508013C581909F4E72DE9F047164698468A680B6963
S31508013C6807469342B8BF1346336091F843200C467A
S31508013C78DDF820900AB1013333602368990642BFFB
S31508013C88336802333360256815F0060506D104F151
S31508013C98190AE36832689B1AAB422BDC94F843305D
S31508013CA82268003B18BF0123920630D4414638469C
S31508013CB804F14302C847013023D02368226903F077
S31508013CC80603042B14BF002533684FF0000608BF06
S31508013CD8E56804F11A0408BFED1A54F8123C08BF3E
S31508013CE825EAE5759342C4BF9B1AED18B5421AD160
S31508013CF8002008E00123524641463846C8470130A4
S31508013D0803D14FF0FF30BDE8F0870135C1E7302010
S31508013D18E11881F843005A1C94F8451022440233E5
S31508013D2882F84310C2E70123224641463846C84766
S31508013D380130E6D00136D9E72DE9FF470F7E9146CE
S31508013D48782F80460C469A460C9E01F1430207D8FD
S31508013D58622F0AD8002F00F0D180582F00F0B880BA
S31508013D6804F1420684F842703AE0A7F16303152B79
S31508013D78F6D801A151F823F0D93D0108ED3D01080E
S31508013D88693D0108693D0108693D0108693D010860
S31508013D98ED3D0108693D0108693D0108693D0108CC
S31508013DA8693D0108EB3E0108173E0108A53E0108D1
S31508013DB8693D0108693D01080D3F0108693D01088A
S31508013DC8173E0108693D0108693D0108AD3E01082C
S31508013DD833681A1D1B68326004F1420684F84230BA
S31508013DE801239CE033682068191D3160060601D550
S31508013DF81D6803E04506FBD5B3F90050002D03DA23
S31508013E082D236D4284F843300A23584811E0216866
S31508013E183368080653F8045B02D4490648BFADB2AD
S31508013E286F2F336014BF0A2308235048002184F8EA
S31508013E3843106668002EA66005DB21682E4321F02B
S31508013E48040121604BD01646B5FBF3F103FB115764
S31508013E58C75D06F8017D2F46BB420D46F4D9082BE6
S31508013E680BD12368DF0708D5236961689942DEBF44
S31508013E78302306F8013C06F1FF36921B22614B46B0
S31508013E8821464046CDF800A003AAFFF7E3FE013014
S31508013E984AD14FF0FF3004B0BDE8F087236843F0F4
S31508013EA8200323607827324884F8457023683168E7
S31508013EB81F0651F8045B02D45F0648BFADB23160EC
S31508013EC8D90744BF43F0200323601DB11023ADE78A
S31508013ED82648E9E7236823F020032360F6E7164610
S31508013EE8BDE733682568181D616930602E061B68A9
S31508013EF801D5196002E06806FBD519800023164624
S31508013F082361BCE7336800211A1D32601E6862689E
S31508013F18304600F03FFA08B1801B60606368236188
S31508013F28002384F84330AAE73246494640462369BE
S31508013F38D0470130ADD023689B0713D4E068039BAB
S31508013F489842B8BF1846A6E701233246494640466D
S31508013F58D04701309DD00135E36803995B1AAB4216
S31508013F68F2DCEBE7002504F11906F5E7826D01088D
S31508013F78936D0108002310B50446C0E90033C0E96A
S31508013F880433836081814366C281836119460822A5
S31508013F985C3000F0FFF80D4B246263620C4BA36298
S31508013FA80C4BE3620C4B23630C4B9C4206D003F182
S31508013FB86802944202D0D0339C4205D104F15800D4
S31508013FC8BDE8104000F0DEB910BD00BFA95F0108C1
S31508013FD8CB5F0108036001082760010890100020DB
S31508013FE8024A0349034800F0A5B800BF8400002027
S31508013FF84D5801089400002041680C4B10B59942A8
S31508014008044601D001F01EFCA168094B994202D069
S31508014018204601F017FCE168064B994204D0204670
S31508014028BDE8104001F00EBC10BD00BF901000207D
S31508014038F81000206011002010B50B4B0B4C0C4AE8
S3150801404820461A6004210022FFF794FF04F168004C
S3150801405801220921FFF78EFF04F1D0000222BDE8EB
S3150801406810401221FFF786BFC811002090100020C2
S31508014078E93F0108014800F086B900BFCD110020C3
S31508014088014800F081B900BFCD11002010B50446DA
S31508014098FFF7F0FF236A1BB1BDE81040FFF7F0BF31
S315080140A8044B2362044B1B68002BF5D1FFF7C4FFA9
S315080140B8F2E700BF01400108C811002030B51446CF
S315080140C8002C05461A469BB005DA8B2303604FF088
S315080140D8FF301BB030BD4FF40273ADF80C304FF00A
S315080140E8000319930CBF234604F1FF330293059382
S315080140F84FF6FF7300910491ADF80E3069461E9B81
S3150801410801F03AF8431CBCBF8B232B60002CE0D086
S315080141180022009B1A70DCE707B5009313460A4686
S31508014128014603480068FFF7C9FF03B05DF804FBB9
S31508014138900000202DE9F8430746884614460026CC
S31508014148D4E90195B9F1010905D52468002CF7D1F7
S315080141583046BDE8F883AB89012B07D9B5F90E3086
S31508014168013303D029463846C04706436835E9E787
S315080141780FB407B5064904AB086853F8042B8168D8
S31508014188019301F01DF903B05DF804EB04B070471B
S315080141989000002003460244934200D1704703F871
S315080141A8011BF9E738B50B4B04461D686B6B53B908
S315080141B8242001F01DFA0246686320B93D21064B01
S315080141C8064800F003F92046696BBDE8384000F057
S315080141D807B800BF90000020A46D0108BB6D01084F
S315080141E82DE9F04100230C46D0E900014C4AF4F7C1
S315080141F8FDFF4FF46161002ABCBF02F5A83202F53A
S31508014208C072B2FBF1F301FB13224FF03C01A36024
S31508014218B2FBF1F301FB132222604FF0070200F506
S315080142282F20ACBF00F66C2000F66B206360C31C18
S3150801423893FBF2F2C2EBC2029B1A3A4955D50733E8
S31508014248A361A0F50E33A3F52C7393FBF1F1364B55
S3150801425840F2B45C03FB010048F6AC63B0FBF3F328
S31508014268B0FBFCF203449B1A304A40F26D17B0FBC7
S31508014278F2F29B1AB3FBF7F26426B3FBFCF3B2FB23
S31508014288F6F5EB1A0344992007FB123303EB830768
S315080142980237B7FBF0FC4FF0050800FB0CF00230BB
S315080142A8B0FBF8F003F1010EAEEB000040F2F95E3F
S315080142B877458CBF6FF00907022767444FF4C87C16
S315080142C80CFB0121012F98BF0131B3F5997F12D350
S315080142D8A3F59973E3610023A1F26C71E060C4E95F
S315080142E8047120462362BDE8F0810028A361A8DB92
S315080142F890FBF1F1ABE712F0030F02D106FB152586
S315080143085DB94FF4C875B2FBF5F605FB1622B2FA84
S3150801431882F252093B331344DCE70122FAE700BF6C
S3150801432880510100B13A02004FC5FDFFB03A0200BB
S31508014338014B1868704700BF9000002070B5002629
S315080143480C4D0D4C641BA410A64209D102F004F9C0
S3150801435800260A4D0A4C641BA410A64205D170BD55
S3150801436855F8043B98470136EEE755F8043B984754
S315080143780136F2E7447101084471010844710108DC
S315080143884871010870477047704700000048704730
S31508014398D0010020034610B5C9B202449342184613
S315080143A801D1002003E0047801338C42F6D110BD0F
S315080143B80A44914200F1FF3300D1704710B511F84C
S315080143C8014B914203F8014FF9D110BD1FB51446A7
S315080143D81A46094B05461B68D8684CB1074BCDE9FF
S315080143E8013400912B46064901F01EFE01F0E4FF4F
S315080143F8044B1C46F3E700BF90000020136E010822
S31508014408206E01084E6E01082DE9F74F03690C69FC
S315080144180746A3427EDB013CA30000F1140501F11E
S315080144281408009305EB8403019358F8243055F8CA
S31508014438242001339A42B2FBF3F608EB84092ED3FA
S315080144484FF0000AC446AE46D3465CF8043B98B218
S3150801445806FB00A01B0C020C06FB0323DEF8002052
S3150801446880B292B2121A5A44DEF800004FEA134A89
S315080144789BB2C3EB224303EB104392B242EA0342CF
S31508014488E1454FEA234B4EF8042BDED2009BEB5845
S315080144982BB9019B043B9D421A462FD33C613846EA
S315080144A801F076FC002825DB2946002058F8042B5C
S315080144B8D1F800C01FFA82FE1FFA8CF3A3EB0E038C
S315080144C80344120CC2EB234202EB1C429BB243EA99
S315080144D80243C1454FEA224041F8043BE6D255F862
S315080144E8242005EB840322B9043B9D421A460BD3C3
S315080144F83C610136304603B0BDE8F08F1268043BCB
S31508014508002ACBD1013CC6E71268043B002AEFD141
S31508014518013CEAE70020EEE72DE9F04F14461D466F
S31508014528C76997B08146CDE90645239E7FB910200C
S3150801453801F05EF80246C9F81C0020B9EF21AC4B18
S31508014548AC48FFF743FFC0E901770760C760D9F8A8
S315080145581C30196859B15A68012393404A608B601F
S31508014568484601F0E3F90022D9F81C301A602B1ED7
S31508014578AFBF0023012223F000430793A8BF336086
S31508014588DDF81C809C4BB8BF326033EA080312D1A8
S3150801459842F20F73229A1360C8F31303234300F0F8
S315080145A85E85249BDFF854A2002B00F060850AF18A
S315080145B8030300F05ABDDDE90623CDE90C23DDE93D
S315080145C80C0100220023F4F757FA074658B10123CC
S315080145D8229A1360249B13B1894B249A1360DFF836
S315080145E824A200F044BD14AB019315AB00934846C9
S315080145F8DDE90C2301F07CFCC8F30A560390002E6A
S3150801460878D0DDE90C010D9BA6F2FF36C3F3130337
S3150801461843F07F5343F440131297194600227A4B05
S31508014628F3F70AFE6CA3D3E90023F3F7BDFF6CA3DE
S31508014638D3E90023F3F702FE044630460D46F3F79D
S3150801464849FF69A3D3E90023F3F7AEFF02460B46F0
S3150801465820462946F3F7F2FD04460D46F4F754FABF
S3150801466800220746002320462946F4F70FFA40B1E7
S315080146783846F3F72FFF22462B46F4F7FDF900B91A
S31508014688013F162F54D8DDE90C01604B03EBC7032C
S31508014698D3E90023F4F7FAF900284BD00023013FA0
S315080146A80F93149B9B1B5A1E49BFC3F10103002391
S315080146B804930023099254BF04930993002F3BDB03
S315080146C8099B0E973B44099300230A93209B092BC0
S315080146D865D8052BC4BF043B2093209BC8BF00247B
S315080146E8A3F10203D8BF0124032B64D8DFE803F03A
S315080146F85355382CDDE914631E4406F23243202B40
S31508014708C1BFC3F1400308FA03F806F2124324FAB3
S3150801471803F3D6BFC3F1200348EA030004FA03F0FA
S31508014728F3F7C8FE0122A1F1F873013E129274E764
S315080147380123B5E70F90B4E7049BDB1B04937B427F
S315080147480A9300230E93C1E701230B93219B07EBD9
S31508014758030B0BF10103012B0893B8BF012306E0EC
S3150801476801230B93219B002B28DD9B4608930021E7
S315080147780422D9F81C0002F114059D4226D9416084
S31508014788484601F093F88246002843D1024640F28A
S31508014798AF111F4BD4E60023E3E70023D5E701242D
S315080147A800230B9420934FF0FF3B00221223CDF8E8
S315080147B820B02192DBE701230B93F4E74FF0010BB5
S315080147C85B46CDF820B0CDF884B0D0E70131520068
S315080147D8D1E700BFAFF3008061436F63A787D23F74
S315080147E8B3C8608B288AC63FFB799F501344D33FC9
S315080147F8A46D01085C6E01080000F07F586E010877
S31508014808816D0108806D01080000F83F706F010885
S31508014818B46E0108D9F81C301860089B0E2B00F2F3
S31508014828A180002C00F09E80002F33DD9C4B07F0F9
S315080148380F0203EBC203F805D3E90034CDE91034B6
S315080148484FEA271416D5DDE90C01964B0326D3E959
S315080148580823F3F7D3FFCDE9060104F00F04914DB8
S3150801486854B9DDE91023DDE90601F3F7C7FFCDE9F8
S31508014878060128E00226F2E7E10708D5DDE9100175
S31508014888D5E90023F3F790FECDE910010136641046
S315080148980835E5E700F0AF80DDE90C017C42804B7D
S315080148A804F00F0203EBC203D3E90023F3F77CFEF6
S315080148B802260023CDE906017A4D2411002C40F081
S315080148C88F80002BD3D1DDE906450F9B002B00F01D
S315080148D89480002220462946734BF4F7D7F8002816
S315080148E800F08B80089B002B00F08780BBF1000F36
S315080148F834DD2046002229466C4BF3F755FE5C4603
S31508014908CDE9060107F1FF3801363046F3F7E2FD2E
S31508014918DDE90623F3F748FE0022654BF3F78EFC1B
S315080149280546A1F15076002C6AD1DDE90601002277
S31508014938604BF3F781FC02460B46CDE906232A4666
S315080149483346F4F7C1F8002840F09882DDE90601F4
S315080149582A4606F10043F4F799F838BBDDE90C3421
S31508014968CDE90634159B002BC0F257810E2F00F3AB
S3150801497854814B4B03EBC703D3E90034CDE904341F
S31508014988219B002B80F2E580089B002B00F3E18030
S315080149980CD1DDE904010022464BF3F705FEDDE9F2
S315080149A80623F4F787F8002800F0668200242546CE
S315080149B8219B56466FEA030800272146484600F018
S315080149C8B5FF002D00F0BD802FB1AF4203D039469F
S315080149D8484600F0ABFF2946484600F0A7FFB0E075
S315080149E8E20705D5D5E90023F3F7DEFD01230136EC
S315080149F86410083562E7022665E7B846089C84E725
S31508014A08274B0B9903EBC40353E9022354440029A2
S31508014A1854D000202849F3F7F1FE33462A46F3F71E
S31508014A280BFC5646CDE91001DDE90601F4F76CF8E9
S31508014A380546F3F74FFD02460B46DDE90601F3F78E
S31508014A48FBFB02460B463035CDE90623DDE9102383
S31508014A5806F8015BF4F71AF8002872D1DDE906238E
S31508014A6800201149F3F7E8FBDDE91023F4F70EF8FE
S31508014A78002840F0B480A6423FF470AFDDE9100182
S31508014A8800220A4BF3F790FD0022CDE91001DDE972
S31508014A980601064BF3F788FDCDE90601C4E700BF11
S31508014AA8706F0108486F01080000F03F00002440B4
S31508014AB800001C40000014400000E03F314628462B
S31508014AC8F3F772FD5646CDE910011394DDE906019F
S31508014AD8F4F71AF80546F3F7FDFC02460B46DDE935
S31508014AE80601F3F7A9FB02460B46303506F8015BC2
S31508014AF8A642CDE906234FF0000224D1DDE91001CB
S31508014B08AE4BF3F79BFB02460B46DDE90601F3F7C5
S31508014B18DBFF002863D1DDE910230020A749F3F755
S31508014B288BFB02460B46DDE90601F3F7AFFF0028C2
S31508014B383FF414AF139E731E139316F8013C302BDA
S31508014B48F8D047463BE09E4BF3F72EFDCDE9060123
S31508014B58BCE75646DDE90645DDE90423204629462C
S31508014B68F3F74CFEF3F7D0FF8046F3F7B3FCDDE91C
S31508014B780423F3F719FD02460B4620462946F3F79F
S31508014B885BFB08F13004089D06F8014BA6EB0A04FD
S31508014B98A54202460B4633D1F3F750FBDDE9042358
S31508014BA804460D46F3F790FFC0B9DDE9042320460C
S31508014BB82946F3F761FF10B118F0010F0ED14846DF
S31508014BC8039900F0B3FE00233370229B01371F6057
S31508014BD8249B002B00F04B821E6048E2B8463346F8
S31508014BE81E4613F8012D392A06D19A45F8D13022DD
S31508014BF808F101088AF800201A7801321A70A0E724
S31508014C0800226F4BF3F7D0FC0022002304460D4619
S31508014C18F3F732FF00289FD0D1E70B9A002A00F054
S31508014C28EA80209A012A00F3CD80129A002A00F018
S31508014C38C18003F233430A9C049E049A01211A444B
S31508014C480492099A48461A44099200F023FF054630
S31508014C5866B1099B002B09DDB342A8BF3346049AFE
S31508014C68F61AD21A0492099AD31A09930A9B0BB30C
S31508014C780B9B002B00F0C680002C00F0C08029464B
S31508014C882246484600F0BEFF039A014605464846AD
S31508014C9800F016FF03998046484600F047FE0A9B2E
S31508014CA81B1B0A9300F0B18041460A9A484600F050
S31508014CB8A9FF03900121484600F0ECFE0E9B044625
S31508014CC8002B00F0D8811A460146484600F09AFF9B
S31508014CD8209B0446012B00F39F80069B002B40F07E
S31508014CE89780079BC3F31303002B40F09380079B18
S31508014CF823F000431B0D1B0533B1049B01330493B1
S31508014D08099B0133099301230A930E9B002B00F093
S31508014D18B881236904EB8303186900F06FFEC0F1B3
S31508014D282000099B184410F01F0000F08280C0F18A
S31508014D382003042B73DD049BC0F11C000344049370
S31508014D48099B064403440993049B002B05DD1A466F
S31508014D584846039900F0B0FF0390099B002B05DD2F
S31508014D6821461A46484600F0A7FF04460F9B002B22
S31508014D7861D02146039801F00BF800285BDA002375
S31508014D880A224846039900F0F3FD0B9B07F1FF3801
S31508014D980390002B00F07781294600230A2248460A
S31508014DA800F0E6FDBBF1000F05466FDC209B022BE0
S31508014DB849DC6BE0149BC3F136033CE70000E03F8E
S31508014DC800002440089B5C1E0A9BA34209DB1C1BA6
S31508014DD8089B002BBFF630AF049B089A9E1A00233E
S31508014DE82BE70A9B0E9AE31A1A440A94049E00248E
S31508014DF8089B0E9221E70A9C049E0B9D28E7DDF87D
S31508014E080C8051E70A9A039950E7CDF80C8051E7C7
S31508014E18002379E7069B77E700230A9379E793D076
S31508014E28049A1C331A440492099A1E441A4409928C
S31508014E388AE70346F4E7089BB846002B20DC9B461D
S31508014E48209B022B1EDDBBF1000F7FF4B1AD214675
S31508014E585B460522484600F08BFD01460446039841
S31508014E6800F096FF00287FF7A3AD5646312308F1CF
S31508014E78010806F8013B9FE5B846089C2546F4E76C
S31508014E88DDF820B00B9B002B00F00181002E05DD13
S31508014E9829463246484600F00FFF05460A9B002B6D
S31508014EA85CD04846696800F001FD064628B90246FD
S31508014EB840F2EF21804BFFF743BB2A6905F10C0144
S31508014EC8023292000C30FFF773FA0122314648463E
S31508014ED800F0F2FE2F4605460AF1010304930AEB90
S31508014EE80B030A93069B03F001030993049B2146C6
S31508014EF8039803F1FF3BFFF787FA03463946303330
S31508014F08069003980B9300F043FF2A46089021461A
S31508014F18484600F059FFC26806460B9B02BB014684
S31508014F28039800F035FF02460B9B31464846CDE902
S31508014F380B3200F0FBFC209B0C9A049E42EA030103
S31508014F48099B19430B9B0DD1392B27D0089A002A9F
S31508014F5801DD069B31338BF800302EE52846B9E783
S31508014F680122E2E70899002904DB209801430998F8
S31508014F78014320D1002AEEDD01220399484604930C
S31508014F8800F09AFE2146039000F002FF0028049BD0
S31508014F9802DCE0D1DA07DED5392BDAD139238BF8E9
S31508014FA8003033461E4616F8012C013B392A4ED0E5
S31508014FB801321A7001E5002A03DD392BEED00133D7
S31508014FC8C9E7049A0A9902F8013C8A4228D00023BB
S31508014FD80A220399484600F0CBFCAF4203904FF0EA
S31508014FE800034FF00A023946484607D100F0C0FCCB
S31508014FF807460546049B0133049377E700F0B8FC96
S315080150082946074600230A22484600F0B1FC054608
S31508015018F0E7BBF1000FCCBF5E46012600275644D0
S31508015028012203994846049300F046FE2146039057
S3150801503800F0AEFE0028B4DC02D1049BDB07B0D42D
S3150801504833461E4613F8012D302AFAD0B5E49A4597
S31508015058A8D1312308F101088AF80030ADE4249B68
S31508015068DFF858A01BB10AF10803249A13605046C1
S3150801507817B0BDE8F08F209B012B7FF72EAE0E9B4C
S315080150880A9301204DE6BBF1000F7FF7D9AE5646C4
S3150801509821460398FFF7B8F900F1300306F8013BF2
S315080150A8A6EB0A029345B4DD00230A22484603996A
S315080150B800F05EFC0390EBE7B46E01084F6E010839
S315080150C82DE9F0471F468E688246BE420C46904631
S315080150D80B682DD8B1F90C2012F4906F26D06569A2
S315080150E8096905EB4505A3EB010905EBD5757B1C94
S315080150F84B446D109D4238BF1D46530527D5294691
S3150801510800F0A0FA064660B34A462169FFF750F946
S31508015118A38923F4906343F08003A38126614E444F
S3150801512826603E466561A5EB0905A560BE4200D91C
S315080151383E4632464146206801F0ABF80020A3688E
S315080151489B1BA360236833442360BDE8F0872A467E
S3150801515800F07CFF06460028E0D15046216901F097
S3150801516847F90C23CAF80030A3894FF0FF3043F0FA
S315080151784003A381E9E700002DE9F04F98468B899A
S3150801518807461B060D4614469DB010D50B6973B91B
S31508015198402100F057FA2860286130B90C233B6092
S315080151A84FF0FF301DB0BDE8F08F40236B61002337
S315080151B8099320238DF8293030234FF00109CDF8BA
S315080151C80C80DFF898818DF82A3023469A4613F819
S315080151D8012B0AB1252AF9D1BAEB040B0BD05B4688
S315080151E8224629463846FFF76BFF013000F0A780AB
S315080151F8099A5A4409929AF80030002B00F09F80C0
S3150801520800234FF0FF32CDE905230AF1010A049379
S3150801521807938DF853301A935446052214F8011B3F
S315080152284E48FFF7B7F8049AD8B9D00644BF2023E1
S315080152388DF85330110744BF2B238DF853309AF84C
S3150801524800302A2B15D0544600204FF00A0C079A2D
S31508015258214611F8013B303B092B4BD9B0B10792CE
S3150801526814E0A0EB080309FA03F31343A2460493CF
S31508015278D2E7039B191D1B680391002BBBBF5B4231
S3150801528842F0020207930793B8BF049223782E2B9C
S315080152980AD163782A2B32D1039B02341A1D1B685B
S315080152A8039243EAE3730593DFF8B4A00322504651
S315080152B82178FFF76FF838B14022049BA0EB0A0062
S315080152C8824013430134049314F8011B0622254826
S315080152D88DF82810FFF75EF8002836D0224B1BBB3D
S315080152E8039B073323F0070308330393099B3344C6
S315080152F809936AE70C4601200CFB0232A8E700234A
S315080153084FF00A0C194601340593204610F8012B6B
S31508015318303A092A03D9002BC6D00591C4E70446B1
S3150801532801230CFB0121F0E703AB00932A46384613
S315080153380E4B04A9FEF762FA421C0646D6D1AB897A
S315080153485B063FF52DAF09982CE703AB00932A4670
S315080153583846064B04A9FEF7EFFCEDE7C56E0108CA
S31508015368CB6E0108CF6E010805380108C950010836
S31508015378936810B4013B002B936007DA9469A3423A
S3150801538801DB0A2902D110BC00F08EBE1368581C2D
S3150801539810601970084610BC7047F8B506460F46DE
S315080153A81446D518AC4201D1002007E03A463046E2
S315080153B814F8011BFFF7DCFF431CF3D1F8BD000005
S315080153C82DE9F04F0D461446984606469DB018B184
S315080153D8036A0BB9FEF75AFE6B6ED90705D4AB8972
S315080153E89A0502D4A86DFEF7CEFFAB891B0701D52E
S315080153F82B699BB92946304600F094FE70B16B6E4D
S31508015408DC0704D54FF0FF301DB0BDE8F08FAB8936
S315080154189805F7D4A86DFEF7B7FFF3E700230993B4
S3150801542820238DF8293030234FF00109CDF80C8057
S31508015438DFF8A8818DF82A3023469A4613F8012BF6
S315080154480AB1252AF9D1BAEB040B0BD05B462246D9
S3150801545829463046FFF7A1FF013000F0A780099ACF
S315080154685A4409929AF80030002B00F09F800023CD
S315080154784FF0FF32CDE905230AF1010A0493079390
S315080154888DF853301A935446052214F8011B5348CC
S31508015498FEF780FF049AD8B9D10644BF20238DF8B0
S315080154A85330130744BF2B238DF853309AF800302D
S315080154B82A2B15D0544600204FF00A0C079A214684
S315080154C811F8013B303B092B4BD9B0B1079214E0CF
S315080154D8A0EB080309FA03F31343A2460493D2E798
S315080154E8039B191D1B680391002BBBBF5B4242F046
S315080154F8020207930793B8BF049223782E2B0AD181
S3150801550863782A2B32D1039B02341A1D1B6803922E
S3150801551843EAE3730593DFF8C8A0032250462178C6
S31508015528FEF738FF38B14022049BA0EB0A008240F7
S3150801553813430134049314F8011B062229488DF8EC
S315080155482810FEF727FF00283FD0274B1BBB039BD4
S31508015558073323F0070308330393099B3B4409934D
S315080155686AE70C4601200CFB0232A8E700234FF034
S315080155780A0C194601340593204610F8012B303ACE
S31508015588092A03D9002BC6D00591C4E70446012385
S315080155980CFB0121F0E703AB00932A463046134B6F
S315080155A804A9FEF72BF90746781CD6D16B6ED907DD
S315080155B805D4AB899A0502D4A86DFEF7E5FEAB8931
S315080155C85B063FF51FAF09981EE703AB00932A460A
S315080155D83046064B04A9FEF7AFFBE4E7C56E01089A
S315080155E8CB6E0108CF6E010805380108A3530108D7
S315080155F8024B0146186800F025B800BF9000002044
S3150801560870B50F4E0C463168054611B900F090FE83
S3150801561830602146284600F08BFE431C03D14FF023
S31508015628FF34204670BDC41C24F00304A042F8D0F8
S31508015638211A284600F07CFE0130F2D1EFE700BFB7
S31508015648D01100202DE9F843CD1C25F003050835AE
S315080156580C2D38BF0C25002D064601DBA94204D9B5
S315080156680C2333600020BDE8F883DFF8D48000F006
S3150801567811F9D8F800301C4644BB29463046FFF7CD
S31508015688BFFF431C044658D1D8F800402746002FC7
S3150801569843D1002C4BD023683946304604EB03091D
S315080156A800F046FE814542D1216830466D1A2946E1
S315080156B8FFF7A6FF01303AD023682B442360D8F8B0
S315080156C800305A6862BBC8F800700FE02268521B9E
S315080156D820D40B2A17D96119A342256018BF596026
S315080156E8636808BFC8F8001062514B60304600F07D
S315080156F8D7F804F10B00231D20F00700C21A1CBFB6
S315080157081B1AA350AFE76268A3420CBFC8F800206A
S315080157185A60EBE723466468AEE73C467F68B6E716
S315080157281A465B68A342FBD100235360DEE70C23C4
S315080157383046336000F0B4F894E70560D6E700BF51
S31508015748D4110020B1F90C20F8B5160705460C4600
S3150801575854D44B68002B02DC0B6C002B48DDE66A37
S31508015768002E45D0002312F480522F68216A2B6037
S3150801577830D0626DA389590705D56368D21A636B58
S315080157880BB1236CD21A00232846E66A216AB04768
S31508015798431CA38906D129681D292BD8284ACA403A
S315080157A8D60727D5002262602269D904226004D562
S315080157B8421C01D12B6803B96065616B2F60B9B1C9
S315080157C804F14403994202D0284600F011FE002349
S315080157D863630DE001232846B0470246501CC9D128
S315080157E82B68002BC6D01D2B01D0162B1DD12F6077
S315080157F8002021E043F040031BB21AE00F69002F8D
S31508015808F6D0930718BF00230E6808BF4B69F61B25
S315080158180F608B60002EEBDD33463A462846216A2F
S31508015828D4F828C0E047002807DCB4F90C3043F05F
S3150801583840034FF0FF30A381F8BD0744361AE9E75C
S315080158480100402038B50B6905460C4613B90025F1
S31508015858284638BD18B1036A0BB9FEF717FCB4F91F
S315080158680C30002BF3D0626ED00704D4990502D404
S31508015878A06DFEF788FD28462146FFF763FF636E8C
S315080158880546DA07E4D4A3899B05E1D4A06DFEF79A
S315080158987BFDDDE70148FEF776BD00BFCC11002088
S315080158A80148FEF771BD00BFCC11002070B5C66965
S315080158B804460D4676B91020FFF79AFE0246E061BE
S315080158C820B96B21174B1848FEF780FDC0E9016618
S315080158D80660C660E669F36883B1E369DB6853F86D
S315080158E82500B8B9012101FA05F6721D204692006C
S315080158F800F069FD60B1C0E901560EE021220421D4
S31508015908204600F060FDE369F060DB68002BE4D10E
S31508015918002070BD026843F825200023C0E9033337
S31508015928F7E700BFA46D0108D66E010870B5C66908
S3150801593805460C4676B91020FFF75AFE0246E86175
S3150801594820B98F21084B0948FEF740FDC0E90166D1
S315080159580660C6603CB1EB696268DB6853F82210D9
S31508015968216043F8224070BDA46D0108D66E01086E
S315080159782DE9F04107460C461E4600200D6901F13E
S31508015988140CDCF80030013099B202FB01611E0CD7
S315080159980B0C02FB063389B201EB034185424FEA38
S315080159A813464CF8041BECDC0EB3A368AB4219DCAE
S315080159B8616838460131FFF779FF804628B90246FA
S315080159C8BA210C4B0C48FEF701FD226904F10C01BA
S315080159D8023292000C30FEF7EBFC21463846FFF7F7
S315080159E8A5FF444604EB850301355E61256120461A
S315080159F8BDE8F081B46E0108D66E01080346B0F514
S31508015A08803F3ABF030410200020B3F1807F3CBFD2
S31508015A181B020830B3F1805F3CBF1B010430B3F1A8
S31508015A28804F3CBF9B000230002B05DB13F0804FEB
S31508015A3800F1010008BF202070470368024613F0E9
S31508015A4807000BD0D90721D4980749BF5B089B08DB
S31508015A58012013605CBF02201360704799B209B927
S31508015A6810201B0CD9B209B908301B0A190704BF3B
S31508015A781B090430990704BF9B080230D90703D4C8
S31508015A885B0800F1010003D01360704700207047D6
S31508015A982020704710B50C460121FFF707FF02467B
S31508015AA828B940F24511044B0448FEF78FFC012337
S31508015AB84461036110BD00BFB46E0108D66E0108C2
S31508015AC82DE9F04F17460A693B6989469A42A2BFEA
S31508015AD83B460F4699463D69D9F810A0BB687968CF
S31508015AE805EB0A06B34285B0B8BF0131FFF7DEFEFA
S31508015AF830B902464FF4B171404B4148FEF766FC8E
S31508015B0800F114042346002204EB860E734520D3BC
S31508015B1807F1140809F1140108EB850501EB8A0355
S31508015B280293EB1B153B23F0030304331537BD42D8
S31508015B3838BF04230193029B03918B420CD8002E8C
S31508015B4803DD5EF8043D002B55D0066105B0BDE8B6
S31508015B58F08F43F8042BD9E7B1F800A0BAF1000F82
S31508015B681FD0C446A14600275CF8042BD9F8003093
S31508015B781FFA82FB9BB20AFB0B333B44D9F8007028
S31508015B88120C3F0C0AFB027202EB13429BB243EA60
S31508015B98024365454FEA124749F8043BE4D8019B95
S31508015BA8E750039B0431B3F80290B9F1000F20D0EE
S31508015BB84746A4464FF0000A2368B7F800B0BCF870
S31508015BC802209BB209FB0B22524443EA02434CF8D2
S31508015BD8043B57F8043B4FEA134ABCF80030BD4268
S31508015BE809FB0A3303EB12434FEA134AE5D8019A2C
S31508015BF8A35004349FE7013EA1E700BFB46E01082C
S31508015C08D66E01082DE9F843154612F00302074630
S31508015C180E4607D0254C013A002354F82220FFF7EF
S31508015C28A7FE0646AD103DD0FC697CB91020FFF7E2
S31508015C38DFFC0246F86128B940F2B3111C4B1D482E
S31508015C48FEF7C4FBC0E901440460C460D7F81C80A8
S31508015C58D8F808404CB940F271213846FFF71AFFBF
S31508015C6800230446C8F8080003604FF00009EB074B
S31508015C780AD5314622463846FFF722FF804631467D
S31508015C883846FFF753FE46466D100BD0206838B9DB
S31508015C98224621463846FFF713FF2060C0F80090D0
S31508015CA80446E4E73046BDE8F88300BF3C6F0108BF
S31508015CB8A46D0108D66E01082DE9F0470C4607467A
S31508015CC891462369496803EB6218A3684FEA621A81
S31508015CD808F10106B3420BDB3846FFF7E7FD05462F
S31508015CE848B902464FF4EF71274B2848FEF76EFB71
S31508015CF801315B00EEE7002300F1140100F11002FF
S31508015D081846534533DB20692AEAEA7A04F114036B
S31508015D1819F01F0901EB8A0103EB800C2BD08A467F
S31508015D280022C9F1200E186800FA09F010434AF84A
S31508015D38040B53F8042B9C4522FA0EF2F3D8ACEB64
S31508015D480403153B23F00303043304F115006045E6
S31508015D5888BF0423CA500AB108F10206013E38462B
S31508015D6821462E61FFF7E2FD2846BDE8F08742F88D
S31508015D78040F0133C5E7043953F8042B9C4541F848
S31508015D88042FF9D8EAE700BFB46E0108D66E0108F0
S31508015D9803460A69006930B5801A0ED114331431DD
S31508015DA803EB820401EB820154F8045D51F8042DD2
S31508015DB8954203D005D24FF0FF3030BDA342F3D345
S31508015DC8FBE70120F9E700002DE9F74F8946064662
S31508015DD8114648461446FFF7DBFF051E12D1294628
S31508015DE83046FFF763FD024628B940F237213E4B94
S31508015DF83E48FEF7EBFA0123C0E90435104603B01D
S31508015E08BDE8F08FBCBF4B46A1463046D9F8041009
S31508015E18BABF1C4601250025FFF748FD024618B9F1
S31508015E2840F24521304BE3E700F1140BD9F810701D
S31508015E3809F11003C5604FF0000C09F11405D9469C
S31508015E48266904F1140E05EB87080EEB86060193FD
S31508015E58019B5EF8040B53F804AF81B201931FFA4C
S31508015E688AF35B1A000C6344C0EB1A4000EB234023
S31508015E789BB243EA004376454FEA204C49F8043B6E
S31508015E88E6D8331B153B23F0030315340433A6421E
S31508015E9838BF04231D445B441E462C4644450ED38D
S31508015EA808F10301491B21F00301033DA84538BF41
S31508015EB800210B4453F8041D99B117619EE7E6467C
S31508015EC854F8041B1FFA81FCF444080C714400EBCE
S31508015ED82C4089B241EA00414FEA204C46F8041B96
S31508015EE8DCE7013FE6E700BFB46E0108D66E010894
S31508015EF82DE97343012190469946089EFFF7D6FC7A
S31508015F08044630B9024640F20F31234B2348FEF7BF
S31508015F185DFAC9F30A55C9F313030DB143F480139E
S31508015F280193B8F1000324D068460093FFF785FD6D
S31508015F38DDE90012D8B1C0F1200302FA03F30B43D5
S31508015F48C24063610192019B002B0CBF0122022208
S31508015F58A3612261ADB1A5F2334505443560C0F1A7
S31508015F683500099B1860204602B0BDE87083616157
S31508015F78E9E701A8FFF761FD019B0122636120306A
S31508015F88E7E7A0F2324004EB820330601869FFF7AD
S31508015F9835FDC0EB4210E4E7B46E0108D66E010878
S31508015FA810B50C46B1F90E1000F0B0F90028ABBFD0
S31508015FB8636DA3891B1823F48053ACBF6365A3815A
S31508015FC810BD2DE9F0411F468B890546DB050C46B0
S31508015FD8164605D502230022B1F90E1000F084F9F8
S31508015FE8A389324623F48053A38128463B46B4F94C
S31508015FF80E10BDE8F04100F0ABB910B50C46B1F981
S315080160080E1000F071F9431CA38915BF606523F4C6
S31508016018805343F48053A38118BFA38110BDB1F9F6
S315080160280E1000F0A7B900000EB403B5014603AB7C
S31508016038054853F8042B00680193FFF7C1F902B024
S315080160485DF804EB03B07047900000202DE9F04194
S31508016058074614460D4621B91146BDE8F041FFF732
S31508016068F1BA2AB900F0C4F925462846BDE8F081EF
S3150801607800F018FA8442064602D8B4EB500FF4D851
S3150801608821463846FFF7DEFA804608B94546ECE761
S31508016098B4422246294628BF3246FEF789F92946D7
S315080160A8384600F0A5F9F1E7F8B50E46144605464F
S315080160B818B1036A0BB9FDF7E9FFA369A360A389B8
S315080160C81A0701D5236943B92146284600F02AF853
S315080160D818B14FF0FF373846F8BD23682269F6B27A
S315080160E8981A63693746834205DC21462846FFF72D
S315080160F8A9FB0028EDD1A368013BA36023685A1CB4
S3150801610822601E706269431C9A4204D0A389DB0780
S31508016118E1D50A2EDFD121462846FFF793FB002849
S31508016128D9D0D6E738B5294B054618680C4618B1AB
S31508016138036A0BB9FDF7AAFFB4F90C30190722D47B
S31508016148DA0607D409222A6043F040034FF0FF30E4
S31508016158A38133E0580712D5616B41B104F14403B1
S31508016168994202D0284600F043F900236363A389BC
S3150801617823F02403A3810023636023692360A38989
S3150801618843F00803A38123694BB9A38903F4207350
S31508016198B3F5007F03D02146284600F03EF8B4F946
S315080161A80C3013F001020AD00022A2606269524239
S315080161B8A261226942B913F08000C5D138BD990791
S315080161C858BF6269A260F4E70020F7E7900000204B
S315080161D870B50C46B1F90E10154600291E4696B03B
S315080161E80CDAA389002113F0800F14BF40234FF45A
S315080161F88063002031602B6016B070BD6A4600F0D6
S31508016208C9F80028EDDB019901F47041A1F500539D
S31508016218594259414FF48063EBE78B89F7B59D07D6
S3150801622806460C4607D504F1470323602361012373
S31508016238636103B0F0BD6A4601ABFFF7C9FF009F6A
S31508016248054639463046FFF7FDF948B9B4F90C3021
S315080162589A05EED423F0030343F00203A381E2E788
S31508016268A389C4E9040743F08003A381019B20603D
S315080162785BB13046B4F90E1000F026F828B1A389A7
S3150801628823F0030343F00103A381A3891D43A581D1
S31508016298CFE7884210B501EB020402D984422346A6
S315080162A807D8431EA14208D011F8012B03F8012F7C
S315080162B8F8E7014602448A4200D110BD13F8014D98
S315080162C802F8014DF7E7000038B50023054D0446E5
S315080162D808462B60F7F749FF431C02D12B6803B11F
S315080162E8236038BDD811002038B50446084611463A
S315080162F80022054D2A601A46F7F741FF431C02D1C9
S315080163082B6803B1236038BDD811002038B5044677
S31508016318084611460022054D2A601A46F7F7EEFE89
S31508016328431C02D12B6803B1236038BDD81100205C
S3150801633838B50023054D044608462B60F7F72CFFA8
S31508016348431C02D12B6803B1236038BDD81100203C
S3150801635838B50446084611460022054D2A601A46EC
S31508016368F5F716F8431C02D12B6803B1236038BD2B
S31508016378D811002038B50023054D044608462B6078
S31508016388F7F7D9FE431C02D12B6803B1236038BD40
S31508016398D811002038B50023064D0446084611468B
S315080163A82B60F7F7D3FE431C02D12B6803B1236090
S315080163B838BD00BFD8110020062008B500F0B0F88E
S315080163C80120F7F790FE70B5A1FB025434B92946A6
S315080163D8FFF738F9064628B9304670BD0C2200265B
S315080163E80260F9E72A462146FDF7D4FEF4E70000DC
S315080163F838B50546002940D051F8043C0C1F002B36
S31508016408B8BFE418FFF746FA1C4A136833B963603C
S3150801641814602846BDE83840FFF742BAA34208D9AE
S31508016428206821188B4201BF19685B680918216021
S31508016438EDE71A465B680BB1A342FAD911685018F9
S31508016448A0420BD120680144501883421160E0D15B
S3150801645818685B68084410605360DAE702D90C23A8
S315080164682B60D6E7206821188B4201BF19685B683B
S315080164780918216063605460CBE738BDD411002040
S3150801648882B001B901A942B14BB113780B601278F0
S31508016498101E18BF012002B070471046FBE76FF0BF
S315080164A80100F8E751F8043C181F002BBCBF0B582C
S315080164B8C01870470346084641B1FF2A04D98A22FB
S315080164C84FF0FF301A60704701200A7070471F297C
S315080164D838B505460C4604D9162303604FF0FF3034
S315080164E838BDC26B12B152F821304BB9284600F0B3
S315080164F831F8224601462846BDE8384000F018B862
S31508016508012B0AD0591C03D1162303600120E7E79A
S315080165180021204642F8241098470020E0E70000A9
S31508016528024B01461868FFF7D2BF00BF900000204A
S3150801653838B50023064D0446084611462B60F7F779
S31508016548C2FD431C02D12B6803B1236038BD00BFC5
S31508016558D8110020F7F7B0BDF8B500BFF8BC08BCDC
S315080165689E467047F8B500BFF8BC08BC9E467047FA
S31508016578434F4E4E2564204572726F723A20256440
S315080165880A000000434F4E4E25642043686172672E
S31508016598696E672046696E69736865643A0A000018
S315080165A84368617267696E6720456E657267793AED
S315080165B82025640A0000000042484D2054696D658B
S315080165C86F75740A0000000050535520726561649E
S315080165D8792074696D656F75742C2073746F707082
S315080165E8696E672E2E2E0A00505355206F6E207439
S315080165F8696D656F75742C2073746F7070696E6731
S315080166082E2E2E0A0000000049736F6C6174696F9B
S315080166186E207761726E696E670A00004375727239
S31508016628656E74206C65616B6167652C20696E738C
S31508016638756C6174696F6E206572726F722C20733E
S31508016648746F7070696E672E2E2E0A005053552086
S315080166586F66662074696D656F75742C2073746F1F
S315080166687070696E672E2E2E0A000000455620693D
S315080166786E666F3A0A0000004742545F76657220D3
S315080166885625642E256425640A000000426174743F
S3150801669865727920747970653A2025640A000000C4
S315080166A8426174746572792063617061636974798A
S315080166B83A2025640A0000004261747465727920DB
S315080166C8766F6C746167653A2025640A00000000D4
S315080166D8426174746572792076656E646F723A20C0
S315080166E8252E34730A000000426174746572792094
S315080166F8534E3A20256C750A0000000042617474ED
S31508016708657279206D616E75666163747572652047
S31508016718646174653A20253032642E253032642E38
S31508016728253034640A000000426174746572792060
S315080167386379636C65733A2025640A004F776E207E
S315080167486175746F3A2025640A0000004556494E5A
S315080167583A20252E3137730A0000000045565F5343
S31508016768575F5645523A20252E38730A000000000D
S3150801677842524D2054696D656F75740A0000000010
S315080167884261747465727920696E666F3A0A000007
S315080167986D61784356202564560A00006D61784371
S315080167A843202564410A0000746F74452025646BEB
S315080167B857680A006D617854202564430A00000069
S315080167C8534F43202564700A00000000566F6C7405
S315080167D82E202564560A00004243502054696D65E7
S315080167E86F75740A0000000042524F2054696D659E
S315080167F86F75740A000000004556206E6F74207282
S315080168086561647920666F722061203630730A00E3
S31508016818505355206E6F742072656164792C207304
S31508016828746F7070696E672E2E2E0A0042434C2FBC
S315080168384243532F42534D2074696D656F75742C05
S315080168482073746F7070696E672E2E2E0A00000009
S315080168584C6F636B206572726F722C2073746F703C
S3150801686870696E672E2E2E0A00000000486F747034
S315080168786C75672064657465637465642C20737424
S315080168886F7070696E672E2E2E0A0000436F6E6E42
S315080168986563746F72206F76657268656174202501
S315080168A8642025642C2073746F7070696E672E2EA8
S315080168B82E0A00004253442054696D656F75740A9F
S315080168C80000000044697361626C65640A0000008F
S315080168D84368617267696E67207374617274656467
S315080168E80A00000057616974696E6720666F72202D
S315080168F842484D0A0000000057616974696E6720AD
S31508016908666F72205053552072656164790A0000D2
S3150801691849736F6C6174696F6E20746573740A00C4
S3150801692857616974696E6720666F7220626174744B
S3150801693865727920696E666F0A0000005761697485
S31508016948696E6720666F7220626174746572792050
S315080169587374617475730A0057616974696E67207F
S31508016968666F7220424D530A00000000496E697429
S3150801697869616C697A696E672063686172676572AD
S315080169880A00000057616974696E6720666F72208C
S3150801699842434C0A000000004368617267696E67E2
S315080169A820696E2070726F67726573730A0000003A
S315080169B84368617267696E672053746F707065649E
S315080169C80A0000004368617267696E672053746F2D
S315080169D8707065642077697468204353440A000017
S315080169E84368617267696E67204572726F720A0039
S315080169F84368617267696E672046696E6973686577
S31508016A08640A0000474254204572726F7220636F08
S31508016A1864653A20307825580A000000436F6E6E7F
S31508016A286563746F723A20556E6B6E6F776E0A00DE
S31508016A38436F6E6E6563746F723A20556E706C7526
S31508016A48676765640A000000436F6E6E6563746F55
S31508016A58723A2044697361626C65640A0000000031
S31508016A68436F6E6E6563746F723A20507265706112
S31508016A7872696E670A000000436F6E6E6563746F0C
S31508016A88723A204175746852657175697265640A46
S31508016A9800000000436F6E6E6563746F723A205783
S31508016AA8616974696E67466F72456E657267790AB8
S31508016AB800000000436F6E6E6563746F723A204377
S31508016AC868617267696E6750617573656445560AC8
S31508016AD800000000436F6E6E6563746F723A204357
S31508016AE868617267696E675061757365644556535F
S31508016AF8450A0000436F6E6E6563746F723A2043E8
S31508016B0868617267696E670A00000000436F6E6EF6
S31508016B186563746F723A204175746854696D656F57
S31508016B2875740A00436F6E6E6563746F723A204610
S31508016B38696E69736865640A00000000436F6E6EC2
S31508016B486563746F723A2046696E69736865644548
S31508016B585653450A00000000436F6E6E6563746FED
S31508016B68723A2046696E697368656445560A000073
S31508016B78436F6E6E6563746F723A205265706C75F1
S31508016B886767696E670A000042454D205265636565
S31508016B98697665642C20666F7263652073746F70F5
S31508016BA870696E672E2E2E0A0000000042454D3A7E
S31508016BB820253032582025303258202530325820A1
S31508016BC8253032580000000020253032582025305B
S31508016BD83258202530325820253032580A0000000C
S31508016BE84253542052656365697665642C2073742B
S31508016BF86F7070696E672E2E2E0A00004253543A3A
S31508016C082025303258202530325820253032582050
S31508016C1825303258000000004C6F636B206572728C
S31508016C286F720A004C6F636B206572726F722072FD
S31508016C38657365740A000000474254204368617207
S31508016C48676572207625642E25640A00536572697C
S31508016C58616C206E756D6265723A2025640A0000BA
S31508016C68426F617264207265766973696F6E3A203C
S31508016C7825640A0046572076657273696F6E3A204D
S31508016C8825642E25642E25640A00000050535520D4
S31508016C986F6E2074696D656F75740A00436F6E743B
S31508016CA86163746F72206572726F722C2073746FC8
S31508016CB87070696E672E2E2E0A00000050535520F3
S31508016CC86F66662074696D656F75740A0000000041
S31508016CD853657420436F6E6669673A2025732025C4
S31508016CE8640A0000506F776572206C696D69743A99
S31508016CF82025640A000000004368617267652070F0
S31508016D0865726D69743A2025640A0005E0930400E2
S31508016D180000000000000000010203040607080934
S31508016D28000000000102030400000405060708091B
S31508016D3800000000000D000001020304050607080B
S31508016D48090A0B0C0D0E0F100000040506070809A1
S31508016D5800000000000D00000102030405060708EB
S31508016D68090A0B0C0D0E0F10494E4600696E66008E
S31508016D784E414E006E616E00300030313233343583
S31508016D88363738394142434445460030313233347F
S31508016D983536373839616263646566005245454E4A
S31508016DA854206D616C6C6F632073756363656564E4
S31508016DB86564002F6275696C642F676E752D746F2B
S31508016DC86F6C732D666F722D73746D33325F313341
S31508016DD82E332E72656C312E3230323430393236D2
S31508016DE82D313731352F7372632F6E65776C69626A
S31508016DF82F6E65776C69622F6C6962632F74696D8A
S31508016E08652F676D74696D652E63002C2066756E2E
S31508016E186374696F6E3A2000617373657274696F7A
S31508016E286E2022257322206661696C65643A20669C
S31508016E38696C6520222573222C206C696E652025CC
S31508016E4864257325730A00496E66696E6974790043
S31508016E584E614E002F6275696C642F676E752D74C5
S31508016E686F6F6C732D666F722D73746D33325F3164
S31508016E78332E332E72656C312E3230323430393234
S31508016E88362D313731352F7372632F6E65776C69F5
S31508016E98622F6E65776C69622F6C6962632F7374EA
S31508016EA8646C69622F64746F612E630042616C6C4D
S31508016EB86F632073756363656564656400232D30A4
S31508016EC82B2000686C4C00656667454647002F62AB
S31508016ED875696C642F676E752D746F6F6C732D6683
S31508016EE86F722D73746D33325F31332E332E72659B
S31508016EF86C312E32303234303932362D313731351C
S31508016F082F7372632F6E65776C69622F6E65776C5E
S31508016F1869622F6C6962632F7374646C69622F6D79
S31508016F28707265632E63004300504F534958002E0B
S31508016F380000000005000000190000007D0000009F
S31508016F480080E03779C34143176E05B5B5B893464E
S31508016F58F5F93FE9034F384D321D30F94877825A1A
S31508016F683CBF737FDD4F1575000000000000F03F38
S31508016F7800000000000024400000000000005940FD
S31508016F880000000000408F40000000000088C34050
S31508016F9800000000006AF8400000000080842E41C5
S31508016FA800000000D01263410000000084D7974111
S31508016FB80000000065CDCD41000000205FA0024217
S31508016FC8000000E876483742000000A2941A6D428C
S31508016FD8000040E59C30A2420000901EC4BCD6427F
S31508016FE800003426F56B0C430080E03779C341432A
S31508016FF800A0D8855734764300C84E676DC1AB43A0
S31508017008003D9160E458E143408CB5781DAF1544BD
S3150801701850EFE2D6E41A4B4492D54D06CFF0804498
S31508017028F64AE1C7022DB544B49DD9794378EA44AD
S315080170380020202020202020202028282828282031
S315080170482020202020202020202020202020202029
S315080170582088101010101010101010101010101091
S315080170681004040404040404040404101010101081
S31508017078101041414141414101010101010101014B
S31508017088010101010101010101010101101010109D
S31508017098101042424242424202020202020202021D
S315080170A80202020202020202020202021010101071
S315080170B82000000000000000000000000000000099
S315080170C800000000000000000000000000000000A9
S315080170D80000000000000000000000000000000099
S315080170E80000000000000000000000000000000089
S315080170F80000000000000000000000000000000079
S315080171080000000000000000000000000000000068
S315080171180000000000000000000000000000000058
S315080171280000000000000000000000000000000048
S309080171380000000044
S30D0801713CEC10FF7F01000000C1
S309080171440D820008A1
S30908017148E9810008C2
S3150801714CE4010000010164000000FF0000000000DA
S3150801715C0000000000000000400000320A32004026
S3150801716C00000000008000320A3200008000000096
S3150801717C0000FA320A32000000FA000000FF003261
S3150801718C0A32000020000000FFFFFF320A3200FF1E
S3150801719CFFFF0000FF0000320A3200200000000049
S315080171AC00FFFF00000000000000000052555301CB
S315080171BC000000FE529E66000024F4001000000038
S315080171CC01000000000000000300000090100020E0
S315080171DC940000200000000090100020F8100020F8
S315080171EC60110020000000000000000000000000F3
S315080171FC0000000000000000000000000000000074
S3150801720C0000000000000000000000000000000063
S3150801721C0000000000000000000000000000000053
S3150801722C4300000000000000000000000000000000
S3150801723C0000000000000000000000000000000033
S3150801724C43000000000000000000000000000000E0
S3150801725C0000000000000000000000000000000013
S3150801726C43000000000000000000000000000000C0
S3150801727C00000000000000000000000000000000F3
S3150801728C43000000000000000000000000000000A0
S3150801729C00000000000000000000000000000000D3
S315080172AC4300000000000000000000000000000080
S315080172BC00000000000000000000000000000000B3
S315080172CC4300000000000000000000000000000060
S315080172DC0000000000000000000000000000000093
S315080172EC4300000000000000000000000000000040
S315080172FC0000000000000000000000000000000073
S3150801730CBD64010889640108000000003870010891
S3150801731C376F01084E6E01084E6E01084E6E010854
S3150801732C4E6E01084E6E01084E6E01084E6E01082E
S3150801733C4E6E01084E6E0108FFFFFFFFFFFFFFFFB0
S3150801734CFFFFFFFFFFFF00000100415343494900BE
S3150801735C0000000000000000000000000000000012
S3150801736C0000000000000000000041534349490099
S3150801737C00000000000000000000000000000000F2
S3110801738C000000000000000000000000E6
S7050800E7D932
